:020000040000FA
:080000000002040000000000F2
:020000040000FA
:100400008F9121000E7F22000E0188000000000065
:100410000C00070080FD2C000100200011000700E7
:10042000000020000000E000020032000000020096
:10043000000000003ADD0200000000000040DA0089
:100440000000FE004440A900A0EA21000000E000F6
:100450000300320000002000A00188004440A800F2
:100460000000060091018800800078000000EB0089
:1004700015003700E280400032A0B4009101BA00BC
:10048000E280400032A0B4009102BA00E280400055
:1004900032A0B4000002EB00472BDE00F507B200EB
:1004A000602CE10004003A000059EB008301E900F0
:1004B000FDFF3E00040037006128E100010032002A
:1004C0000082EB00040007001101BA000200E00006
:1004D000E8FF3A00000006003159BA008301E90044
:1004E0000C0032002159BA008301E90008003200F3
:1004F0000400E00003003A00E280400032A0B400B3
:10050000F5FF370011D9BA008301E900FAFF3A007C
:100510008100E800E180400032A0B4000000060045
:1005200032FE0400000000008CFE04000000000009
:10053000DAFE04000000000064F304000000000084
:10054000E4F304000000000032F4040000000000A6
:10055000286A0400000000002A6A0400000000006D
:10056000366A040000000000D0AA04000000000069
:10057000D6AA040000000000ECAB0400000000005C
:10058000D4AA04000000000042AB040000000000F8
:10059000F0AB040000000000E0FC040000000000DC
:1005A00054FD040000000000B0FD04000000000045
:1005B000C4D9040000000000DED9040000000000DF
:1005C000F6D90400000000000EDA0400000000006C
:1005D00016DA04000000000026DA04000000000023
:1005E00068DA04000000000082DA04000000000065
:1005F000A4DA040000000000CADA040000000000D1
:1006000006DB0400000000002CDB040000000000FA
:100610005EDB04000000000084DB0400000000003A
:10062000D4DB040000000000DCDB0400000000005C
:10063000E4DB040000000000ECDB0400000000002C
:100640001EDA040000000000EEDB040000000000E1
:100650001ADC040000000000C09404000000000048
:10066000D894040000000000109504000000000071
:100670001695040000000000229504000000000010
:100680003295040000000000709504000000000096
:100690009095040000000000CE95040000000000CA
:1006A000EE950400000000004296040000000000E7
:1006B00062960400000000007C9604000000000028
:1006C000AE96040000000000E89604000000000060
:1006D0000E970400000000003E9704000000000098
:1006E0006C970400000000009A97040000000000CE
:1006F000C897040000000000F2970400000000000A
:100700000E9804000000000026970400000000007E
:100710001498040000000000469804000000000047
:100720007898040000000000AA980400000000006F
:10073000D698040000000000289904000000000082
:1007400036990400000000006C99040000000000CD
:10075000E2C7040000000000FCC704000000000025
:1007600006C804000000000024C8040000000000C7
:100770002CC804000000000034C804000000000081
:10078000C6C8040000000000E0C80400000000002B
:1007900004C904000000000038C904000000000083
:1007A00040C9040000000000AAC9040000000000C5
:1007B00042C90400000000004AC904000000000013
:1007C0006EC904000000000078C8040000000000AA
:1007D000CEC9040000000000F2C9040000000000BF
:1007E0001ECA040000000000A8CA040000000000A7
:1007F00062CA0400000000000040DA000000FE00B1
:100800001004B100030035009001B10001003C006C
:100810001000050000000500800078001104B10000
:10082000030035009101B10001003C000050A00020
:10083000000006001004B100070035009001B1006F
:10084000040034007000B100030035009001B100D5
:1008500001003C0010000500000005006900E100F7
:10086000040035006D00E100030034000002B10017
:100870000100320000000500100005000A00FA0027
:1008800080017800E20F500028003E00A0C48000E4
:10089000E10F500008003200802320000000E0003B
:1008A00005003200042320002523200046232000D9
:1008B0008001780004003700042220002522200057
:1008C0004622200083222000144090000004E00013
:1008D000040035008009EB00144090000074A00073
:1008E00010429800154090000028A30003003A0031
:1008F000154090000024A000904298008001EB0079
:1009000007003700154090000008A300FDFF3200EB
:1009100063C078000000FB00000B78008301E80052
:10092000828F5100F7FF3A000800370030002000A6
:10093000B0BF9F00C3BF9F00D1BF9F00E2BF9F0019
:100940006A80570000C0DA006FB997000200780093
:100950000080FA00000006002002E20004003D00D2
:100960002342AB00020032002302AB00FEFF320044
:100970000040DA00FEFF37000A00FA0011002000F4
:10098000B1BF9F00C0BF9F006A80570000C0DA005F
:100990004FB897000080FA00000006000A00FA0035
:1009A00051002000B1BF9F00C0BF9F006A80570068
:1009B00000C0DA005FB897000080FA00000006006F
:1009C0000A00FA00881F7800800178000000E0002B
:1009D00029003A00A0C48000E10F50000800320056
:1009E000802320000000E0000500320004232000E6
:1009F00025232000672320008001780004003700B1
:100A000004222000252220006722200083222000CB
:100A1000144090000004E000040035008009EB0061
:100A2000144090000074A000104298000002EB00F7
:100A30000C003700130A2000154478006140640060
:100A400002003A008301E900FBFF3A000402E800DB
:100A50009541780061C06100050032001700780000
:100A60008058780004035100820F5200F1FF3A00D1
:100A7000060051000800370020002000A0BF9F00A2
:100A8000B3BF9F00C1BF9F00D2BF9F006C805700C3
:100A900000C0DA005FB897004F0478000080FA00C9
:100AA00000000600889FBE0080047800B0C480006B
:100AB0000000E00003003A00100007000000E00022
:100AC0000A003500B0C480000900E00002003A00CE
:100AD0000004780006003700000478000900400098
:100AE000060007000000E00001003D000084EB006C
:100AF000080078004F04BE00000006008000780067
:100B00000000E00004003A0080892100B0C48800A1
:100B100001017800060037000081EB008091210080
:100B2000808F500002003E00B1C488000001EB003D
:100B30000200780000000600020AB900001BB9009C
:100B40000200B8008100420081004300000006005E
:100B5000889FBE008A9FBE00010578000100E0006A
:100B60000400350008003C000000E00020003200D6
:100B70000500370060001000E080180002003B0014
:100B800001F02C001A0037000004BE006011B8000C
:100B90006B0920000982CF00020039000882CF00D3
:100BA0000441B000694252000E00320008003B00D0
:100BB00082817100610164008904D1000884D3003E
:100BC0008B05E8000442E800F9FF3A000500370011
:100BD0000804440089844C008B05E9000442E900C4
:100BE000FBFF3A00840207000AF0A70001F0A00012
:100BF0004F05BE004F04BE0000000600889FBE00E7
:100C00008A9FBE008C1F7800A1020700A802330053
:100C100003866C006450E1002E0032006420E10085
:100C2000330032006150E1002F0032006120E1000A
:100C30003100320085855500EB07B0000900200027
:100C400008042000050037000804440089844C0093
:100C50000A0031000603430087834B000001530064
:100C600081815B00F8FF33000203BE000800A00092
:100C70000804440089844C00F6FF3900C639DD00C1
:100C80008301730001003200130020008904D100A9
:100C90000884D3000998A300050032000800A700CB
:100CA0000300A0008904D1000884D3008B05E8006C
:100CB0008904D1000884D3000001EB000281D20036
:100CC0004D02070001F0A1000CF0A70001F0A00008
:100CD000800237006420E100820232000801BE0079
:100CE0000200BE00F7FF37006120E1007D02320004
:100CF0006000B800F3FF37000000200001F8270073
:100D0000F0FF370003F0A200889FBE008A9FBE005C
:100D10008C1F78005E020700650233006450E1001A
:100D20004F0032006420E1005200320003826C0068
:100D300007003B000905D0000306D000820F5400D5
:100D40000C065D00020039000200320089017800C3
:100D5000030678008582550004003D000003FD0075
:100D60008103FD008502EA008B854200840F72003A
:100D700002003B0060001000E08018006011B80025
:100D80000005EB007A28E1000A003900060078002F
:100D9000C75DDD00F707B200878075002D003700C2
:100DA000828171000A017800610560008180D100B4
:100DB0000080D3008502E900F9FF3B0006044000F3
:100DC0008784480002003B0060041400E0841C009B
:100DD0000988A300070032008A81710082817100B6
:100DE000610164008904D1000884D3008B05E80008
:100DF000170037000978A30013003A000B00E00049
:100E0000130034008B05E9000804440089844C0079
:100E10000A4474000978A3000D003A000B00E000BA
:100E2000070034008B05E9000804440089844C0065
:100E300001003A000B0020000978A300F7FF320000
:100E40000001EB0002003700828171000A01780086
:100E5000E90107000CF0A70001F0A0001D02370017
:100E60006420E10002003A00838F6C001D02330011
:100E70000801BE000200BE0016023700F4FF2F007A
:100E80001B0237000400200019023700889FBE00B3
:100E90008A9FBE008C1F7800FD010700040233000A
:100EA00003866C006450E100240032006420E100FD
:100EB000270032006150E100220032006120E10091
:100EC000210032008B854200EB07B1000134B800ED
:100ED000003AB8000804420089844A00013AB80088
:100EE0000030B8008880400009014A000400330047
:100EF0000000400081804800020149008B05E900A4
:100F0000C909DD00830170000100320013002000D8
:100F1000C814DE004814DD004709DE001200B200EC
:100F2000C808DE0008847000B301070001F0A100CA
:100F30000CF0A70001F0A000E60137006120E100FD
:100F4000E80132000801BE000200BE00F7FF3700D2
:100F50006150E100FCFF3A00E20137000001BE00F1
:100F6000FE0107000470A70003F0A10003F8A3002E
:100F700013003A006509B100100032000900350085
:100F80006928E1000200350001002800000005008A
:100F900000004000818048008502E900FCFF3A0023
:100FA00000000600F88F4200050035008100D100E6
:100FB0000080D3008502E800FCFF3A000000060034
:100FC0008000EB00000005000001BE00E301070007
:100FD0000470A70003F0A1006509B10016003200FB
:100FE0000D0035006828E10006003500F0FF2F00F5
:100FF000F1FF27000300E00013003B000100280080
:101000000000050000004000818048008502E900E2
:10101000FCFF3A0008003700F88F420002003C0055
:101020008000EB00000005008100D1000080D300AB
:101030008502E800FCFF3A000300E00002003B00EC
:1010400060001000E0801800000006006022B80078
:10105000060220000000D0008180D2000482D2006D
:101060008582D2000000A0000202520083825A0052
:10107000030031000202420083824A000000A10006
:101080000603E900F3FF3A0000000600EFFF070047
:101090000400BE00000006000001EB00C4010700D0
:1010A000040032000200200003F8230001F0A60033
:1010B00015FF0700000006000001EB00BC0107005F
:1010C000040032000200200003F8230001F0A70012
:1010D0000CFF070000000600839F68000100E0008D
:1010E00002003D0060001000E08018000300E000F6
:1010F00002003D0060011100E0811900D3FF0700EC
:101100004F00E00002003B0060001000E08018008B
:1011100000000600889FBE008A9FBE008C1F7800DA
:101120000205BE000004BE000006EB00E00F500008
:10113000E08F5800E00F5900E08F590007003D0094
:101140006000B8006011B80008045000898458009D
:101150000A0559008B8559001C002000E00F520041
:10116000E08F5A00E00F5B00E08F5B0002003D0063
:101170000F0007000C00A2000800BE000A01BE001C
:10118000B20107000203BE000002BE000C00E00036
:1011900001003200060007000400BE000601BE0088
:1011A0004F0678004F05BE004F04BE000000060049
:1011B0006000B8006011B800040250008582580039
:1011C000060359008783590000000600881F780035
:1011D000000478005001BE004000BE000400400042
:1011E000858048000601490087814900009CBE00B7
:1011F0000294BE000400E1000588E1000690E100D1
:101200000798E10002003100680044001008E8007F
:101210004F04780000000600F4874700889FBE0056
:101220008A9FBE008C9FBE008E1F78000205BE0004
:101230000004BE00D4B79F00E5B79F00F6B79F003B
:1012400087BF9F000000EB00C0B79F00B0B79F00B2
:10125000A0B79F0090B79F0080B79F000D042000AB
:10126000BFB097004FB09700000140000000E000C1
:101270000F003D004F08DE0000007100C0B79F0066
:101280009E00070001003D0012002000A1000700A1
:1012900001003D0012002000A6000700B100070079
:1012A000B60007000F004000C8FF0700220037000B
:1012B0004F08DE0000067100CCB79F008F000700CA
:1012C00001003D00120020009200070001003D00D7
:1012D0001200200097000700A20007000FB297003D
:1012E0009FB297002FB39700BFB39700A9000700E4
:1012F0000000520081805A0002015B0083815B0084
:1013000080B79F0091B79F00A2B79F00B3B79F001F
:101310000007EB009F0007000020E10001A8E100AA
:1013200002B0E10003B8E100010031001E0020001E
:101330000E005600C0B79F004FB297000400E000B7
:101340000700350010002000010020006011B800E7
:1013500008047000898470000A0571008B85710093
:101360008D06E900BEFF3A000400E00003003D00E6
:10137000820007000F00400094FF07004FA897006D
:101380000000E00004003A000FB497009FB49700FB
:101390002FB59700BFB59700940007004F0778005E
:1013A0004F06BE004F05BE004F04BE004F01B10006
:1013B00000000600881F780018002000881F7800B1
:1013C00095FF07008F87E9004F04780000000600B2
:1013D000801FEB0090FF07008F87E90000000600E8
:1013E000889FBE008A9FBE008C1F78006E00070099
:1013F00007003D0073000700E00F5B00E08F5B001B
:1014000007003D00320007000006EB000400370033
:101410003400070002003D002A0007001C002000E5
:1014200072000700E3FF07000203BE000002BE00D7
:101430000C00E00001003200220007000400BE00A2
:101440000601BE004F0678004F05BE004F04BE00E7
:1014500000000600889FBE008A9FBE008C1F780097
:101460005100070005003D0056000700E00F5B003B
:10147000E08F5B0006003D00040037001900070004
:1014800003003D006000B8006011B80010000700C4
:1014900056000700CEFF07000203BE000002BE0098
:1014A0000C00E00001003200060007000400BE004E
:1014B0000601BE004F0678004F05BE004F04BE0077
:1014C000000006006000B8006011B800000037009E
:1014D0000402500085825800060359008783590092
:1014E000000006000006EB00E00F5200E08F5A00FB
:1014F000E00F5B00E08F5B00000006000180400011
:1015000090B79F000001EB008FB097000100E00052
:10151000000006000200700090B79F0001804000AC
:1015200080B79F000001EB00FFA897000100E000DA
:10153000000006000200700080B79F00018040009C
:101540006FAA9700CF20DE0001007000F0AF9F006F
:1015500004024200250007004F18DE00000272005E
:1015600000000600E4AF9F000804440089844C009A
:101570000A054D008B854D00000006003FB2970024
:10158000CFB297005FB39700EFB3970000FE2F0034
:10159000000006003FB09700CFB097005FB1970002
:1015A000EFB19700000006000205BE000004BE0077
:1015B000E00F5000E08F5800E00F5900E08F590015
:1015C000000006006000B8006011B8000804500078
:1015D000898458000A0559008B8559001C00200099
:1015E000E00F5200E08F5A00000006000800BE0025
:1015F0000A01BE0000000600810020006180550045
:101600000B003D000B00200061FE2F000100E100F7
:101610001D00340082817100610164008904D100E1
:101620000884D3000000E800FAFF3A0071002000AF
:1016300061006400030070000200600009003200D5
:1016400061044400E0844C000988A50005003200D4
:101650008B05E8006808E10002003A008904D10027
:101660000884D300F20F20000258E10005003D007D
:10167000C75DDD00F907B2008980750008007800B9
:10168000000006000BF827008B0078000000050022
:101690000004BE00310007000003BE000405BE00C8
:1016A0000200BE002D000700844F750000000600F8
:1016B0000200BE006450E100050036006420E10035
:1016C000020036000968A30001003A000800BE00CD
:1016D0000160A0004F0678004F05BE004F04BE0019
:1016E00000000600F0FF2F00F1FF2700F9FF370090
:1016F000889FBE008A9FBE00841F7800E4FF070019
:101700004F00780011003300F0FF2F00838F6C0032
:1017100006003B00040565000A00A700080037002A
:1017200009F0A6001000200008003700820F5400C6
:10173000838F5C00030039001000200001003E0090
:101740000000200009F0A7000000EA004F05BE00DD
:101750004F04BE000000E00000000600C70ADE00E3
:10176000F107B200F50FB20008003200E1CF4200ED
:10177000020032000170A00024000500810F7000FB
:10178000010032000408050044000500810F7000CC
:1017900002003A00140005008502E9000000400044
:1017A00081C04800FCFF3B000170A0002400050040
:1017B000889FBE008A9FBE000003BE00E7FF0700AF
:1017C0008505780082815200020020006220E1003D
:1017D00004003A00F307B100040035007718E10077
:1017E000040035000600BE00140037006000B80099
:1017F0000F003700F50F2000FAFF2F008502D100FF
:101800000A85D3008301E900FCFF3B00818462006C
:1018100000046500890F7400F2FF32008582EA003F
:101820000A85EA00818462000004650072FF0700F7
:1018300007F0A70001F0A0000081EB000200E0002B
:101840004F05BE004F04BE0000000600889FBE008A
:101850008A9FBE008C9FBE000404B8000506B80035
:101860008904460060854E000606B8000A05460059
:10187000E0854E000706B8008B054600040EB80050
:10188000890446000A854E00E0854D00050EB8002B
:101890000A0546008B854E00060EB8008B054600F3
:1018A0000416B8000A0546008B854E000516B800E0
:1018B0008B054600041EB8008B0546000800BE00DC
:1018C0000A01BE004F06BE004F05BE004F04BE0019
:1018D000000006000400FA00E0BF9F00E48157000A
:1018E000812978000002EB000F0037006FB89700E5
:1018F000904078007FB89700104078000402E8001C
:1019000080CF5000040032008180FB000080FB008B
:1019100000805000070037006FB897000000E80013
:10192000E0BF9F009309E800820F5200EFFF3A00EA
:101930000000EB000080FA00000006001041780073
:10194000B141510003003A000000E8000204E00049
:10195000FAFF3A000300FB00000006008001780057
:101960000001780031407800005978000004E00060
:10197000FCFF3A000300780000000600889FBE00CC
:101980000004BE00060037000804E8000000FB0069
:1019900089007800F0000700E10F400004003200E9
:1019A000184078000004E000F7FF3A000000EB0068
:1019B0004F04BE0000000600881F78000186210049
:1019C000EEFF07000004780001862100A00020003F
:1019D000E1000700080078004F04780000000600CE
:1019E0000000FA00CFB897006881570000862100F8
:1019F000200107000080FA00000006008001EB00D3
:101A000002003700817178008301E800828F510065
:101A1000FCFF3A00000006000000FA00CFB8970073
:101A200068815700130107000080FA0000000600DB
:101A3000810178000000E9000081EB00E50F500013
:101A400004003E0080004000808721006081780013
:101A500003B0780002007800000006000001780062
:101A60000000E900E50F50000F003E00800040003C
:101A700080872100E08078000100E00002003A0049
:101A800010002000B0030700E18F40000600320084
:101A90000000EB00E18F50000400320002007800EB
:101AA00001000100000005000080EB0000000600BE
:101AB00010002000E9FF070010002000A20307002B
:101AC0008002780080017800010037008301E8007F
:101AD0001304E000FDFF3A000002EB00820F520009
:101AE0000600320064C07800805978000402E800E3
:101AF0000004E00002003200F8FF37008049EB00EC
:101B000005007800000006000C00FA00889FBE0067
:101B100000047800CFB09700F0FF2700D0BF9F00EF
:101B20008004EB0099BF9F0088BF9F00A8BF9F0063
:101B3000200C2000B0BF9F007881570070805700B4
:101B4000CC0007000FB89700094878000FB897003D
:101B500008045000080078004F04BE000080FA001E
:101B600000000600810178000002EB000B00370046
:101B7000E44078000104E000030032000402E800C1
:101B800093CF5000040032008180FB001380FB00E3
:101B900000805000000006008301E800820F520020
:101BA000F3FF3A00000005000C00FA00A0BF9F0000
:101BB000C0BF9F000A000700B0BF9F00F0BF9F009A
:101BC000100C2000D0BF9F0074815700EFB0970029
:101BD0006C8057008C0307000080FA0000000600AC
:101BE000800078003004E000FEFF3A000100500061
:101BF0000000E9000000060010417800814F51000C
:101C0000040032000000E8000204E000FAFF3A009D
:101C10000000EB00000006008001EB00020037002E
:101C200061F079008301E800828F5100FCFF3A00E7
:101C300000000600889FBE008A9FBE0080007800DA
:101C400000C2B300010037008900780081047800E9
:101C500039447800804F5400FBFF3200E94F5400B4
:101C6000F9FF3200D0C2B300804F540004003A00A4
:101C7000194478008184E8001AC0B30006003700D8
:101C80000045EB00B0C2B300804F540002003A00A0
:101C9000194478008184E8006022B8000A00370007
:101CA000A2002000030020000400BE00A2FB0700E9
:101CB0000B4144000281FB000300200000024100B0
:101CC00081824900394478000880FB000BFD2F0019
:101CD0000B004000E90F5000F1FF36000A04E0005D
:101CE0000200320060021200E0821A000400BE000E
:101CF0004F05BE004F04BE00000006000003780040
:101D000080027800020278008001EB0008003700B2
:101D10000402E90063C07800805A78008301E8007B
:101D20000004E00002003A008000EB0006003700EB
:101D3000828F5100F6FF3A00FBFF37000040EB00B6
:101D400080F07A008100E800848F5000FBFF3A00A9
:101D50000600780000000600889FBE0000017800A1
:101D600001047800B10090000118A3003D0032008A
:101D70000198A30003003A00180090000000E00062
:101D800038003A000190A0003104980082047800E5
:101D9000F90FB200180090000000E00002003A00C5
:101DA00028009000000C7800EA8F540006003A00EA
:101DB000380090000078A30003003A008800780003
:101DC000D0002000E4FF0700980090005800900029
:101DD000808F50000B0032000100E80010049800D2
:101DE0001800780009587800000C780011C0B30082
:101DF0008088210001487800EA8F540006003200F4
:101E00001900370088007800094078001F04070097
:101E10008004780014003700380090000088A30088
:101E20001100320018019000A800900048009000B6
:101E300092FA070098009000810F500004003200D1
:101E4000380090000003B300300498008084EB0059
:101E50000000EB001004980028009000000C7800AF
:101E6000010037008084EB00090078004F04BE00B9
:101E700000000600FE874700889FBE008A9FBE00C4
:101E80008C9FBE008E1F7800F0B79F00010778007E
:101E900082BF9F000000EB00A0B79F009F023700A9
:101EA0008006EB0050C2B30080CF50000900320022
:101EB0000100FB00FFB09700A7FF0700E10F400003
:101EC00096023200AFB097008100E800A1B79F00F2
:101ED000920237009E407800D0C2B30080CF5000FD
:101EE0000C00320007003C006D40500080CF5000D5
:101EF0000A0032006B40400080CF50000E003A00D4
:101F00000800370000C3B30080CF50000A003A0039
:101F1000060037000D30A000050037000D00A000BE
:101F2000030037000D10A000010037000D20A000B5
:101F30000E07E800E7FF37000D18A300010032008C
:101F40000D00A1000D38A300010032000D20A100FA
:101F50000100FB0002FD2F0002004000E90F5000CD
:101F60000E003E000002EB00C4B79F008201780023
:101F7000CFB297006A28B9001E01FB0000014100A2
:101F800003014100C2B79F005E00FB000300400058
:101F9000E90F50000B003E00F5FF37000006EB0094
:101FA000CCB79F00A0C2B30080CF500005003A001C
:101FB0000FB89700C000780080BF9F00C1B79F0096
:101FC0000E07E8000001EB00B2B79F00E0C2B300CB
:101FD0009E4F100018003A000DE0A0008E00E800AF
:101FE00064405000914F1000020032000107780059
:101FF0000C0037000FBA9700C402780084BF9F001E
:10200000B5B79F000E87E8000B0037003FB697007A
:102010006A60B9000000410003004000B0B79F00B3
:102020000E07E8001E01FB0003FD2F000300410026
:10203000E90F5000F5FF3600BE407800E1D79F0061
:10204000C0C6B30080CF5000220032000F003C0019
:102050006940500080CF50007700320004003C00FF
:102060000104E000310232006B4050000F003700E5
:1020700040C6B30080CF500093003200654040005E
:1020800080CF50008B003A008F00370030C7B3007C
:1020900080CF50001A00320007003C00644050001E
:1020A00080CF5000110032000040E80080CF500087
:1020B00080003A000F00370050C7B30080CF5000B7
:1020C000800032006340400080CF500079003A0029
:1020D00009003700000028000D48A30001003A0065
:1020E0000001200080867600D3FF37000D60A0003D
:1020F000750037000D50A0000D70A0007200370071
:102100008FB897004100780081BF9F0000047800DD
:102110000000E00001003A00888221008004EB000A
:10212000010037008104E80089007800088044003D
:102130001004E000FBFF3A003FB197000200E0000E
:1021400003003200890F5100010031008204780041
:102150000002EB00E4AF9F00CFB29700898F5200DE
:102160000200360009805200E0AF9F004368DE00A5
:10217000E10660001B003A000D06780009003700F8
:10218000FFB0970000022000F3FE0700E10F4000BF
:10219000030032002FB097000000E800A0B79F00B6
:1021A0000C06E800EFA89700810F5600F4FF3A00F4
:1021B0000081EB00E2AF9F000A0037008800780042
:1021C0003100FB0001047800FFB09700E2FE070039
:1021D000E10F4000030032002FB297000402E80034
:1021E000A4B79F000900E90080047800E10F4000D7
:1021F000F2FF3A000006EB000D00E0000A003A0092
:10220000C6013700FFB0970000022000D2FE070091
:10221000E10F400003003200AFB297008502E800F2
:10222000A5B79F000C06E8006FA89700800F560026
:10223000F4FF3A00B90137008FB8970041007800E9
:1022400081BF9F00CF80DE0001017800820178000D
:102250000205BE000004BE000203BE000002BE0074
:102260004822DE00482EDD0004027600E4D79F00FD
:102270000D48A3000A0032000404E0000800320008
:10228000E14F42000600320071FD2F00018047003F
:102290000448780018409800290020000200370008
:1022A000F0D79F001900200072FD2F000284470024
:1022B000A1FF370064FD2F000484470019002000AF
:1022C0009DFF37000D0CB3000D007800000CB2002C
:1022D00028003A000D00E00005003D008FBA97008D
:1022E0004505BE004504BE0085BF9F0014003700B1
:1022F0000D48A3000B0032000FBE97004C00BE003B
:102300008CBF9F004F89DE00CF91DE000002BE002F
:1023100002037800820378000605BE000404BE00B4
:10232000070037008FB897004100780081BF9F00F9
:1023300000047800CFC4DE00090578008A05780023
:10234000E00F5400E08F5C00E00F5D00E08F5D0067
:102350001F003D003D00B3006000B8006011B800F0
:1023600008045000898458000A0559008B855900DB
:10237000170037000D00E00005003D000FB9970081
:102380004205BE004204BE0082BF9F00100037001D
:102390000D48A300070032000FBA97004400BE00AA
:1023A00084BF9F006011B8000205BE000004BE009B
:1023B000070037008FBA97004500780085BF9F005F
:1023C00000047800090020000A0020000B00200013
:1023D0003FB697000C00E00007003A00E00F540001
:1023E000E08F5C00E00F5D00E08F5D0002003A00CE
:1023F00010002000B0B79F008D007800010CB200E3
:10240000E1B79F0000042000808F500030003200B0
:1024100003003C000100E0000800320040003700EB
:10242000000820006FB19700800F510014003200A7
:10243000000C2000800F510039003A0014C0B30096
:10244000857821000B0037000400FB004300DD000D
:10245000050040005001BE004000BE000040E10009
:1024600001C8E10002D0E10003D8E1002B003900EF
:102470000442E800F44F5200F3FF3A00270037000F
:1024800000012000010020006011B80014C0B3005A
:102490000040E10001C8E10002D0E10003D8E10002
:1024A0001E003900450020000000D0008180D200CD
:1024B0000281D2008381D2008502E900FAFF3A004E
:1024C0000442E800F04F5200F1FF3A0013003700D9
:1024D00080002000010020006011B80014C0B3008B
:1024E0000040E10001C8E10002D0E10003D8E100B2
:1024F0000A0039003C0020000000D0008180D2009A
:102500000281D2008381D2000C06E900FAFF3A0072
:102510000442E800F54F5200F1FF3A00E4D79F0073
:10252000EFD097000100FB003FB19700820F5000F1
:1025300002003D00E2D79F00040037003FB2970041
:10254000800F520001003D00B0B79F00CFB297004E
:102550000500E000040032006380660002003200E3
:102560008502E900C5B79F000DE8A3000B0032000B
:102570004FB697003FB09700800F560003003C0015
:102580008000EB00C1B79F00040037004FB19700F7
:102590003FB2970004015100C2B79F00EFD29700ED
:1025A0000500FB000006EB00DCAF9F00CFB09700FA
:1025B000808F50000200340000805000D0AF9F0098
:1025C0000D28A30037003200E18066000D18A3003B
:1025D0000C003200D00220000100E00001003A00AF
:1025E0000080E900FFB09700DBFD0700E10F40002D
:1025F0000E0032002FB197000201E800A2B79F0041
:102600000A0037000100E00008003200FFB0970028
:1026100000022000D0FD0700E10F4000030032005F
:102620002FB297000402E800A4B79F00DFAA97002A
:102630000500E0000F0032000006EB00FFB097003D
:1026400000032000C4FD0700E10F4000030032003A
:102650002FB097000000E800A0B79F000C06E8002C
:10266000DFA89700810F5600F4FF3A000001EB004D
:10267000D2AF9F003FB29700C320DD000078210059
:102680008080400091B79F004220DD006400500030
:1026900080B79F006320B900F0AF9F006306500031
:1026A00084003700DFAA97000500E0001100320027
:1026B000688066000F003A0000067800FFB09700BF
:1026C00000022000A4FD0700E10F400003003200DB
:1026D0002FB097000000E800A0B79F000C06E800AC
:1026E000DFA89700810F5600F4FF3A000001EB00CD
:1026F000D2AF9F00E18066000D18A3000C003200ED
:10270000D00220000100E00001003A000080E90052
:10271000FFB0970090FD0700E10F4000D5FF3200A9
:102720002FB297000402E800A4B79F00D1FF370042
:102730000100E000CFFF3200FFB097000002200050
:1027400085FD0700E10F4000CAFF3200AFB29700DD
:102750008502E800A5B79F00C6FF370000042000EF
:10276000EFB09700808F50003100320003003C0032
:102770000100E000080032003E00370000082000A1
:102780006FB19700800F510011003200000C200043
:10279000800F510037003A001FB097003002BE0092
:1027A0002003BE000800BE000A01BE0001FB0700B6
:1027B000A4002000050020006033B80004FB0700DF
:1027C00004C3B30004424000E4D79F00290037004F
:1027D000F5822100D5B79F000D58A30002003A00F2
:1027E00000842100D0B79F001400200005002000C5
:1027F0006033B8008FB097008100E9000500330016
:102800000402D0008582D2000683D2008783D200E2
:10281000F9FF37000800BE000A01BE00E5FA070014
:102820006F0060005FB197006240780010003700D1
:1028300014002000050020006033B8000C00780070
:102840000000E900050033000402D0008582D200B8
:102850000683D2008783D200F9FF37000800BE004C
:102860000A01BE00D3FA0700674060000043B000D1
:10287000E0D79F00EFD097000100FB00FFB097006A
:1028800035FD0700E10F4000030032002FB1970033
:102890000201E800A2B79F001FB297006802520031
:1028A00094B79F008FB29700E482520085B79F00D3
:1028B00063065600D0FF2F003FB197000090B9008B
:1028C0007FAA97000000420063005000800F56006E
:1028D000A2FF3A000D38A30010003200DFAA9700D3
:1028E0000500E0000D0034000006EB00FFB097008B
:1028F0000002200018FD0700E10F40000300320035
:102900002FB097000000E800A0B79F000C06E80079
:10291000DFA89700810F5600F4FF3A00BE40780010
:10292000E1D79F000104E0005DFD3A002FB0970061
:102930004F0778004F06BE004F05BE004F04BE0093
:10294000EF01B100000006000004780092010700CA
:102950000800780000F80700889FBE000004780097
:102960008144780000FD2F0000004400E90F500072
:1029700002003E00000178000D00370008007800DA
:102980009FF707000000E000030032000800780015
:10299000A1F707000004780008007800A5F70700F9
:1029A0000000E0000700320090FA2F000001440010
:1029B0000980FB00800F510002003D000280FB00F7
:1029C00001003700F00F20004F04BE000000060099
:1029D000881F780050C480007D0107000004780043
:1029E0009EF707000000E000FAFF3A00E10F440004
:1029F0000300320051C4800008007800A8010700DD
:102A00004F04780000000600EC874700889FBE0056
:102A10008A9FBE008C9FBE008E1F780081BF9F00E2
:102A20000207780050C488008046EB00040137009C
:102A30008884FB000900780088F707008000780090
:102A40000000E00002003200E1FF0700FC00370058
:102A500050C2B300804F5400F0003A000FBD970001
:102A600020C0B300C0EF9F00D1EF9F0081EF9F0017
:102A70000300370040C0B300C0EF9F000FBD9700B8
:102A80000FB99700B240780082BF9F008184FB009D
:102A900090C6B30080CF50003500320017003E00D2
:102AA0006640500080CF5000620032000C003E00B3
:102AB0007740500080CF50002800320006003E00D2
:102AC0000104E0009B003200A0C2B30080CF5000A0
:102AD0006E003A001D00370080C5B30016003700B5
:102AE00040C6B30080CF5000210032006440400057
:102AF00080CF500065003A001200370030C7B300A5
:102B000080CF50001E00320007003E00674050009A
:102B100080CF5000110032006340400080CF500051
:102B20005A003A001400370050C7B30080CF50005D
:102B30000F0032006340400080CF500053003A0045
:102B40006500370020C0B300CBFF3700DFE89700F7
:102B50008140E800D1EF9F00C8FF37004FE99700A0
:102B600080C0B300E24F5100C3FF3A00C1FF3700FD
:102B7000ACC0B300590037008CC0B3005700370019
:102B800093FF0700DFE897000104E00002003A002D
:102B90004E017800D2B79F0050C480000C0107009E
:102BA00000047800E10F4000A20032008FEC970093
:102BB000120037000A85E8008ABF9F001600370020
:102BC0008FB897001100FB00800F5400F9FF32000E
:102BD0005FE997000204E00003003A005FB097004D
:102BE00008587800D0B79F008944E9000A003200F5
:102BF00050C48000F6000700000478000800E800D8
:102C0000E10F5000040036000800780013F70700B9
:102C10000000E000EAFF3200DFE897000104E00076
:102C200087003A008D46E8005FB1970001497800BF
:102C3000830037005FE897000004E00003003A00DB
:102C40008D46E800CE007800D1B79F0050C48000C8
:102C5000DF000700E10F4000760032005FE99700D7
:102C60000204E00003003A00DFB0970080587800CB
:102C7000D1B79F000FE997000241E90082EF9F0062
:102C80004240A9006E003400F0FF37000180FB00D5
:102C900008FD2F0008004000E90F50005F003E00D3
:102CA0000A0078001B01070080EF9F008800780071
:102CB000030037000FB897000000E80080BF9F00B6
:102CC0000FB997001200FB0001004000E90F50000F
:102CD000F8FF360069FF37000CC1B3003CFF070066
:102CE00050C48000BA000700000578000040EB00E7
:102CF000E0EF9F00D0022000800F550005003A0051
:102D000050C48000B20007000005780011C0B30075
:102D1000E1EF9F008C4078000A0078000EFF07006A
:102D2000E14F40000A003A0051C480000A007800D8
:102D3000DB0007000D04E0004B003A0050C48000A7
:102D4000300090000048A3004300320048003700E4
:102D50008FED97006044B8000C81FB000300200059
:102D60000800BE0074F707000004BE008C40780025
:102D70000A007800F8FE07000080FB000100200038
:102D800008044000898448008B45E90007003200B0
:102D900050C480008E000700000578008C40780049
:102DA000EDFE0700E14F4000EBFF3A008C40780059
:102DB0000A007800E8FE0700E14F400003003A00F7
:102DC00051C480000A007800B50007006FE9970041
:102DD0000204E0000200320060041400E0841C00E1
:102DE0005FE897000004E00015003A008D46E80017
:102DF000CFE89700E4CF500003003A004E0078007F
:102E00000888BE000E0037000E81E9000207780036
:102E100012007800080878000900370050C48000CC
:102E20006B000700808F540005003200E10F400066
:102E30000B003A000D04E0000D0032000A003700DC
:102E40008FB897003144780081BF9F000804E000EC
:102E5000F7FE3A00040037000000EB0005003700E1
:102E600051C480008E0007000D80FB000100370078
:102E70000080EB004F0778004F06BE004F05BE00F4
:102E80004F04BE00CF00B100000006000200FA00AF
:102E9000889FBE00A0FF9F0001047800B100900051
:102EA000810478000904B200020032000000FB0037
:102EB000360037000118A30005003A000103B300F3
:102EC00031049800190498000080EB002F003700AF
:102ED000580090000000E00006003A004800900012
:102EE00012002000E680570064F6070019049800DD
:102EF00024003700280090000000E00008003A009D
:102F00004088210020049800000C78002000200058
:102F100050049800100498000130A000310498007B
:102F200018019000A80090004800900053F6070098
:102F300028009000000C78000080EB00100498003E
:102F400018007800AFF8970001587800000C78005E
:102F50002FF89700EA4F50000A003A00380090001E
:102F60000088A3000700320018019000A80090001C
:102F70004800900041F6070019049800A80090004E
:102F8000010C7800AFF897000100FB004F04BE0071
:102F90000080FA0000000600881F780060C48000EE
:102FA0000000E0000100320000000100488521001F
:102FB000080078007B0007006C0444008087210033
:102FC000800F5400FAFF3A004F047800000006001A
:102FD000881F780000047800B00090000148A3002A
:102FE00007003A000108A300050032000198A30081
:102FF00008003200100090000000E00005003200E0
:10300000380090000040A000300498008080EB0061
:10301000200037000190A1003104980018009000B2
:103020000000E000060034000000E90010049800F1
:1030300018007800B080FB00000C78000600370014
:10304000380090000068A300EDFF3A000800780007
:103050008C00070080007800380090000078A30002
:103060000C003A00FA8F500008003A002800900047
:103070000000E000E2FF3200180090000000E800CD
:1030800010049800180CE900DDFF3700ED8F5000A8
:10309000E2FF3200010078004F04780000000600D3
:1030A00080017800E10F40001700320031009000ED
:1030B0000008A300140032000098A30012003A0098
:1030C000210290000400E0000F0032001101900086
:1030D00051009000800F51000B0032001100780069
:1030E000840F500002003A008008E8000200370018
:1030F0000200E800900098001100E90080087800C4
:1031000003487800010037008081EB00030078005D
:10311000000006000001780000C2B3000100370083
:103120000201E8009240780080CF5000FCFF32009E
:10313000E9CF5000FAFF3200D0C2B30080CF500078
:1031400003003A000201E80014C0B3000500370094
:103150000042EB00B0C2B30080CF500001003A0043
:103160000201E8008000EB0005FD2F00040037009D
:103170006A08B90000804100850040000201E800B3
:103180009201FB0005804100E90F5000F8FF360076
:103190000404E000010032008100EA000100780030
:1031A00000000600889FBE008A1F78000004780097
:1031B00030009000630060002400320008007800B6
:1031C0007E0007003805900080EF2F0000006500AA
:1031D00030049800280090000000E0000400320055
:1031E000E804650002003A00AD00070029049800D9
:1031F00048009000E0F50700E10F400013003200A6
:10320000B80090000102B20010003A000AC8A30002
:103210001800320080C480000000E0001500320079
:103220000001780081047800012A20001228900013
:10323000880F5000070032004205B0004905B00079
:10324000818F54000B003200F8FF37000080EB0044
:103250000900370002007800D0F5070080C4800024
:10326000090040008000EB00112898000100780060
:10327000010037000000EB004F0578004F04BE004E
:10328000000006000200FA00889FBE008A1F780036
:10329000000478000000EB00100498003800900053
:1032A0008080EB000008A3003F00320080882100EE
:1032B0001004E0001000320049852100AA85210099
:1032C0001A0078006C0545002010B2002110200083
:1032D000810F500002003A00090078003700070013
:1032E000EC84440080872100808F5400F4FF3A0072
:1032F000808821000048EB004800900058019000B1
:103300000200E0000D003A001204980012002000B4
:10331000E8805700AAF50700E10F500003003A00CB
:103320000FF897008080FB001F00370038009000E6
:103330000040A0003004980012003700A800900060
:103340009FF50700100498000000E0000300320021
:10335000E10F40000D003A000300370038009000F4
:103360000040A00002003700380090000003B300C6
:1033700030049800A8009000010C78000000EB00D9
:10338000100498008080EB0007003700A800900030
:10339000010C78000000E90010049800010078009A
:1033A000B080FB00000C7800010078004F05780029
:1033B0004F04BE000080FA0000000600881F78005D
:1033C00000047800300090000008A30007003200DD
:1033D000800078000120B20004003A001104980037
:1033E000A8009000010C7800170037000018A30017
:1033F000190032000098A30017003200A8009000C6
:103400000100E00014003200180190000200E0000A
:10341000110032004800900018F507009800900055
:10342000810F500003003200380090000003B30009
:10343000300498000000EB00100498002800900071
:10344000000C7800380090000058A3000200320001
:103450000080EB00010037000000EB004F04780013
:103460000000060071C480000100E000030032008B
:103470001100780070C4880003003700200020008D
:1034800088F5070080007800E18F400002003A00D4
:10349000906E260090C488000100780000000600AD
:1034A00071C480000108780070C488000000060024
:020000040000FA
:0200000401F009
:04000C00FBFF0000F6
:020000040000FA
:0200000401F009
:04001000FDFF0000F0
:020000040000FA
:0200000401F009
:040014007FFF00006A
:020000040000FA
:10000800FC030000C2DC000092DC0000AADC000057
:10001800DADC0000F2DC0000FC030000FC03000056
:10002800FC0300005AE40000FC030000BA000100D1
:10003800FC030000ACE40000FC030000FC0300002B
:1000480022DD0000FC030000FC03000036FE000077
:10005800FC030000FC030000FC030000FC0300009C
:10006800FC030000FC030000FC030000FC0300008C
:10007800FC030000FC030000FC030000FC0300007C
:10008800FC030000FC030000FC0300002AD500006C
:1000980000D60000FC03000008FD0000FC0300007F
:1000A800FC030000FC030000FC030000FC0300004C
:1000B800FC030000FC030000FC030000FC0300003C
:1000C800FC030000FC030000FC030000FC0300002C
:1000D800FC030000FC0300000ADD0000FC03000034
:1000E800FC030000FC030000FC030000FC0300000C
:1000F800FC030000FC030000FC030000FC030000FC
:10010800FC030000FC030000FC030000FC030000EB
:10011800FC030000FC030000FC030000FC030000DB
:10012800FC030000FC030000FC030000FC030000CB
:10013800FC030000FC030000FC030000FC030000BB
:10014800FC030000FC030000FC030000FC030000AB
:10015800FC030000FC030000FC030000FC0300009B
:10016800FC030000FC030000FC030000FC0300008B
:10017800FC030000FC030000FC030000FC0300007B
:10018800FC030000FC030000FC030000FC0300006B
:10019800FC030000FC030000FC030000FC0300005B
:1001A800FC030000FC030000FC030000FC0300004B
:1001B800FC030000FC030000FC030000FC0300003B
:1001C800FC030000FC030000FC030000FC0300002B
:1001D800FC030000FC030000FC030000FC0300001B
:1001E800FC030000FC030000FC030000FC0300000B
:0801F800FC030000FC03000001
:020000040000FA
:10020800FC030000C2DC000092DC0000AADC000055
:10021800DADC0000F2DC0000FC030000FC03000054
:10022800FC0300005AE40000FC030000BA000100CF
:10023800FC030000ACE40000FC030000FC03000029
:1002480022DD0000FC030000FC03000036FE000075
:10025800FC030000FC030000FC030000FC0300009A
:10026800FC030000FC030000FC030000FC0300008A
:10027800FC030000FC030000FC030000FC0300007A
:10028800FC030000FC030000FC0300002AD500006A
:1002980000D60000FC03000008FD0000FC0300007D
:1002A800FC030000FC030000FC030000FC0300004A
:1002B800FC030000FC030000FC030000FC0300003A
:1002C800FC030000FC030000FC030000FC0300002A
:1002D800FC030000FC0300000ADD0000FC03000032
:1002E800FC030000FC030000FC030000FC0300000A
:1002F800FC030000FC030000FC030000FC030000FA
:10030800FC030000FC030000FC030000FC030000E9
:10031800FC030000FC030000FC030000FC030000D9
:10032800FC030000FC030000FC030000FC030000C9
:10033800FC030000FC030000FC030000FC030000B9
:10034800FC030000FC030000FC030000FC030000A9
:10035800FC030000FC030000FC030000FC03000099
:10036800FC030000FC030000FC030000FC03000089
:10037800FC030000FC030000FC030000FC03000079
:10038800FC030000FC030000FC030000FC03000069
:10039800FC030000FC030000FC030000FC03000059
:1003A800FC030000FC030000FC030000FC03000049
:1003B800FC030000FC030000FC030000FC03000039
:1003C800FC030000FC030000FC030000FC03000029
:1003D800FC030000FC030000FC030000FC03000019
:1003E800FC030000FC030000FC030000FC03000009
:0803F800FC030000FC030000FF
:020000040000FA
:1034B000705F000061700000705F0000636F0000CB
:1034C0006E66000069670000007300007263000010
:1034D0002F480000756200002F4800007562000050
:1034E0002E63000000250000733A000025690000EB
:1034F00020250000732000002D2D00002061000019
:103500007373000065720000746900006F6E000044
:1035100020660000616900006C650000640A00001C
:10352000000000000000000000000000000000009B
:10353000000000000000000000000000000000008B
:10354000000000000000000000000000000000007B
:10355000000000000000000000000000000000006B
:10356000000000000000000000000000000000005B
:10357000000000000000000000000000000000004B
:10358000000000000000000000000000000000003B
:10359000000000000000000000000000000000002B
:1035A000000000000000000000000000000000001B
:1035B000000000000000000000000000000000000B
:1035C00000000000000000000000000000000000FB
:1035D00000000000000000000000000000000000EB
:1035E00000000000000000000000000000000000DB
:1035F00000000000000000000000000000000000CB
:1036000000000000000000000000000000000000BA
:1036100000000000000000000000000000000000AA
:10362000000000000000000000000000000000009A
:10363000000000000000000000000000000000008A
:10364000000000000000000000000000000000007A
:10365000000000000000000000000000000000006A
:10366000000000000000000000000000000000005A
:10367000000000000000000000000000000000004A
:10368000000000000000000000000000000000003A
:10369000000000000000000000000000000000002A
:1036A000000000000000000000000000000000001A
:1036B00000460000697200006D7700006172000032
:1036C000652000003D200000257500002E2500002B
:1036D000752E000025750000004C000045440000D8
:1036E0004272000069740000652000003D20000067
:1036F0002575000000480000616E00006443000072
:10370000747200006C2000003D2000002564000061
:103710000057000069720000656400002049000045
:10372000502000003D200000256400002E250000F0
:10373000642E0000256400002E25000064000000B7
:103740005769000046690000204D00006F640000CA
:10375000203D0000202500006400000057690000A3
:1037600046690000436F00006E6E0000203D0000BF
:103770002025000064000000576900004669000031
:10378000465600004F6B0000203D00002025000041
:1037900064000000576900004669000046560000BA
:1037A00065720000203D000020250000752E0000FD
:1037B000257500002E2500007500000057690000E7
:1037C000466900005353000049440000203D0000BA
:1037D00020250000730000005769000046690000C2
:1037E0004164000064720000203D000020250000BC
:1037F000642E0000256400002E250000642E0000C9
:10380000256400000057000069460000695300006D
:10381000656300004D2000003D200000256300008E
:10382000005700006946000069530000656300000E
:103830004B2000003D200000257300000000000028
:103840000000000000000000000000000000000078
:103850000000000000000000000000000000000068
:103860000000000000000000000000000000000058
:103870000000000000000000000000000000000048
:103880000000000000000000000000000000000038
:103890000000000000000000000000000000000028
:1038A0000000000000000000000000000000000018
:1038B0000000000000000000000000000000000008
:1038C00000000000000000000000000000000000F8
:1038D00000000000000000000000000000000000E8
:1038E00000000000000000000000000000000000D8
:1038F00000000000000000000000000000000000C8
:1039000000000000000000000000000000000000B7
:1039100000000000000000000000000000000000A7
:103920000000000000000000000000000000000097
:103930000000000000000000000000000000000087
:103940000000000000000000000000000000000077
:103950000000000000000000000000000000000067
:103960000000000000000000000000000000000057
:103970000000000000000000000000000000000047
:103980000000000000000000000000000000000037
:103990000000000000000000000000000000000027
:1039A0000000000000000000000000000000000017
:1039B0000000000000000000000000000000000007
:1039C00000000000000000000000000000530000A4
:1039D000636100006E2000002049000044200000C8
:1039E0003D2000002564000000530000432000003B
:1039F000496E000064650000782000003D20000052
:103A000025640000004E000065740000436F000054
:103A1000756E0000742000003D2000002564000049
:103A200000530000636100006E5300005349000022
:103A3000442000003D2000002573000000530000DA
:103A400065630000204D00006F64000065200000E9
:103A50003D20000025640000004E00006574000059
:103A60002054000079700000652000003D20000017
:103A7000256400000053000069670000202000005A
:103A800053740000722000003D20000025640000F7
:103A9000004C00006F610000644400006F6E000085
:103AA000652000003D2000002564000000000000AB
:103AB0000000000000000000000000000000000006
:103AC00000000000000000000000000000000000F6
:103AD00000000000000000000000000000000000E6
:103AE00000000000000000000000000000000000D6
:103AF00000000000000000000000000000000000C6
:103B000000000000000000000000000000000000B5
:103B100000000000000000000000000000000000A5
:103B20000000000000000000000000000000000095
:103B30000000000000000000000000000000000085
:103B40000000000000000000000000000000000075
:103B50000000000000000000000000000000000065
:103B60000000000000000000000000000000000055
:103B70000000000000000000000000000000000045
:103B80000000000000000000000000000000000035
:103B90000000000000000000000000000000000025
:103BA0000000000000000000000000000000000015
:103BB0000000000000000000000000000000000005
:103BC00000000000000000000000000000000000F5
:103BD00000000000000000000000000000000000E5
:103BE00000000000000000000000000000000000D5
:103BF00000000000000000000000000000000000C5
:103C000000000000000000000000000000000000B4
:103C100000000000000000000000000000000000A4
:103C20000000000000000000000000000000000094
:103C30000000000000000000000000000000000084
:103C40000000000000000000000000000000000074
:103C50000000000000000000000000000000000064
:103C60000000000000490000502000003D2000003E
:103C7000256400002E250000642E0000256400004D
:103C80002E250000640000004D610000736B0000F1
:103C9000203D000020250000642E00002564000067
:103CA0002E250000642E000025640000004700005F
:103CB000617400006577000061790000203D00001C
:103CC00020250000642E0000256400002E25000041
:103CD000642E000025640000005000004E530000D8
:103CE000203D000020250000642E00002564000017
:103CF0002E250000642E0000256400000053000003
:103D00004E530000203D000020250000642E0000DE
:103D1000256400002E250000642E000025640000AC
:103D200000440000656600002E200000495000009D
:103D3000203D000020250000642E000025640000C6
:103D40002E250000642E00002564000000440000C1
:103D5000656600002E2000004D610000736B0000BE
:103D6000203D000020250000642E00002564000096
:103D70002E250000642E0000256400000044000091
:103D800048430000502000003D2000002564000052
:103D9000004E000065740000424900004F530000CF
:103DA000203D000020250000730000004D41000070
:103DB000432000003D2000002573000000000000AB
:103DC00000000000000000000000000000000000F3
:103DD00000000000000000000000000000000000E3
:103DE00000000000000000000000000000000000D3
:103DF00000000000000000000000000000000000C3
:103E000000000000000000000000000000000000B2
:103E100000000000000000000000000000000000A2
:103E20000000000000000000000000000000000092
:103E30000000000000000000000000000000000082
:103E40000000000000000000000000000000000072
:103E50000000000000000000000000000000000062
:103E60000000000000000000000000000000000052
:103E70000000000000000000000000000000000042
:103E80000000000000000000000000000000000032
:103E90000000000000000000000000000000000022
:103EA0000000000000000000000000000000000012
:103EB0000000000000000000000000000000000002
:103EC00000000000000000000000000000000000F2
:103ED00000000000000000000000000000000000E2
:103EE00000000000000000000000000000000000D2
:103EF00000000000000000000000000000000000C2
:103F000000000000000000000000000000000000B1
:103F100000000000000000000000000000000000A1
:103F20000000000000000000000000000000000091
:103F30000000000000000000000000000000000081
:103F40000000000000000000000000000000000071
:103F50000000000000000000000000000000000061
:103F60000000000000000000000000000000000051
:103F700000000000004300006F6E00006669000052
:103F8000672000003D2000002564000000000000C4
:103F90000000000000000000000000000000000021
:103FA0000000000000000000000000000000000011
:103FB0000000000000000000000000000000000001
:103FC00000000000000000000000000000000000F1
:103FD00000000000000000000000000000000000E1
:103FE00000000000000000000000000000000000D1
:103FF00000000000000000000000000000000000C1
:1040000000000000000000000000000000000000B0
:1040100000000000000000000000000000000000A0
:104020000000000000000000000000000000000090
:104030000000000000000000000000000000000080
:104040000000000000000000000000000000000070
:104050000000000000000000000000000000000060
:104060000000000000000000000000000000000050
:104070000000000000000000000000000000000040
:104080000000000000000000000000000000000030
:104090000000000000000000000000000000000020
:1040A0000000000000000000000000000000000010
:1040B0000000000000000000000000000000000000
:1040C00000000000000000000000000000000000F0
:1040D00000000000000000000000000000000000E0
:1040E00000000000000000000000000000000000D0
:1040F00000000000000000000000000000000000C0
:1041000000000000000000000000000000000000AF
:10411000000000000000000000000000004E000051
:10412000657700002048000075620000204900000B
:10413000502000003D200000256400002E250000D6
:10414000642E0000256400002E250000640000009D
:104150004E650000772000004875000062200000D6
:104160004D610000736B0000203D00002025000021
:10417000642E0000256400002E250000642E00003F
:1041800025640000004E0000657700002048000014
:104190007562000020470000572000003D2000000D
:1041A000256400002E250000642E00002564000018
:1041B0002E250000640000004E65000077200000FE
:1041C0004875000062200000444800004350000091
:1041D000203D000020250000640000004E65000026
:1041E0007720000057690000466900002049000060
:1041F000502000003D200000256400002E25000016
:10420000642E0000256400002E25000064000000DC
:104210004E650000772000005769000046690000E5
:10422000204D0000617300006B2000003D20000065
:10423000256400002E250000642E00002564000087
:104240002E250000640000004E650000772000006D
:104250005769000046690000204700005720000011
:104260003D200000256400002E250000642E000083
:10427000256400002E250000640000004E6500004B
:1042800077200000576900004669000020440000C4
:1042900048430000502000003D200000256400003D
:1042A0000053000045540000000000000000000022
:1042B00000000000000000000000000000000000FE
:1042C00000000000000000000000000000000000EE
:1042D00000000000000000000000000000000000DE
:1042E00000000000000000000000000000000000CE
:1042F00000000000000000000000000000000000BE
:1043000000000000000000000000000000000000AD
:10431000000000000000000000000000000000009D
:10432000000000000000000000000000000000008D
:10433000000000000000000000000000000000007D
:10434000000000000000000000000000000000006D
:10435000000000000000000000000000000000005D
:10436000000000000000000000000000000000004D
:10437000000000000000000000000000000000003D
:10438000000000000000000000000000000000002D
:10439000000000000000000000000000000000001D
:1043A000000000000000000000000000000000000D
:1043B00000000000000000000000000000000000FD
:1043C00000000000000000000000000000000000ED
:1043D00000000000000000000000000000000000DD
:1043E00000000000000000000000000000000000CD
:1043F00000000000000000000000000000000000BD
:1044000000000000000000000000000000000000AC
:10441000000000000000000000000000000000009C
:10442000000000000000000000000000000000008C
:104430000000000000000000005300006572000052
:10444000696100006C2000004E7500006D62000084
:1044500065720000203D0000202500006C75000002
:1044600000000000686500006164000065720000E3
:104470002E6900006E630000006600006F6F000090
:1044800074650000722E0000696E00006300000079
:104490002144000045460000000D00000A00000015
:1044A0007478000074000000687400006D00000063
:1044B000687400006D6C0000006300006769000014
:1044C000007800006D6C0000006300007373000052
:1044D0000067000069660000007000006E67000061
:1044E000006A000070670000006300006C6100005B
:1044F000007700006176000000000000000000006E
:104500000000000050A2000054A2000058A20000C9
:104510005DA2000061A2000065A2000069A2000087
:104520006DA2000071A2000075A2000079A2000037
:104530007DA2000074650000787400002F700000F8
:104540006C610000696E0000007400006578000076
:10455000742F0000687400006D6C0000007400008F
:1045600065780000742F0000786D00006C0000007A
:1045700074650000787400002F63000073730000FE
:10458000006900006D610000676500002F67000092
:1045900069660000006900006D6100006765000049
:1045A0002F7000006E670000006900006D61000060
:1045B000676500002F6A000070650000670000005A
:1045C00061700000706C000069630000617400009D
:1045D000696F00006E2F00006A61000076610000C4
:1045E0002D7600006D000000617500006469000018
:1045F0006F2F0000782D00007761000076650000C5
:10460000000000009AA20000A5A20000A5A20000E0
:10461000A5A20000AFA20000B8A20000C1A2000045
:10462000CBA20000D5A20000E0A20000F4A200008E
:1046300001A3000048540000545000002F31000036
:104640002E3100002032000030300000204F0000EA
:104650004B0D00000A4300006F6E00006E65000005
:1046600063740000696F00006E3A00002063000070
:104670006C6F0000736500000D0A00000048000028
:1046800054540000502F0000312E00003120000053
:10469000343000003020000042610000642000003F
:1046A000526500007175000065730000740D000014
:1046B0000A4300006F6E00006E6500006374000026
:1046C000696F00006E3A0000206300006C6F00000C
:1046D000736500000D0A00000D0A00003430000070
:1046E000302000004261000064200000526500009C
:1046F0007175000065730000743A000020630000CB
:10470000616E00002774000020680000616E0000E8
:10471000646C000065200000436F00006E740000B0
:10472000656E0000742D00004C6500006E6700008F
:10473000746800000D0A0000004800005454000096
:10474000502F0000312E00003120000034300000D6
:1047500031200000556E0000617500007468000093
:104760006F720000697A0000656400000D0A0000A5
:1047700057570000572D0000417500007468000075
:10478000656E0000746900006361000074650000DC
:104790003A200000426100007369000063200000BD
:1047A00072650000616C00006D3D00002250000049
:1047B000726F00007465000063740000656400009F
:1047C000220D00000A4300006F6E00006E650000BD
:1047D00063740000696F00006E3A000020630000FF
:1047E0006C6F0000736500000D0A00000D0A0000E8
:1047F0003430000031200000556E0000617500006B
:10480000746800006F720000697A0000656400003F
:104810003A2000005061000073730000776F0000C1
:10482000726400002072000065710000756900006C
:1048300072650000640D00000A000000485400008A
:10484000545000002F3100002E31000020340000B1
:1048500030340000204E00006F740000206600001D
:104860006F7500006E6400000D0A0000436F0000C9
:104870006E6E000065630000746900006F6E0000DA
:104880003A200000636C00006F730000650D0000AB
:104890000A4300006F6E0000746500006E74000033
:1048A0002D54000079700000653A0000207400006B
:1048B00065780000742F0000687400006D6C0000C3
:1048C0000D0A00000D0A000034300000343A0000E8
:1048D00020460000696C0000652000006E6F00003B
:1048E00074200000666F0000756E0000643C0000DC
:1048F000627200003E55000073650000203C00001D
:104900006120000068720000656600003D22000022
:104910002F750000706C00006F61000064220000C1
:104920003E4D00005046000053200000557000002E
:104930006C6F0000616400003C2F0000613E0000CD
:10494000207400006F200000707200006F6700008C
:10495000726100006D200000776500006220000099
:104960007061000067650000730D00000A00000020
:1049700048540000545000002F3100002E31000038
:104980002034000031340000205200006571000026
:1049900075650000737400002D5500005249000039
:1049A000205400006F6F0000204C00006F6E00006C
:1049B000670D00000A4300006F6E00006E65000086
:1049C00063740000696F00006E3A0000206300000D
:1049D0006C6F0000736500000D0A00000D0A0000F6
:1049E0003431000034200000526500007175000071
:1049F00065730000742D000055520000492000002E
:104A0000546F00006F2000004C6F00006E670000C4
:104A10003A200000427500006666000065720000E2
:104A2000206F000076650000726600006C6F000069
:104A30007720000064650000746500006374000066
:104A4000656400000D0A0000004800005454000096
:104A5000502F0000312E00003120000035300000C2
:104A600030200000496E000074650000726E000086
:104A7000616C000020530000657200007665000044
:104A80007220000045720000726F0000720D00007D
:104A90000A4300006F6E00006E6500006374000042
:104AA000696F00006E3A0000206300006C6F000028
:104AB000736500000D0A00000D0A0000353000008B
:104AC00030200000496E000074650000726E000026
:104AD000616C0000205300006572000076650000E4
:104AE0007220000045720000726F0000723A0000F0
:104AF00020450000787000006563000074650000C8
:104B0000642000006461000074610000206E0000F9
:104B10006F74000020700000726500007365000073
:104B20006E7400000D0A000000480000545400009C
:104B3000502F0000312E00003120000035300000E1
:104B4000312000004E6F000074200000496D00000D
:104B5000706C0000656D0000656E000074650000FB
:104B6000640D00000A4300006F6E00006E650000D7
:104B700063740000696F00006E3A0000206300005B
:104B80006C6F0000736500000D0A00000D0A000044
:104B900035300000312000004E6F0000742000000E
:104BA000496D0000706C0000656D0000656E0000CE
:104BB00074650000643A0000204F00006E6C000035
:104BC000792000004745000054200000616E00007D
:104BD00064200000504F0000535400002073000078
:104BE00075700000706F0000727400006564000052
:104BF0000D0A00000048000054540000502F00002F
:104C0000312E000031200000323000003020000042
:104C10004F4B00000D0A0000436F00006E6E000055
:104C200065630000746900006F6E00003A200000A8
:104C3000636C00006F730000650D00000A43000004
:104C40006F6E0000746500006E7400002D5400004B
:104C500079700000653A000020740000657800005B
:104C6000742F0000687400006D6C00000D0A0000D5
:104C70000D0A00003C680000746D00006C3E0000EE
:104C80003C6200006F640000792000007374000033
:104C9000796C0000653D0000226D0000617200002B
:104CA000676900006E3A000031300000307000008B
:104CB000782200003E3C0000666F0000726D00002C
:104CC000206D000065740000686F0000643D000006
:104CD000706F0000737400002061000063740000B6
:104CE000696F00006E3D0000222F0000757000000B
:104CF0006C6F00006164000022200000656E0000FF
:104D00006374000079700000653D0000226D0000B2
:104D1000756C00007469000070610000727400001E
:104D20002F6600006F7200006D2D000064610000AE
:104D300074610000223E00003C6200003E4D000015
:104D40005046000053200000496D000061670000DC
:104D500065200000557000006C6F00006164000069
:104D60003C2F0000623E00003C7000003E3C000012
:104D7000696E0000707500007420000074790000F6
:104D8000706500003D660000696C00006520000051
:104D90006E6100006D6500003D6900002073000039
:104DA000697A0000653D0000343000003E200000BC
:104DB000266E000062730000703B0000203C000083
:104DC000696E0000707500007420000074790000A6
:104DD000706500003D730000756200006D690000A1
:104DE00074200000766100006C750000653D0000D5
:104DF00022550000706C00006F610000642200000A
:104E00003E3C00002F6600006F7200006D3E000007
:104E10003C2F0000626F0000647900003E3C0000FF
:104E20002F680000746D00006C3E00000048000018
:104E300054540000502F0000312E0000312000009B
:104E400032300000302000004F4B00000D0A0000FF
:104E5000436F00006E6E000065630000746900001F
:104E60006F6E00003A200000636C00006F7300005A
:104E7000650D00000A4300006F6E000074650000BD
:104E80006E7400002D54000079700000653A000037
:104E90002074000065780000742F00006874000022
:104EA0006D6C00000D0A00000D0A00003C68000057
:104EB000746D00006C3E00003C6200006F640000F6
:104EC0007920000073740000796C0000653D0000DB
:104ED000226D000061720000676900006E3A0000F8
:104EE0003130000030700000782200003E3C0000AD
:104EF000623E00004D500000465300002055000067
:104F000070640000617400006520000053750000AB
:104F1000636300006573000073660000756C000039
:104F20003C2F0000623E00003C7000003E3C000050
:104F30006120000068720000656600003D220000EC
:104F40002F2200003E53000069740000652000001D
:104F50006D610000696E0000207000006167000054
:104F6000653C00002F6100003E3C00002F62000005
:104F70006F640000793E00003C2F00006874000060
:104F80006D6C00003E0000004854000054500000CA
:104F90002F3100002E31000020350000303000009D
:104FA000204900006E740000657200006E61000010
:104FB0006C200000536500007276000065720000EE
:104FC00020450000727200006F7200000D0A0000A0
:104FD000436F00006E6E000065630000746900009E
:104FE0006F6E00003A200000636C00006F730000D9
:104FF000650D00000A4300006F6E0000746500003C
:105000006E7400002D54000079700000653A0000B5
:105010002074000065780000742F000068740000A0
:105020006D6C00000D0A00000D0A00003C680000D5
:10503000746D00006C3E00003C6200006F64000074
:105040007920000073740000796C0000653D000059
:10505000226D000061720000676900006E3A000076
:105060003130000030700000782200003E3C00002B
:10507000623E00004D5000004653000020490000F1
:105080006D61000067650000204300006F72000042
:105090007275000070740000206F00007220000024
:1050A000577200006F6E0000672000005665000018
:1050B00072730000696F00006E3C00002F620000F8
:1050C0003E3C0000703E00003C6100002068000093
:1050D00072650000663D0000222F00007570000020
:1050E0006C6F000061640000223E000054720000FA
:1050F0007920000061670000616900006E3F0000D8
:105100003C2F0000613E00003C2F0000626F000059
:10511000647900003E3C00002F680000746D0000C0
:105120006C3E00000048000054540000502F000066
:10513000312E00003120000033300000322000000A
:10514000466F0000756E0000640D00000A43000009
:105150006F6E00006E65000063740000696F0000F0
:105160006E3A0000206300006C6F00007365000061
:105170000D0A00004C6F00006361000074690000BC
:105180006F6E00003A2000000048000054540000F8
:10519000502F0000312E000031200000343000007C
:1051A00033200000466F0000726200006964000056
:1051B000646500006E0D00000A4300006F6E000081
:1051C0006E65000063740000696F00006E3A0000B5
:1051D000206300006C6F0000736500000D0A000082
:1051E0000D0A00003430000033200000466F00003C
:1051F0007262000069640000646500006E3A00009D
:1052000020530000534C0000205200006571000044
:105210007569000072650000642000002D20000008
:1052200075730000652000004854000054500000D1
:10523000530D00000A0000001AA300001AA300008A
:105240003FA300009DA300001EA40000B8A400001E
:1052500025A5000095A50000FBA5000001A3000006
:1052600017A70000C4A7000093A80000C5A800006D
:10527000436F00006F6B0000696500003A0000009A
:1052800041750000746800006F720000697A0000C8
:1052900061740000696F00006E3A00000043000076
:1052A0006F6E0000746500006E7400002D4C0000ED
:1052B000656E000067740000683A0000000000009E
:1052C00038A9000040A900004FA900004745000090
:1052D00054000000504F00005354000000750000BF
:1052E000706C00006F61000064000000666F0000D9
:1052F0006375000073650000722E00006874000082
:105300006D0000000D0A00000D0A0000333000009F
:1053100034200000526500006469000072650000DE
:10532000637400003A200000004300006F6E00002C
:10533000746500006E7400002D5400007970000048
:10534000653A000020000000436F00006E7400000A
:10535000656E0000742D0000456E0000636F000054
:10536000646900006E6700003A200000677A000060
:10537000697000000D0A0000004300006163000036
:10538000686500002D4300006F6E0000747200001D
:105390006F6C00003A200000006E00006F2D0000CE
:1053A0006361000063680000650000006D6100003B
:1053B000782D000061670000653D000000360000A8
:1053C0003030000000530000657400002D430000E1
:1053D0006F6F00006B690000653A0000200000005C
:1053E0000D0A00000D0A0000000D00000A0D00006B
:1053F0000A4D00005046000053020000010000006A
:1054000054680000652000007265000063650000BC
:105410006976000065640000206300006F6D000085
:105420006D6100006E6400002069000073200000C0
:10543000666F0000726D000061740000746500000A
:1054400064200000696E0000636F0000727200004B
:1054500065630000746C000079000000546800006F
:105460006520000072650000636500006976000039
:1054700065640000206300006F6D00006D61000036
:105480006E6400002077000061730000207400004B
:105490006F6F0000206C00006F6E0000670000005E
:1054A000546800006520000072650000636500001C
:1054B0006976000065640000206300006F6D0000E5
:1054C0006D6100006E640000206300006F6E0000DC
:1054D00074610000696E00006564000020690000CE
:1054E0006E760000616C00006964000020700000AE
:1054F00061720000616D000065740000657200005B
:105500007300000054680000652000007265000010
:105510006365000069760000656400002069000092
:10552000646500006E740000696600006965000033
:105530007220000077610000732000006E6F000091
:105540007420000072650000636F0000676E000049
:10555000697A00006564000000540000686500007E
:10556000206300006F6D00006D6100006E6400003C
:105570002072000065630000656900007665000028
:10558000642000007761000073200000666F000057
:1055900072200000616E0000206900006E7600003D
:1055A000616C0000696400002074000061720000FA
:1055B00067650000742000006465000076690000E3
:1055C000636500000054000068650000206300006F
:1055D0006F6D00006D6100006E64000020690000C6
:1055E00073200000696E0000766100006C690000A5
:1055F00064200000626500006361000075730000B4
:1056000065200000746800006520000064650000EB
:1056100076690000636500002069000073200000C7
:10562000686F00006D6900006E67000000540000A4
:1056300068650000206300006F6D00006D61000070
:105640006E6400002069000073200000696E000095
:10565000766100006C69000064200000776800003B
:10566000696C0000652000006E6F0000207400006F
:10567000656D0000706500007261000074750000C7
:105680007265000020700000726F0000626500000B
:105690002069000073200000617400007461000044
:1056A00063680000656400002E000000546800007C
:1056B00061740000206400006576000069630000EA
:1056C000652000007479000070650000206400000F
:1056D0006F650000732000006E6F000074200000F2
:1056E0006578000069730000742E0000004500001A
:1056F000727200006F720000207400006578000074
:10570000742000006E6F00007420000064650000CB
:10571000666900006E65000064000000556E0000C0
:10572000616200006C650000207400006F200000C2
:10573000636F00006E6E000065630000742000005F
:10574000746F0000205700006946000069200000C7
:10575000426F000061720000640000004E650000AE
:1057600077200000576900004669000020730000A0
:1057700065740000746900006E670000732000000B
:105780006172000065200000696E0000636F000018
:10579000727200006563000074000000546800002D
:1057A00065200000636F00006D6D0000616E0000F9
:1057B0006420000066610000696C00006564000000
:1057C00020620000656300006175000073650000E1
:1057D0002074000068650000206600006F63000010
:1057E00075730000657200002069000073200000DE
:1057F00064690000736300006F6E00006E65000056
:1058000063740000656400000054000068650000D7
:10581000206300006F6D00006D6100006E64000089
:1058200020660000616900006C65000064200000D3
:105830006265000063610000757300006520000070
:105840007468000065200000726F00007461000041
:10585000746F000072200000697300002064000073
:1058600069730000636F00006E6E000065630000E6
:1058700074650000640000005468000065200000AA
:10588000636F00006D6D0000616E00006420000019
:1058900066610000696C0000656400002062000021
:1058A00065630000617500007365000020740000EE
:1058B00068650000206600006F63000075730000DB
:1058C0006572000020690000732000006E6F000008
:1058D00074200000686F00006D6500006400000027
:1058E0005468000065200000636F00006D6D0000CB
:1058F000616E00006420000066610000696C0000B9
:1059000065640000206200006563000061750000AE
:1059100073650000207400006865000020720000BC
:105920006F740000617400006F7200002069000055
:10593000732000006E6F000074200000686F00008C
:105940006D650000640000005468000065200000E0
:10595000636F00006D6D0000616E00006420000048
:1059600066610000696C0000656400002062000050
:10597000656300006175000073650000207400001D
:1059800068650000207200006F7400006174000000
:105990006F720000206D000061790000206200003D
:1059A00065200000636F00006E6E000065630000FC
:1059B0007465000064200000746F00002074000013
:1059C00068650000206600006F63000075730000CA
:1059D00065720000207000006F720000740000000B
:1059E0005468000065200000636F00006D6D0000CA
:1059F000616E00006420000066610000696C0000B8
:105A000065640000206200006563000061750000AD
:105A100073650000207400006865000020720000BB
:105A20006F740000617400006F7200002069000054
:105A3000732000006174000020740000686500009D
:105A4000206C0000696D0000697400000000000017
:105A50000000000000000000000000000000000046
:105A60000000000000000000000000000000000036
:105A70000000000000000000000000000000000026
:105A80000000000000000000000000000000000016
:105A90000000000000000000000000000000000006
:105AA00000000000000000000000000000000000F6
:105AB00000000000000000000000000000000000E6
:105AC00000000000000000000000000000000000D6
:105AD00000000000000000000000000000000000C6
:105AE00000000000000000000000000000000000B6
:105AF00000000000000000000000000000000000A6
:105B00000000000000000000000000000000000095
:105B10000000000000000000000000000000000085
:105B20000000000000000000000000000000000075
:105B30000000000000000000000000000000000065
:105B40000000000000000000000000000000000055
:105B50000000000000000000000000000000000045
:105B60000000000000000000000000000000000035
:105B70000000000000000000000000000000000025
:105B80000000000000000000000000000000000015
:105B90000000000000000000000000000000000005
:105BA00000000000000000000000000000000000F5
:105BB00000000000000000000000000000000000E5
:105BC00000000000000000000000000000000000D5
:105BD00000000000000000000000000000000000C5
:105BE00000000000000000000000000000000000B5
:105BF0004375000072720000546500006D70000073
:105C0000203D000020250000730000004E6F0000C2
:105C100020500000726F0000626500000043000029
:105C2000757200007253000074650000702000005F
:105C30003D200000256C000075000000546100004C
:105C4000726700005374000065700000203D000082
:105C5000202500006C75000000490000734D000015
:105C60006F760000696E0000672000003D20000094
:105C70002575000000490000734800006F6D0000AA
:105C8000696E0000672000003D20000025750000BF
:105C90000049000073200000486F00006D6500009F
:105CA000642000003D200000257500000054000025
:105CB000656D000070500000726F000062200000EF
:105CC0003D2000002575000000520000656D0000B9
:105CD0006F740000654900004F2000003D20000067
:105CE0002575000000480000435300007461000067
:105CF00074750000732000003D2000002575000031
:105D0000004800006F6D0000652000005377000020
:105D1000692000003D200000257500000000000003
:105D20000000000000000000000000000000000073
:105D30000000000000000000000000000000000063
:105D40000000000000000000000000000000000053
:105D50000000000000000000000000000000000043
:105D60000000000000000000000000000000000033
:105D70000000000000000000000000000000000023
:105D80000000000000000000000000000000000013
:105D90000000000000000000000000000000000003
:105DA00000000000000000000000000000000000F3
:105DB00000000000000000000000000000000000E3
:105DC00000000000000000000000000000000000D3
:105DD00000000000000000000000000000000000C3
:105DE00000000000000000000000000000000000B3
:105DF00000000000000000000000000000000000A3
:105E00000000000000000000000000000000000092
:105E10000000000000000000000000000000000082
:105E20000000000000000000000000000000000072
:105E30000000000000000000000000000000000062
:105E40000000000000000000000000000000000052
:105E50000000000000000000000000000000000042
:105E60000000000000000000000000000000000032
:105E70000000000000000000000000000000000022
:105E80000000000000000000000000000000000012
:105E90000000000000000000000000000000000002
:105EA000000000000000000000000000004E0000A4
:105EB000696300006B6E0000616D000065200000EA
:105EC0003D20000025730000004D000061780000B7
:105ED0005374000065700000732000003D20000036
:105EE000256C00007500000044650000762000006D
:105EF0005479000070650000203D0000202500005E
:105F000063000000544300006F6D0000702000002B
:105F10004F6E0000203D000020250000317500007C
:105F200000540000434D00006F6400006520000035
:105F300025630000203D00002025000064000000D3
:105F40004375000072720000656E0000544300004B
:105F5000203D00002025000063000000424C0000AE
:105F6000436F00006D7000004F6E0000203D000088
:105F70002025000075000000424C00004353000043
:105F80007465000070730000203D000020250000B3
:105F900075000000544300002053000074610000AD
:105FA00072740000203D00002025000075000000F4
:105FB000484F00006E5300007461000072740000CE
:105FC000203D0000202500007500000000000000BA
:105FD00000000000000000000000000000000000C1
:105FE00000000000000000000000000000000000B1
:105FF00000000000000000000000000000000000A1
:106000000000000000000000000000000000000090
:106010000000000000000000000000000000000080
:106020000000000000000000000000000000000070
:106030000000000000000000000000000000000060
:106040000000000000000000000000000000000050
:106050000000000000000000000000000000000040
:106060000000000000000000000000000000000030
:106070000000000000000000000000000000000020
:106080000000000000000000000000000000000010
:106090000000000000000000000000000000000000
:1060A00000000000000000000000000000000000F0
:1060B00000000000000000000000000000000000E0
:1060C00000000000000000000000000000000000D0
:1060D00000000000000000000000000000000000C0
:1060E00000000000000000000000000000000000B0
:1060F00000000000000000000000000000000000A0
:10610000000000000000000000000000000000008F
:10611000000000000000000000000000000000007F
:10612000000000000000000000000000000000006F
:10613000000000000000000000000000000000005F
:10614000000000000000000000000000000000004F
:106150000000000000000000000000004375000087
:10616000727200005374000065700000203D000052
:10617000202500006C7500000054000061720000D2
:106180006753000074650000702000003D2000008F
:10619000256C0000750000004C6100007374000065
:1061A0005374000065700000203D000020250000B1
:1061B0006C7500000043000075720000656E000001
:1061C00074500000412000003D200000256C0000BC
:1061D00075000000546100007267000065740000E3
:1061E00050410000203D0000202500006C7500009B
:1061F00000490000734D00006F760000696E0000DA
:10620000672000003D2000002575000000490000C7
:10621000734800006F6D0000696E00006720000089
:106220003D2000002575000000490000732000009B
:10623000486F00006D650000642000003D200000F4
:1062400025750000000000000000000000000000B4
:10625000000000000000000000000000000000003E
:10626000000000000000000000000000000000002E
:10627000000000000000000000000000000000001E
:10628000000000000000000000000000000000000E
:1062900000000000000000000000000000000000FE
:1062A00000000000000000000000000000000000EE
:1062B00000000000000000000000000000000000DE
:1062C00000000000000000000000000000000000CE
:1062D00000000000000000000000000000000000BE
:1062E00000000000000000000000000000000000AE
:1062F000000000000000000000000000000000009E
:10630000000000000000000000000000000000008D
:10631000000000000000000000000000000000007D
:10632000000000000000000000000000000000006D
:10633000000000000000000000000000000000005D
:10634000000000000000000000000000000000004D
:10635000000000000000000000000000000000003D
:10636000000000000000000000000000000000002D
:10637000000000000000000000000000000000001D
:10638000000000000000000000000000000000000D
:1063900000000000000000000000000000000000FD
:1063A00000000000000000000000000000000000ED
:1063B00000000000000000000000000000000000DD
:1063C00000000000000000000000000000000000CD
:1063D00000000000004E0000696300006B6E0000CA
:1063E000616D0000652000003D2000002573000065
:1063F000004D0000617800005374000065700000DB
:10640000732000003D200000256C00007500000096
:10641000446500007620000054790000706500009B
:10642000203D00002025000063000000424C0000D9
:10643000436F00006D7000004F6E0000203D0000B3
:106440002025000075000000424C0000435300006E
:106450007465000070730000203D000020250000DE
:1064600075000000484F00006E530000746100008A
:1064700072740000203D000020250000750000001F
:1064800069520000657600006572000073650000C7
:10649000203D000020250000750000004D61000037
:1064A000785300007065000065640000203D000026
:1064B0002025000075000000707200006F7400005D
:1064C0006563000074000000736E00006D700000D2
:1064D00000610000646D0000696E0000006D000046
:1064E00069630000726F000063680000697000005B
:1064F00000730000656E0000644300006D640000DE
:10650000006600006F630000757300006572000094
:10651000312E0000687400006D0000006E65000000
:10652000747700006F7200006B2F0000636F000033
:106530006E660000696700002E680000746D000040
:10654000000000000000000000000000000000004B
:10655000000000000000000000000000000000003B
:10656000000000000000000000000000000000002B
:10657000000000000000000000000000000000001B
:1065800000690000700000006777000000730000E1
:1065900075620000006400006E73000031000000AE
:1065A000646E000073320000006D00006163000043
:1065B000006800006F730000740000006468000051
:1065C00063700000002F00006E650000747700000B
:1065D0006F7200006B2F000072650000626F000098
:1065E0006F7400002E680000746D00003F00000012
:1065F000256400002E250000642E000025640000A4
:106600002E250000640000002F6E0000657400005D
:10661000776F0000726B00002F6300006F6E000048
:1066200066690000672E0000687400006D000000BD
:106630004175000067200000203500002032000076
:106640003032000036200000313400003A340000BF
:10665000323A00003338000000760000352E00008A
:1066600034320000006E0000616D00006500000023
:106670006E6F00007420000073650000740000005D
:106680003C6200003E550000706C00006F6100002D
:106690006420000061200000466900006C65000075
:1066A0003C2F0000623E00000063000068650000AF
:1066B000636B000065640000006600006169000013
:1066C0006C00000054680000652000004479000060
:1066D0006E6100006D69000063200000444E000000
:1066E00053200000436C0000696500006E740000D8
:1066F00020690000732000006E6F0000742000000D
:10670000656E0000616200006C650000642E000090
:10671000006E00006F6E000065000000626C0000FB
:106720006F6300006B00000000000000000000002C
:1067300000000000002500006C750000004E000005
:106740006F200000507200006F62000065000000C2
:106750000000000000000000000000000000000039
:106760000000000074720000756500000066000003
:10677000616C000073650000000000000000000074
:106780000000000000000000000000000000000009
:1067900000000000000000000000000000000000F9
:1067A00000000000000000000000000000000000E9
:1067B00000000000000000000000000000000000D9
:1067C00000000000000000000000000000000000C9
:1067D00000000000000000000000000000000000B9
:1067E00000000000000000000000000000000000A9
:1067F0000000000000000000000000000000000099
:10680000003300003630000030300000300000005F
:106810000000000000000000000000000000000078
:106820000000000000000000000000000000000068
:106830000000000000000000000000000000000058
:106840000000000000000000000000000000000048
:106850000000000000000000000000000000000038
:106860000000000000000000000000000000000028
:106870000000000000000000000000000000000018
:106880000000000000000000000000000000000008
:106890000000000000250000752E00002575000096
:1068A0002E25000075000000000000000000000020
:1068B00000000000000000000000000000000000D8
:1068C00000000000000000000000000000000000C8
:1068D00000000000000000000000000000000000B8
:1068E00000000000000000000000000000000000A8
:1068F00000000000000000000000000048650000EB
:1069000072630000756C0000657300002056000083
:10691000320000004865000072630000756C0000E2
:106920006573000000470000656D0000696E00009F
:10693000692000005632000000470000656D00002D
:10694000696E0000690000004745000054430000E4
:106950004647000000530000455400004C4500002D
:106960004400000047450000544400004247000036
:1069700000520000454200004F4F0000540000004C
:1069800052450000534500005448000000570000E5
:1069900046530000534900004400000057460000E1
:1069A00053450000434D00000057000046530000CF
:1069B000454300004B0000005746000057450000CB
:1069C000504B000000500000555300004857000095
:1069D0004600000057520000455300004554000097
:1069E00000570000494600004952000042000000E4
:1069F0005746000053430000414E0000004700008E
:106A0000455400004E450000540000004E58000060
:106A1000544E00004554000000470000455400005B
:106A20004849000050000000534500005453000046
:106A30004950000000530000455400004853000036
:106A40004D0000005345000054480000534700002B
:106A5000005300004554000048530000440000006B
:106A6000534100005645000049500000005300000B
:106A700049500000525300005400000047450000F8
:106A800054570000495000000053000045540000D6
:106A900057490000500000005345000054570000C3
:106AA000534D0000005300004554000057530000B0
:106AB00047000000534500005457000053440000B5
:106AC00000530000415600004557000046000000FA
:106AD0005345000054440000445600000053000099
:106AE0004554000053450000520000004745000097
:106AF00054530000455200000025000075000000BE
:106B00005345000054000000535400004F52000051
:106B1000450000004445000046410000554C00007F
:106B2000545300000052000045530000455400003B
:106B300000530000434100004E000000256C00009F
:106B400075000000000000000000000000000000D0
:106B50000000000000000000000000000000000035
:106B60000000000000000000000000000000000025
:106B70000000000000000000000000000000000015
:106B80000000000000000000000000000000000005
:106B900000000000000000000000000000000000F5
:106BA00000000000000000000000000000000000E5
:106BB00000000000000000000000000000000000D5
:106BC00000000000000000000000000000000000C5
:106BD00000000000000000000000000000000000B5
:106BE00000000000000000000000000000000000A5
:106BF0000000000000000000000000000000000095
:106C000000000000000000000000000045740000CB
:106C100068200000536F0000636B00006574000083
:106C20002044000069730000636F00006E6E000076
:106C30006563000074200000436F0000756E000063
:106C4000743A0000203D000020250000750000007F
:106C50004574000068200000536F0000636B000063
:106C600065740000204300006F6E00006E65000038
:106C700063740000204300006F7500006E74000014
:106C80003A2000003D20000025750000004500006E
:106C900074680000204200007974000065730000F1
:106CA00020520000783A0000203D0000202500001E
:106CB0006C750000000000004745000054440000CF
:106CC0004E4E0000004700004554000053540000A1
:106CD00041000000474500005443000046470000C3
:106CE000004400004F480000414C000054000000E8
:106CF00053450000544400004E4E0000004D00007B
:106D00004F5600004142000053000000444F000075
:106D1000484F00004D45000000430000454E000074
:106D2000544500005200000053450000544200004A
:106D3000434500000053000045540000424300005A
:106D40005300000053450000544800004F5300001A
:106D5000005300004554000054430000450000006B
:106D60005345000054540000435300000044000009
:106D70004F4D00004F56000045000000444F0000FA
:106D8000535400004F5000000053000045540000D1
:106D9000544300004D0000005345000054540000CF
:106DA00043430000005200004553000045540000DA
:106DB00046000000534500005444000045560000C2
:106DC000004D00004F5600004557000046000000EF
:106DD000464F0000524300004548000000460000B6
:106DE0004F52000043450000500000004E69000073
:106DF000636B00006E6100006D650000203D0000C7
:106E000020000000256C00007500000025750000C2
:106E10000000000047450000544400004E4E0000B2
:106E2000004700004554000053540000410000009A
:106E3000474500005443000046470000004400005E
:106E40004F480000414C0000540000005345000032
:106E5000544400004E4E0000004D00004F5600000C
:106E60004142000053000000444F0000484F000022
:106E70004D4500000053000045540000484F0000FD
:106E800053000000444F00004D4F000056450000E5
:106E9000004400004F530000544F00005000000019
:106EA00052450000534500005452000000530000BA
:106EB00045540000524500005600000053450000B4
:106EC00054440000455600000053000045540000A3
:106ED00042430000450000005345000054420000BA
:106EE00043530000004D00004F5600004550000085
:106EF000410000004D4F000056450000574600007D
:106F0000004400004F520000414D000050000000BE
:106F1000464F000052430000454800000046000074
:106F20004F52000043450000500000005345000050
:106F3000544C0000494D000000550000534500002E
:106F40004C4900004D0000004E690000636B0000DA
:106F50006E6100006D650000203D00002000000013
:106F6000256C000075000000257500000000000081
:106F70003000000073720000632F0000436C0000BB
:106F8000696500006E740000436F00006E6E0000C3
:106F900065630000746900006F6E0000732F0000CD
:106FA000436C0000696500006E7400002E630000F1
:106FB00000250000733A000025690000202500002C
:106FC000732000002D2D000020610000737300006D
:106FD00065720000746900006F6E0000206600009A
:106FE000616900006C650000640A00000021000077
:106FF00000000000004500004E440000007000004A
:107000005F6300006C690000656E0000742D000075
:107010003E770000726900007465000000450000C2
:10702000525200004F52000020490000442000004E
:107030003D20000025640000004500005252000081
:107040004F5200002054000045580000542000001A
:107050003D2000002573000000210000000000001A
:10706000507200006F670000726100006D20000028
:107070007374000061720000740000005069000029
:1070800063200000496E0000697400000054000095
:10709000696300006B200000496E00006974000005
:1070A000004D00005046000053200000496E0000D3
:1070B000697400000041000070700000204300006F
:1070C0006F6E00006669000067200000496E0000D6
:1070D000697400000053000074610000636B0000DD
:1070E000204900006E69000074000000436C00003D
:1070F000696500006E74000073200000496E000096
:10710000697400000A4200006F6F000074200000E4
:10711000436F00006D7000006C6500007465000036
:107120000000000004A30000000000000047000071
:10713000454D0000494E00004900000008000000D5
:10714000C80000002C01000008000000C80000007A
:107150002C01000008000000C80000002C01000005
:107160000A00000080010000800000000A0000000A
:1071700080010000800000000A0000008001000083
:107180008000000032320000303200003230000057
:1071900000000000000000000000000000000000EF
:1071A00000000000000000000000000000000000DF
:1071B0000000000000000000000000000D0A0000B8
:1071C00044480000435000002F5000006F7700003B
:1071D0006572000020650000766500006E74000096
:1071E000206F00006363000075720000726500008C
:1071F000640000004D5000004653000002010000F2
:04720000000000008A
:020000040000FA
:107204008040780080D7BF00814F50000F003200CB
:10721400E24F400004003200100B07000E0009008A
:1072240030197800E201B1000100780080F7B7005E
:10723400E2CF40000500320001407800070B070050
:107244000E00090032187800E201B10000000600C7
:1072540081D7BF0001782100914078000104E1004A
:1072640017003200E24F40000C003200E2C1B300CC
:107274000440BC007C03410045CB200062807A00BE
:1072840081FD2F00010040008402200013C0B300E0
:1072940082D62000E6C07A006C0A070080D7BF00BF
:1072A40081F7B70082FD2F00616E8000010141006B
:1072B40084022000160B070080D62000630A070012
:1072C40000000600889FBE008A9FBE008C1F7800C5
:1072D4008217E20007003A0048C2020000000000E2
:1072E400F27F200002006000024020000200400003
:1072F40010BC8800C20320008000EB0000D92000ED
:10730400FE0C02000000000048F920000005EB001C
:10731400F9892B000A407800B9FF07000900E8004A
:107324009000780063804400100178001904E000A4
:1073340008003A000280400008004000AB02200030
:107344008085450000ED2100808F55000200360045
:10735400FFFF3700FFFF3700E86DEF0080022000D9
:1073640008004000606E8800008040000000E800D3
:10737400706E880000004100806E8800D0002000FC
:10738400106F8800E46DA900B1FF070079F8970039
:107394008FEDB700FC0607000A05E800E684440008
:1073A400E60F5500020032000B047800D9FF3700C5
:1073B4004F0678004F05BE004F04BE0000000600D3
:1073C4000400FA00889FBE008A9FBE008C1F7800CC
:1073D40090BF9F00A1BF9F008245780003067800FC
:1073E400844478000004EB000845780008407800E5
:1073F40083FF0700106F8000ED0F50005B003A0020
:1074040093FF0700094078008F4DE30057003A00CE
:1074140080212000606C88000B04E00006003A0024
:10742400CC6B8800E46DA80040002000106F880039
:107434003C6F88004B00370000C02F008217B40057
:1074440081F82000810F5000020036000040200027
:1074540010BC880010BC8000C06B88000000E800ED
:1074640010BC8800BC6B88005C00020001000000B6
:10747400D06E8800E16E8800E48DA800E3CF55004B
:107484001400320003003E00E1CF550035003900FE
:1074940003003700E4CF550032003A0019003700EA
:1074A400740A07000B4078000014A2000080FB005F
:1074B4000000E9004F00DE004200DD00516C800056
:1074C4000120A10080807000516C8800E22DEF0043
:1074D400240037002FB897009FB8970001004000A0
:1074E40000004600C16B800001006800306F880016
:1074F400600A0700640A070020002000106F88005B
:10750400180037001FB99700224090000080FB004C
:10751400B2409000C808DD00808070009281FB00BA
:10752400124090004800DD0003007000808040009D
:1075340081004600C06B800080806800316F880045
:10754400E0D720000900090032587800A200B100F9
:1075540050002000106F880011C0B30020C0B30099
:10756400820407000A80FB00040037000804E800D6
:10757400E60F54009CFF3A00E00F20004F0678000D
:107584004F05BE004F04BE000080FA000000060054
:1075940011002000E54F500009003E0018FF0700CD
:1075A400216F8000000021000080600002003A008A
:1075B4008000780002003700E58DA900110020004A
:1075C40001007800000006008000EB00E54F500049
:1075D40005003E000AFF07008000EB002F0A0700A9
:1075E40001003A0011002000F5FF3700E54F50007C
:1075F40035003E0002FF0700B06E8000C06E8800B8
:10760400106F8000E50F50002E00320006003E008F
:10761400E10F50000D0032002A003900E30F500042
:1076240025003E0027003700EB0F50001500320004
:1076340003003E00E70F50001F003E000700370024
:10764400EE0F50001C003A001800370084B7020007
:10765400000000004C0607001B00370011C0B300F7
:1076640010C1B300410407007A0DE20002003200A9
:107674000D0A0700F9FF3A0080002000106F88000F
:107684001100370011C0B30010C1B3003704070064
:107694007A0DE20002003200030A0700F9FF3A0003
:1076A400C0002000106F880007003700D0002000C1
:1076B400106F8800040037008040EB0040C1B30025
:1076C4002A0407003006070000000600881F78001F
:1076D40000447800E54F500004003E00C8FE070057
:1076E400E46DA90008407800C0FF07004F0478004B
:1076F400000006008000EB00E54F500009003E004A
:10770400BFFE0700D2FE070080CA2000E1D7200098
:107714000900090031587800B06B8000906588003A
:1077240081CA2000A6FF3700E54F500006003E0046
:10773400B3FE0700C6FE0700DB09070002003200A3
:10774400DD0907000904070000000600E54F5000AA
:1077540012003E00AAFE0700E2CDBF00E74F500032
:1077640002003200EB4F50000C003A00926E800091
:10777400A16E8000810F510005003900D109070076
:1077840082805000010040000000E900040037003E
:10779400028050000000E900010037000000EB0007
:1077A400000006000200FA00889FBE000044780032
:1077B400A1FF9F00E54F500031003E0090FE0700FE
:1077C40008407800E1FF0700800478000000E00032
:1077D4002B003200E10F500002003A00084078000C
:1077E400D1FF0700E50DAB0007003A00B50907001B
:1077F4000000D100808F540003003E000840780050
:10780400C9FF0700E50DA800BB090700906E8000C2
:107814001400200084417800668157000B0907009A
:10782400916E80008100E800916E8800706E800087
:10783400808F500002003900606E8000906E8800D6
:10784400E18F540004003A0008407800B6FF0700B6
:10785400090078000B00370010002000E4ADAB00F5
:1078640008003A00E4ADA800740002000100000022
:1078740078004000F06E88001000200001003700FE
:107884000000EB004F04BE000080FA000000060078
:10789400889FBE008A9FBE008C9FBE000044780073
:1078A40001067800820578000000EB00E54F5400E3
:1078B4003F003E000840780051FE07000840780071
:1078C400A2FF0700000578000000E00004003A0071
:1078D4000840780094FF07000A007800340037005D
:1078E4008B0F5000020036008B0478000100370033
:1078F40080047800E50DAB0007003A007109070029
:107904000000D100800F550003003E0008407800BD
:1079140085FF0700E50DA800956E8000716E80005C
:10792400058044008006EB00810F50000B003900F5
:1079340085865000700907000D02780013C0B3005B
:107944000C01780005007800C00807000D06460009
:107954008D845400606E8000906E88006609070074
:10796400906E80000902780013C0B3000C01780007
:10797400B608070009007800D22DB4008B0F55001B
:1079840003003E000840780067FF07000700370047
:10799400E4ADAB0005003A00E4ADA80074000200B9
:1079A4000100000078004000F06E88000980460065
:1079B4004F06BE004F05BE004F04BE000000060087
:1079C400889FBE008044780001047800010078009C
:1079D400F00D02000000000000017800880078002B
:1079E40009407800AAFF0700000044004F04BE00CD
:1079F40000000600889FBE00804478000000EB0071
:107A0400E5CF540009003E0009407800FCFD070062
:107A1400686E8000706E8000080450000804E9005D
:107A24000940780049FF0700000054004F04BE00DD
:107A340000000600881F7800004478000A00070050
:107A44000000E0000600320008407800ECFD07006A
:107A5400B06E8000C06E880017090700430307005A
:107A64004F047800000006008000EB00E54F500052
:107A74000B003E00E2FD0700150907000200390073
:107A84008100510006003700806E800081005000A4
:107A9400706E800000005100808040008100E8008A
:107AA400C7FE3700889FBE008A1F78000044780014
:107AB40001057800ECFF0700800478000000E00076
:107AC4001500320008407800CDFD07000A00E000F0
:107AD40006003200C26E800014002000090907006D
:107AE400844078000A00780058080700C16E8000BE
:107AF4008100E800C16E8800806E8000808F500095
:107B040002003600706E8000C06E8800E18F540061
:107B140003003A00E54DA800090078000900370089
:107B240010002000E4ADAB0006003A00E4ADA8006C
:107B34007400020001000000A007B000F06E88008D
:107B4400100020004F0578004F04BE00000006001E
:107B5400889FBE008A9FBE0080447800810578001B
:107B640002047800C0FF0700000578000000E00070
:107B74002C00320009407800A1FD0700880F550051
:107B8400010031000A047800C26E8000816E80001A
:107B9400020044008004EB00810F50000B0036000B
:107BA400028050008004E8000B00E0000400320072
:107BB400090278006A08070024080700898545003F
:107BC40009045400706E8000C06E88000B00E00051
:107BD40003003200C26E8000530807001B08070030
:107BE40008007800D82DB40008844400080055002B
:107BF400800F540003003900E54DA8000800780008
:107C040008003700E4ADAB0005003A00E4ADA8007D
:107C14007400020001000000A007B000F06E8800AC
:107C2400080078004F05BE004F04BE0000000600A7
:107C3400889FBE00804478000000EB00E5CF54002C
:107C440008003E00094078006DFD0700786E800052
:107C5400806E8000080450000940780082FF07000D
:107C6400000054004F04BE0000000600889FBE00C0
:107C74008A9FBE00004478008105780002057800E0
:107C840083047800E54F500022003E000200E0002B
:107C9400200032005AFD07000840780072FF0700F8
:107CA4008000780009004500808F500001003100F9
:107CB40009855000C06E800000814400816E800000
:107CC400810F51000100360028080700028050008F
:107CD4000004E800880F550005003E000A02780001
:107CE4001F080700D90707000A0078000A003700B8
:107CF4000D080700D5070700726E80000B004400D2
:107D04000802550082080700D00707000A0078001F
:107D1400010037000000EB004F05BE004F04BE0019
:107D2400000006000200FA00810178001200200021
:107D34008F80E900CDFF0700EFF897000180FB007A
:107D44000080FA00000006000F03B000889FBE0008
:107D54008A9FBE008C9FBE008E1F7800004478006E
:107D6400E1B79F00F2B79F00830578008404780090
:107D740085BF9F00E54F5000A1003E000200E000D7
:107D84009F0032001EFD07000840780036FF070000
:107D94000B0750007FB097008E0F50009A003E00F2
:107DA4000900E00003003200890F5700010036008B
:107DB40009077800C06E800000814500816E800054
:107DC400810F510001003600E807070002805000CF
:107DD4000000E800C0B79F00EFB09700A1B79F0074
:107DE400B1447800A1B79F000FBA97000400E000E7
:107DF40006003200F0C9B30000C04400F94F50003F
:107E040002003E0000CEB30080C444007FB597005A
:107E1400BBB79F00D2B79F002FB697008006EB0038
:107E24000BC2B3004FB09700FF0F500001003E009B
:107E34008FED97000B80FB00800F5700010031008D
:107E44008E4578000B84FB00080278002D0807009B
:107E54005FB1970011C0B30040FC2F000F00400039
:107E64007A07070088027800DFB097008880400016
:107E7400D1B79F004FB2970008025200C4B79F00C9
:107E840004003A00706E8000D0B79F008080EB0041
:107E9400C1B79F000FBA97000400E0005F003A00EA
:107EA4005B0037000042EB0043FC2F008F81410050
:107EB400F6C9B30007CEB3003FB09700FFB09700F8
:107EC40001045000030178009340780006C040008C
:107ED400F94F500001003E0087C9400092CF540082
:107EE4000E003A000A05E90004003A000480FB0091
:107EF400000044000000E8004B003700BC44780058
:107F040006C044001D002000F94F500010003E0040
:107F140087C444001D0020000D0037000D00E00060
:107F240002003A007FB59700090037006FB0970050
:107F34009044780006C04400F94F500001003E0010
:107F440087C444007FB597002FB697008006EB00E6
:107F54000442E8008301E80084CF55002100320088
:107F6400D8FF37000041EB008000EB003FB29700E0
:107F74007FB097008001520044FC2F000F024200A2
:107F840064C0780080CF540009003A000A05E90073
:107F940004003A000280FB00008041000000E80079
:107FA40021003700BC4478001D0020000900370080
:107FB4000D00E00002003A007FB59700050037008D
:107FC4006FB09700904478007FB597002FB6970064
:107FD4008006EB000241E8008100E80082CF5500F2
:107FE400E5FF3A00050757008E0F550006003E00D6
:107FF400BFB0970085804000B1B79F0088FF37006D
:108004000000EB00080037000080EB00060037009A
:108014000B04E000D3FF3A00F2FF37000B04E0004A
:10802400A0FF3A00EFFF37004F0778004F06BE006D
:108034004F05BE004F04BE000F03B1000000060050
:108044000200FA00E1FF9F00840278000302780036
:1080540082017800120020008F80E9003AFF0700B7
:108064000080FA0000000600E6874700889FBE00F3
:108074008A9FBE008C9FBE008E1F78000005EB0017
:108084002E002000EDD820000A4678000A4078002F
:108094005BFC0700206F800001602000010060008D
:1080A40031003200C6600200000000000000E00061
:1080B4002D003200206F80004A00DE00E1056000E0
:1080C40009C1B3002A00370061FC07007440B900FD
:1080D4008001780002D9200002004000E1D720008E
:1080E40009000900B0587800A000B100EA804100FE
:1080F400E1007900B16B8800EC804100828040008F
:10810400160020000700200031024300A1824B002A
:10811400846B8800956B8800F16B8000076C80008D
:1081240087804000B26B800082804000C26B800078
:1081340082806800316F880061002000116F880020
:10814400620214007422B90041DA20000181410066
:1081540013C0B30083407800BC060700C82DEF00AD
:1081640029C1B300310037008044EB008005EB00E7
:10817400E4ADAB0007003200F86E8000740002002A
:1081840001000000000454004240A90001003C002A
:1081940009C1B300E4CDAB0007003200086F8000D2
:1081A4007400020001000000000454004240A900D1
:1081B40001003C0009C1B300106F8000EB0F5000B8
:1081C40009003A00086F80007400020001000000FA
:1081D400000454004240A90003003C00C0002000F9
:1081E400106F880019C1B300106F8000E40F5000B5
:1081F4000C003A00326F80000004EB0001DA20002A
:10820400110078000000E00006003200820F5000E8
:10821400ADFF32000804E800F4804000E30F54008E
:10822400F7FF3A000904E0000400320011C0B30073
:108234008BC05000094078004C010700E48DAB006E
:108244001D003A0015070700CF003A005C00020049
:1082540001000000CA060700CB003300216F800034
:1082640067806000E60F50000B003A00430CDE000C
:10827400614464000C407800DCFC07000C4078008A
:10828400DAFC07000804E000BF003A00E000200028
:10829400106F8800BC003700EDFB070021C0B3005D
:1082A40000C1B300310107005C00020001000000BE
:1082B4000B070700B40037005C0002000100000057
:1082C400AF060700B0003300E1FB0700106F800029
:1082D40001002000EC0F5000E08F580087003E00A2
:1082E400006001000C0037001C0037003700370025
:1082F4003F00370081003700570037006200370025
:108304006A003700710037008000370073003700BF
:10831400660037007500370078B7020000000000DF
:108324000000E0007500320011002000116F880089
:108334008A4DAB0004003200F06B80009EB702004F
:10834400000000006D003700F06B800011C0B30026
:108354009EB70200000000006800370072805700DA
:10836400C8B70200000000000000E0006300320013
:1083740084B70200000000000000E0000E0032009C
:108384007FB097008FB89700F06B8800016C88006D
:108394001E6F8800F06B8000800DB400B16B80000C
:1083A40001004000C16B800001006800306F88004C
:1083B400B5060700510037005C0002000100000010
:1083C400C7060700E22DEF004C00370074000200DE
:1083D40001000000F06E8800E0D7200020EB0200CE
:1083E4000000000030002000106F880043003700B8
:1083F40021D82000E0D720004CEB02000000000050
:108404000000E0000F003A007400020001000000C8
:10841400F26E800002005000426B8000820F500018
:10842400360036008ECDBF00E54F500003003E00FD
:108434000040E8008EEDB700560607001E6F880066
:108444002E00370050002000106F88000004EB005D
:1084540029C0B3004600370029C0B30012C0B300DE
:108464009D4F11006E0036000E0078008EEDB700AF
:10847400444B2C00446B880044002000546B88005B
:108484008E4478006600370015C0B3009DCF1200FB
:108494005E003600206F8000680060001B003A0018
:1084A40029C0B300000478001A00370026C0B300C6
:1084B4009D4F13005700360080002000106F880085
:1084C40019C1B3000004EB001200370027C0B30049
:1084D4009DCF1300510036000C00370020C0B300BC
:1084E4009D4F10004B0036000800370021C0B30038
:1084F4009DCF100049003600040037000004EB0053
:108504000904E00003003A001F00370049C1B3002A
:10851400180020000B00E000150032008E6DEC0006
:108524001C060700A06B8000A36E800003015000AE
:10853400830F500002003100620607000001410071
:10854400606B8000716B800002005000E080580076
:1085540066060700020078007A2DB400A36B880039
:108564008040EB00094078008000070003003700DA
:1085740011C0B300094078007C0007000800E00047
:1085840001003200800207000A05E800E60F5500EA
:10859400BDFE3A008004EB000AD920007448B900FB
:1085A400000478007000400060007D000000E000DE
:1085B4001D0032007400020001000000720144003A
:1085C40062017D000200500072722000820F500090
:1085D4000A003600628214007422B90042DA2000D4
:1085E400020144000A00440013C0B3008340780031
:1085F40096050700C82DEF008904E9008904E80006
:10860400E28F540008003E00E4FF370029C1B300A4
:108614000300370009C1B3000100370019C1B300DA
:108624000004EB00BDFF37004F0778004F06BE0083
:108634004F05BE004F04BE006F00B10000000600ED
:108644002000FA00889FBE008A1F7800800478000A
:10865400020578001082FB00104090004800DD0005
:1086640004017000294290000482FB00394090000C
:108674004800DD008401700072845700028CBE0043
:108684001101BE0092BF9F00A3BF9F000040EB00FA
:10869400E0F79F0060C0B300F0F79F00CABF9F00DF
:1086A4000A0078004EC5020000000000C0BF9F0011
:1086B400C1002000080078008EC502000000000000
:1086C400000478000A0078003E6402000000000004
:1086D4008880EA00808F50001D003A000000EB0003
:1086E4002CFB02000000000041012000A0FD2F002F
:1086F4000F0040007266020000000000A0FD2F0081
:108704000F004000FC0107003FB097004400DE006A
:108714006F4060004200DD00744050000080FB00A8
:10872400000055007404500089007800A0FD2F005B
:108734000F0040005B0107000000E000040032006D
:1087440088007800A0FD2F000F0040007A02070087
:10875400DC60020000000000100020004F057800DB
:108764004F04BE000080FA00000006002600FA0054
:10877400889FBE008A9FBE000044780001457800AF
:10878400B3FA07000808A30002003200E56DA80050
:108794000804A100E4ADA900E4CDA900E4EDA9001A
:1087A400E52DA900E54DA900E50DA900C66002006C
:1087B400000000000000E000FCFF320066006400DE
:1087C4008004EB004E003A00906E8000A26B8000A3
:1087D4008004EB00820F50003E003200110036008E
:1087E40002005000D16B8000810F50000100360060
:1087F40001007800696C8000890F500002003E007F
:108804008004780001003700E54DA80009027800D3
:10881400670507000D05070009007800742DB400F2
:108824002C003700716E800082815000B3BF9F001E
:1088340083004000606E800000805000D16B800097
:10884400810F50000100360001007800696C80003F
:10885400890F500002003E008004780001003700B8
:10886400E54DA800838F540001003100B9BF9F007B
:108874003FBA97004E050700F40407003FB897007D
:1088840000825400B4BF9F0008003200626E800072
:10889400A06B8000CE0DB500919D2000010040002A
:1088A400980507008040EB00E8040700A06B8000F7
:1088B40080804400A16B8800726E8000828F50001B
:1088C40004003900606E80000000510000805000F8
:1088D400A06B8800E56DAB0007003200D06B800010
:1088E400808F540004003200606C8000808F54003C
:1088F400010032000804A0000900E00002003A0070
:108904006300640011003200090078007A2DB5007C
:108914000900E000010032000834A0000A08A300A6
:10892400050032008E6DEF00D1122300416B8800E8
:1089340011002000516B88005C000200010000005F
:10894400FB040700E48DA800250037000A18A300E3
:108954000E003200206F80008040E800E780600055
:1089640082FF2F000200600001007000206F880069
:10897400606B8000716B800061005000E0805800E3
:108984005A0507001900200015003700206F8000E9
:108994007000600002003A00800478001000370084
:1089A4000A08A3000A003A008ECDBF000800320076
:1089B4000040E9008EEDB700406B8000516B8000F1
:1089C4008100D1000080D300406B8800516B880087
:1089D4005C00020001000000D50407008004EB00E5
:1089E40041FD2F0001804700C26B8000020878001F
:1089F400B16B800011009800626B8000736B800083
:108A0400C2AF9F00D3AF9F00ED040700E0AF9F000B
:108A1400F1AF9F000FB09700F1FF23000100600049
:108A240001FF2F000100600080B79F0098E79F00BE
:108A34000000EB00B0B79F0009014100E08149004C
:108A4400626B8800736B88008880FB000100D10092
:108A540061006000804578000004E00013003200EB
:108A64000148A30003003A006000B800E0AF9F0093
:108A7400F1AF9F008A2DAB00070032004FA897008A
:108A8400DFA8970061005000E0805800C0AF9F004D
:108A9400D1AF9F000500370061014100E08149002A
:108AA400626B8800736B88008A2DA8000808A300F5
:108AB400010032008A0DA8000505070006003900F0
:108AC400706E8000D00DB50081005100010050008F
:108AD40090B79F0003003700028050000000E900B7
:108AE40090B79F000661020000000000800078003B
:108AF40090AF9F00F0032000808F500003003E00E1
:108B04008000EB0091AF9F000300370000FC2F00B2
:108B14000080400090AF9F009FA897001FB097006F
:108B2400810F50000100360091B79F0042FD2F00D5
:108B340002804700F000070074854400F2F02F0023
:108B44000FB09700820060000105B30081B79F0059
:108B54000B04E0000A0032007885440020C0B30012
:108B640080EF9F0040C0B30090EF9F002080210061
:108B7400D0B79F00028060000006B30080B79F005A
:108B840021802000914078008180FB0003C8BF0051
:108B94004800DD0001017000418020009140780010
:108BA4008180FB0005C8BF004800DD008101700022
:108BB40074845700028CBE00F06B8000016C80004E
:108BC40080BF9F0091BF9F000040EB00C0F79F0053
:108BD40069C0B300D9F79F00BABF9F000A007800AC
:108BE4004EC5020000000000B0BF9F00C10020007D
:108BF400080078008EC50200000000000080EA0032
:108C0400A0B79F00109B20009663020000000000A4
:108C14000A01780089407800E0D72000A4FA020015
:108C2400000000004101200042FD2F0002804700A7
:108C340012670200000000000B04E0000400320090
:108C440041002000788057001267020000000000F5
:108C5400509C2000C0630200000000000A0078005D
:108C64003E6402000000000090AF9F00509D200071
:108C740096630200000000002100200020FD2F0068
:108C84000F00400012670200000000007262020040
:108C9400000000004F05BE004F04BE000080FA0033
:108CA40000000600889FBE008A9FBE008C1F7800CB
:108CB4008005780001067800900190000300E00030
:108CC40088003200214090000080FB00B1409000F9
:108CD400C808DD00808070001C81FB001C409000EF
:108CE4004800DD0002007000808040009B8040004E
:108CF40001856900E9CFB3000004EB000840780067
:108D04003FF90700106F8000ED0F5000180032008B
:108D1400E40F500006003A009B009000306F800082
:108D2400810F500012003A00884478001000370088
:108D3400306F8000800F55000D003A0044F90700A1
:108D44009B009000C06B8000808F500008003A00A8
:108D5400B06B80009B0F100005003A001B04070055
:108D6400F06B8000016C80002204070015003200C3
:108D74000804E800E60F5400E0FF3A00E2CF4400A4
:108D840031003200094078001DF9070030F907006E
:108D94003A6F8800E0D72000090009003C587800A9
:108DA400AC00B1001B017800B26B88009B059000F9
:108DB400CB6B8800636E8000A36B880010002000DA
:108DC40049003700100020004700370074000200FB
:108DD400010000007449B9007201410004D9200067
:108DE40000317A000000EB003F003700744CB900FA
:108DF4000AD920000A004400090009003C58780000
:108E0400A000B100AC00B1006A0044001B307D003A
:108E14000A0044002B019000BB01900062009800FE
:108E240073009800700044009B0590000B307D0097
:108E340074000200010000007204440000347D004C
:108E44000000EB00280037006B0090000098A3009E
:108E540024003200C80DE20022003A008004EB0036
:108E640004DA2000940078000100E00010003200D1
:108E74001B009000808F500009003A0054B89700FE
:108E84009B0F500006003A00D003070004B8970077
:108E940094B89700820F5000838F5800CBFF3200A4
:108EA4008904E80074024200E38F5400EDFF3A00A5
:108EB4000004EB0008407800D1F80700E46DAB0033
:108EC40005003200E2F807009B009000C06B8000B0
:108ED400810F5000C5FF32000804E800E60F54007B
:108EE400F4FF3A000000EB004F0678004F05BE0087
:108EF4004F04BE0000000600881F780000047800BC
:108F0400100078004EC5020000000000000C78003C
:108F1400180090004EC502000000000010049800E4
:108F240028009000B800900060C502000000000016
:108F3400200498003104980048009000D800900064
:108F440060C502000000000040049800510498002D
:108F5400780090004EC502000000000070049800E4
:108F6400080890004EC5020000000000000C9800A4
:108F7400180890004EC5020000000000100C980074
:108F84004F04780000000600B1F80700C06B8000B1
:108F9400306F8800606E8000906E8800A06E88003C
:108FA400706E8000B06E8800C06E880040002000A3
:108FB400E46DAB0001003A00D0002000106F88007F
:108FC400E40DA900E42DA900E44DA900E48DA90055
:108FD400E4ADA900E4CDA900E4EDA900E50DA900E4
:108FE400E52DA900E54DA900E56DA900E58DA800D2
:108FF4008A0DA9008A2DA9008A6DA9008A8DA9006D
:10900400606E8000A06B88000EC2020000000000A9
:10901400606B88000EC2020000000000706B8800C4
:1090240088ADEF0010002000D06B8800000006001F
:109034000200FA00889FBE00C00020002CFB020042
:10904400000000005C66020000000000000FB20097
:109054004280DE00F44450003300320071002000EE
:109064000000EB0072660200000000002B003700D5
:109074005C660200000000000004E0002A003200E8
:10908400E14F500025003200E24F500017003A0033
:10909400E2CF5400240036000000EB00D0BF9F0054
:1090A4005C66020000000000E44F500006003A0035
:1090B4005C66020000000000B0FF9F005C660200D6
:1090C40000000000A0FF9F00DFB89700702120007F
:1090D400808F500014003600D039B000808F5000CB
:1090E40012003E000100780010003700E1CF540068
:1090F4000D0036005C6602000000000000447800A9
:10910400894F500008003E008080FB000000EB0007
:10911400726602000000000088C454008944E9001B
:10912400E1CF4400D2FF3A00802120004F04BE006A
:109134000080FA0000000600F0874700889FBE0008
:109144008A9FBE008C9FBE008E1F780000057800A9
:1091540001077800504C900040069000D006900023
:10916400B000900020009000D0B79F00E1B79F00AE
:10917400E40DA900E42DA900E44DA900E48DAB00A1
:1091840003003A005C0002000100000054030700E1
:10919400146F8000E40F520003003200E50F520008
:1091A40045003A00160037000880FB000028A300A1
:1091B40038023A000048A300060032006C6B8800B5
:1091C4007D6B88008040EB0040C0B30067FD070062
:1091D400300237000018A3002E0232005FB197005E
:1091E400EFB1970061014100E0814900826B880082
:1091F400936B88008EFF0700606C8800280037009E
:109204008880FB000128A30026023A004408DE00FF
:1092140061006000804578000004E0000A0032002C
:10922400686B8000796B8000880F5600898F5E0020
:1092340005003200F20207004CFD0700686B88004D
:10924400796B8800170237000118A3001502320059
:109254005FB29700EFB2970061024200E0824A00D9
:10926400846B8800956B88007A059000DA6B88001F
:109274006FFF0700606C88000B04E00008003200F8
:109284000D03070039FD070070002000106F8800EF
:109294005C00020001000000DE020700010237004A
:1092A40011C0B30020C1B30030FD070060002000EE
:1092B400106F8800FB0137008882FB00E1856200A3
:1092C4008BF79F000B04E00002003A00CEB79F002A
:1092D400020037008E00E800C1B79F000884FB003D
:1092E4000818A300030032004FB197000201E80000
:1092F400C2B79F00F602070005003900706E8000B7
:10930400D00DB500810051008104500002003700E7
:10931400028050008004E900A90207005FB19700B1
:10932400EFB1970000005100818059000001BE0098
:10933400F0B79F004FB397000600E0001E00320014
:109344000900E00027003200E00F5000E08F5800D1
:10935400040035006148B800820F5000838F580024
:1093640009003E004FB3970006004100E080490029
:109374004240A9000600340006805400CF80DE007D
:109384009C02070002003C00160020000100370088
:109394000003EB006148B800960207000F003D008F
:1093A400FFB097004FB19700028040004240A900EF
:1093B4000F003C0009003700E00F5000E08F580018
:1093C4000B003200070035006148B800820F5000DE
:1093D400838F580006003E00020037000600E000BC
:1093E40003003A000828A300AE013A00AB0137009D
:1093F40066806200A7013A000848A300A901320070
:10940400EB0F520005003E00E70F5200150031003B
:10941400E60F5200BB003A0003003700EC0F520085
:10942400B8003A00AF003700646B8000756B8000B1
:10943400A4B79F00B5B79F00840F5600858F5E00C8
:10944400060032006E020700C8FC07002FB0970028
:10945400BFB09700A50207009201370070002000FA
:10946400106F8800A46B8000926E8000840051000D
:1094740002003B009302070080804000626B800082
:10948400736B800001004100E08049000000560039
:1094940081805E004240A9000B0034008A0DAB00BD
:1094A40003003200E10F5000E08F58000400320046
:1094B4008040EB0000C1B300ACFC07007901370029
:1094C40061065600E0865E00A56E8000050052002D
:1094D400CF80DE000003510081835900850F5200C4
:1094E400020039000600BE000300370075020700C1
:1094F40000005300E0805B000001560081815E00A3
:109504004240A900280034006E0207000100200038
:109514003802070024003E008A6DA9008A8DA90044
:10952400E50DA900A06E800002024000A46E880030
:10953400A16B8000810F500005003E00810F520096
:10954400090036000100520035020700060037000A
:109554005C02070000804000800F520002003600C9
:10956400000052002E020700716E8000810F52002D
:1095740004003900606E800000805000000052003A
:10958400A06E8800A26B8000716E8000810F510074
:109594001A003900606E8000008050000000510005
:1095A400A06B880015003700850F520013003200AD
:1095B400506C80000038A3000F0032000048A30064
:1095C4000C003200666B8800776B8800A06B80000B
:1095D400808F5200050036003A020700CF80DE007B
:1095E4000000530081805B0040020700A56B8800E7
:1095F400E54DA8008A8DA8008A6DA800A16E8000A0
:10960400906E8000808F50000C003A00E56DAB0036
:1096140004003A005C00020001000000FD010700A4
:10962400060037000502070004003A008A0DAB006B
:1096340002003200E48DA900E56DA900636B80008F
:109644008C8051007A009000010050007A0DE200F5
:1096540003003A000000E00001003200E52DA800FC
:10966400D06B8800106F8000E80F50000D003A00A6
:10967400F201070023003A008A0DAB0021003200FA
:109684005C0002000100000022BC2E00B300200098
:10969400A9010700E48DA80090002000106F880045
:1096A40018003700E90F500009003A000B00E000F1
:1096B40014003A006C6B88007D6B88008B40780046
:1096C40040C1B30029FC07002FFE0700F500370056
:1096D400EA0F50000B003A00D8010700F1003A00ED
:1096E400EC003700646B8000756B80006100420001
:1096F400E0804A00800F5600818F5E00E9003A0046
:10970400E40037000858A300E6003A00106F800018
:10971400EB0F5000E3003200EA0F5000E10032008A
:10972400EC0F5000DF0032000E00E0009400320025
:10973400FFB597000B00E00044003C006A00900075
:109744004200DE00C003B2000B0050002CFB0200FC
:10975400000000007FB39700060547008A8F54007D
:109764000100310009057800950107000A00400056
:10977400E0804800806B8800916B8800B56E8000A3
:10978400816E800005004500810F50000E003600F8
:10979400058450000804E8006C0107002B01070051
:1097A40008045500D4010700706E80000802780098
:1097B400A701070025010700706E80000004440023
:1097C400B86E880006003700CB0107000A02780053
:1097D400600107001D0107000A007800D62DB400BF
:1097E400406C8000E10F4000650032008A005000A8
:1097F400416C8800E06B8000008140001100330060
:109804000100E0005E003C006D0107000200400022
:10981400E0804800806B8800916B8800B06E800007
:1098240080004100B16E8800806E8000808F5000FF
:1098340004003600CE0DB500008040000000E900B1
:10984400B06E880088ADEF004D003700FFB0970080
:1098540001004700808F540001003100018754004B
:109864006A0090004200DE00C003B2002CFB02003C
:1098740000000000B16E80007FB1970081024100BA
:10988400826E800005004700820F500016003600EB
:1098940001005100FFB19700030050000004E800EC
:1098A4000800330029010700E800070092010700BF
:1098B400706E80000802570065010700E30007008E
:1098C4000D0037008C01070002007800CE0DB500B2
:1098D400008042000000E9000E0278005C010700ED
:1098E400DA00070004003700830107000E02780045
:1098F40018010700D5000700406C8000E10F40000C
:1099040003003A004B6C8800EE6B88001C003700A3
:10991400800078007FB29700800F52000E00310063
:1099240004014700E06B800000804000800F51007C
:1099340002003E00828F500002003600EE6B880069
:1099440003003700FFB2970005005000E06B880069
:109954004B6C88000A0037007FB39700060147006C
:10996400E06B800000804000800F5100040036004E
:10997400800F530002003E0001005100E06B88009C
:109984004FB097000000E0001200320043010700CE
:1099940002003200B16E8000C16E8800E4EDAB00BD
:1099A400040032004401070070FB070028F607009A
:1099B40008003700E4EDA800E4CDAB0005003A0050
:1099C400E4CDA8007400020001000000D003B00040
:1099D400006F88000FF197000204E00031003200AC
:1099E400846B8000956B800061014200E0814A0035
:1099F4004FB397005FB29700EFB2970006004200A2
:109A0400E0804A00FB00070026003A00826B8800D1
:109A1400936B8800210107000F00320003003E0011
:109A2400E60F50001D003A0005003700E80F500013
:109A340010003200E90F500018003A0012003700FD
:109A4400C0002000106F880011C0B30010C1B30023
:109A540046FB070013003700B0002000106F880099
:109A64007400020001000000A007B000006F88002D
:109A74000A003700F100070003003200A0002000B4
:109A8400106F8800050037008040EB0000C1B30070
:109A940036FB07003CFD0700020037000601070003
:109AA40032FB07004F0778004F06BE004F05BE008B
:109AB4004F04BE000F01B10000000600889FBE00E5
:109AC4008A9FBE00010478008205780083447800F0
:109AD400E54F500058003E00C9F507000800E000BB
:109AE40001003A0018002000606E8000D00DB5001F
:109AF4000005E9000B044400880F55004E003900AE
:109B0400D3F507006380640001003A003940B300D4
:109B1400080055008981FB000318A30002003A00E5
:109B24008B007800060037000308A300030032000E
:109B34000000D1008080450001003700808045008E
:109B4400606E8000008040000004E800B46E800075
:109B5400416C8000E18F400009003200E06B80001E
:109B64000080400000024200806E8000800F52009E
:109B740003003600CE0DB500000042000002E900EB
:109B8400C06E8000800F520003003600800F540026
:109B94000A00360005003700800F5200050031002E
:109BA400706E8000800F5400070036000328A30065
:109BB40021003A00C86E8800B86E8800C06E80002C
:109BC400800F5200100031000328A3000E00320061
:109BD400726E8000C80007000202520081417800C2
:109BE4000800780019000700B16E8000C06E800084
:109BF400808F50000400310008007800CE0DB500BD
:109C040000805000B06E8800786E8800606E80001E
:109C1400A06B8800A06E8800906E88001100200060
:109C24009E00070005003A00A3000700CFFA0700D2
:109C340011002000010037008000EB0001007800D3
:109C44004F05BE004F04BE0000000600889FBE0002
:109C54008A1F7800000578008204780004047800E4
:109C64000304E00016003200E1CF51002B003A005B
:109C74000104E00008003200E1CF500027003A0060
:109C840004017800890078000A0078000C0E0200B4
:109C94000000000021003700E10F450003003200FE
:109CA4000A00780096630200000000008800780033
:109CB4000900780012670200000000001700370056
:109CC4000104E0000C003200E1CF500013003A0020
:109CD400E10F41000300320002007800C06302007B
:109CE40000000000880078000A0078007266020014
:109CF40000000000090037000401780089007800A2
:109D04000A007800CE6402000000000046660200EB
:109D1400000000000000E000FCFF32004F05780066
:109D24004F04BE0000000600080278000C00370053
:109D3400426B8000536B8000000141008181490027
:109D4400D26E8800E36E8800000006006A000700F7
:109D5400080278003E0007000500780000000600B5
:109D64006B0007000B00780000000600010078007B
:109D7400CE0DB500000041000001E900000006001E
:109D8400D26E8000E36E8000020050008380580091
:109D940000000600406B8000516B80000000400012
:109DA40081804800406B8800516B880000000600E9
:109DB400540007008040EB00909D20000000060046
:109DC400806B8000916B8000000006009C80FB008B
:109DD4001C4090004800DD0001017000AC40900080
:109DE4008180FB003C4090004800DD008101700050
:109DF40000000600800F5100818F5900000006000A
:109E04006C6B88007D6B880011C0B30040C0B30048
:109E14000000060032000700E48DA90000000600DF
:109E2400626B8000736B800000004100E080490099
:109E34002E000700A46B880000000600606B800001
:109E4400716B8000800F5600818F5E000000060059
:109E54008041EB000081EB0000000600E2C1B3008A
:109E64000440BC0040CB200000014100C0DC2000C5
:109E7400000006007FB097008FB89700F06B880051
:109E8400016C8800000006008E6DEF00810920003F
:109E9400416B88006A2DEF0000000600106F8000FF
:109EA400E70F500000000600916E8000A06B800058
:109EB400808F50000000060011C0B30000C1B30041
:109EC40000000600606E8000CE0DB50000000600A4
:109ED400B26E8000C16E8000810F51000000060048
:109EE40042782D007301200093FF3700606B8800D7
:109EF400716B88000000060081DE2000914078002C
:109F04000000060083DE2000934178000000060074
:109F1400FCFF070011C0B3000000060092022000FD
:109F2400820F5000E08F58009A003E00006001004C
:109F3400290037002B0037002D0037002F00370091
:109F44003100370033003700350037003700370061
:109F5400390037003B0037008E0037008D00370092
:109F64008C0037008B0037008A0037003800370038
:109F74003A0037003C0037003E003700400037000D
:109F840042003700440037004600370048003700DD
:109F94004A0037004C0037004E00370050003700AD
:109FA400520037005400370056003700580037007D
:109FB4005A0037005C0037005E003700600037004D
:109FC400620037006400370066003700680037001D
:109FD4006A0037006C00370020232A00BE06070001
:109FE400720037003A6F0200000000006F00370073
:109FF400D0232A00B80607006C003700466F020021
:10A004000000000069003700BC700200000000007E
:10A01400660037006E6F0200000000006300370026
:10A02400A46F02000000000060003700E47002002A
:10A03400000000005D003700147102000000000001
:10A044005A00370032710200000000005700370048
:10A054005C7102000000000054003700246F02000D
:10A064000000000051003700666E0200000000008E
:10A074004E003700E66D0200000000004B00370080
:10A08400F26D02000000000048003700026E02007A
:10A094000000000045003700166E020000000000BA
:10A0A400420037002A6E0200000000003F00370023
:10A0B4003E6E0200000000003C003700526E0200B9
:10A0C4000000000039003700BC6E020000000000F0
:10A0D40036003700C06E0200000000003300370075
:10A0E4003A720200000000003000370006720200DD
:10A0F400000000002D0037006E7202000000000016
:10A104002A003700A4720200000000002700370074
:10A114007E7102000000000024003700C2710200BA
:10A124000000000021003700A071020000000000C0
:10A134001E003700E4710200000000001B0037001D
:10A14400EC6F020000000000180037000E700200DF
:10A15400000000001500370030700200000000000D
:10A164001200370052700200000000000F00370098
:10A1740074700200000000000C00370098700200A8
:10A184000000000009003700CA6F02000000000050
:10A19400060037005E0707004200200081242A00E1
:10A1A4003B0707004A3C02000000000000000600D4
:10A1B40057070700E1C7B30022112100604079006E
:10A1C400D43B02000000000000000600889FBE008F
:10A1D4008A9FBE000040EB0018F1B7000B1121006C
:10A1E4008004EB006A0920000084FB004244DD0087
:10A1F4000B0044000908780084C0B3000305200064
:10A20400094178006000B800E23902000000000053
:10A214000884E80000F47D0000C0EB008EF0B70075
:10A224008FF0B70082112100124178000281FB00F7
:10A234000A91B90000ED210002004000966302007B
:10A2440000000000000478008A007800A0072100C4
:10A254001267020000000000080078009663020004
:10A26400000000001851EC0018F1B700E14F500055
:10A27400DDFF36000900780018F1B7004F05BE0075
:10A284004F04BE0000000600889FBE008A9FBE00E7
:10A294008C1F78008004EB00281121000C11210090
:10A2A400894578000805780018407800E24F40009E
:10A2B40027003200CA3A0200000000000000E0005B
:10A2C4001800320009407800290007001007070031
:10A2D4000C0040000008EB008ED0BF00E14F4000AE
:10A2E400030032004AB30200000000008EF0EF00C9
:10A2F4008FD0BF00E14F4000030032004AB3020098
:10A30400000000008FF0EF008306070043C0B30095
:10A314000001EB001100200060407E00604D02004F
:10A324000000000078B897000000E00005003A0043
:10A334001A407800363D0200000000000000E000F2
:10A34400030032000B4078000900070032000700C8
:10A354008904E80064044400E28F5400D0FF3A000A
:10A364004F0678004F05BE004F04BE0000000600F3
:10A37400889FBE008A9FBE008C1F780080457800AD
:10A3840018D1BF008B4F50001F0032000080FB002B
:10A39400680920000880B9000CED21000000460087
:10A3A400966302000000000080047800AA072100E0
:10A3B400880078000A00780012670200000000009C
:10A3C4000900780096630200000000000B80FB0087
:10A3D4000880B90000004600C063020000000000CD
:10A3E40080047800880078000A0078007266020011
:10A3F4000000000009007800C063020000000000B3
:10A404000B00780018F1B7004F0678004F05BE0026
:10A414004F04BE0000000600F6874700889FBE0078
:10A424008A9FBE008C9FBE008E1F78000E112100F3
:10A4340018D1BF000081FB004210DD0060007F00E6
:10A444000100200018002000EB0F5000E08F58009E
:10A4540013033E000060010015003700360037008A
:10A464001D0137007F0137009B013700A101370030
:10A47400E4013700F901370064023700D4023700E1
:10A48400E4023700F302370023060700220020000D
:10A494008000EB0060407F00AA3D02000000000045
:10A4A4009B0607003100200001307F00E0FF3700E9
:10A4B400091121004210DD000080E80060C07C002A
:10A4C400363D0200000000000000E000F602320009
:10A4D40060092100508488008D06070011002000C7
:10A4E40001B07C0091F0EF000044EB000004FD009B
:10A4F40090F0B7000004FD005C00020001000000C1
:10A504006606070086B0EF0088B0EF007A30EF00EF
:10A514007C30EF00080078000EF1B700FE0507005C
:10A5240053C0B3000001EB001100200060C07C00A8
:10A53400604D020000000000081121005E060700C3
:10A5440060407C002240020000000000E10F400057
:10A5540013003A00C40507001A3E02000000000080
:10A56400180020000000E00004003A00ED05070098
:10A574007200200002307F000004EB005C00020047
:10A5840001000000EA050700C5023400EE050700DB
:10A59400F83A020000000000EE050700A4FF3700AF
:10A5A4005C000200010000003C060700EC05070007
:10A5B4002240020000000000E50F500001003600B8
:10A5C400500020000001E800E8050700AA3D020051
:10A5D400000000003200200061962A00600921007A
:10A5E4006A0C0200000000000000E00002003A00D3
:10A5F400908488000D00370042002000A1962A00B4
:10A60400600921006A0C0200000000000000E00064
:10A6140003003A00140020009484880003003700EB
:10A6240070002000908488001E013700CC050700CC
:10A634002240020000000000000478003C060700ED
:10A644008801780004017800F1C3B30060407F0002
:10A65400224002000000000008017800800F54002E
:10A664000100360000017800B0062000800F510080
:10A6740003003600500020009084880067013700F2
:10A68400BA050700AA3D020000000000610921008C
:10A69400010040000048EB0001007800930307002C
:10A6A40060092100F00D02000000000000047800A1
:10A6B40072002000F1962A00700921006A0C020041
:10A6C400000000000000E0000D003A0070092100C5
:10A6D4003A6A02000000000091F0B7009210E20014
:10A6E40003003A00800020009084880002003700B4
:10A6F40090002000908488009F0507004CFF3700DD
:10A704008804E9005009210000004400F1C2B300AC
:10A7140090CF1000040032007009210010B2020032
:10A72400000000008EF0B700E008210000C2EB003A
:10A73400904F120014003A007C804400A2072100CC
:10A7440002004000F1C2B30090CF100003003200B9
:10A754007C004400017079000804E80060092100CD
:10A764000000440061972A000B000900315878006A
:10A77400C000B1006B0444007009210010B2020053
:10A78400000000008EF0B700500921008000440052
:10A7940060092100808F500007003200E0C2B3003E
:10A7A400914F1000040032008100E900600921008B
:10A7B400808F5000F9FF3A000104E8000000EB002C
:10A7C400A084880029282A0000004000E0807C0042
:10A7D40008007800FEC40200000000000004E0004D
:10A7E400040032009410EC00A0848800EA0F5000AA
:10A7F400F5FF3600700921003A6A020000000000EB
:10A8040091F0B7008ED0BF00E14F40000B00320042
:10A8140044B60200000000000018A3000700320044
:10A824008ED0BF000EB70200000000000000E80058
:10A83400F4B20200000000008FF0B70009112100FB
:10A84400A305070060C07C00224002000000000055
:10A854004D0507001600320010C0B30090F0B70099
:10A864002D050700E1FD2F008F80400060C07C00B3
:10A87400543D0200000000000801E90050072000D8
:10A88400800F51000200360042050700E8FE370041
:10A894005884800035050700AA3D0200000000002E
:10A8A4000004440060C2B300005C7800588488004F
:10A8B4008105070060407F00224002000000000084
:10A8C4000001E8008505070060407F00AA3D020002
:10A8D4000000000028050700180020000D112100C9
:10A8E400F2FD2F000F01410082BF9F007205070097
:10A8F40060C07E0022400200000000008004780056
:10A90400E10F400014003A00260507001A3E020039
:10A9140000000000800078000000E00004003A001D
:10A92400000507007400200004B07E0001047800D4
:10A934005C00020001000000FD040700D80134009F
:10A9440018050700F83A0200000000006605070039
:10A9540001B07E00B6FE37005C000200010000007A
:10A964004E050700E18F5400C7FE32000B11210091
:10A974006F0507008901780004017800A1C3B300C2
:10A9840060C07D0022400200000000000005780045
:10A994000084E800F00F5400130036000901E800B9
:10A9A40003050700AA3D0200000000000004EB00BC
:10A9B400CEFF37000A40780022020700D6040700C1
:10A9C400080278008801780008017800A1C0B3006B
:10A9D40060C07E00224002000000000000067800F3
:10A9E4001800200019003700F40407008FB89700FE
:10A9F40060C07E00AA3D0200000000008A00E8005A
:10AA04000040EB000FB9970080707900088654006D
:10AA14000005EB0009962A00FBFD2F008F854500F9
:10AA2400990078000B0078009E0C020000000000E2
:10AA3400D5040700DFFF32000A05E8008984E80036
:10AA4400E30F5500F6FF3A000004EB000C01E800A8
:10AA54002205070060C07E00AA3D0200000000003D
:10AA6400A2FF37009150E2000600350030002000BC
:10AA7400908488004210DD007400200004307F00C0
:10AA84006BFE3700508480000048EB006009210011
:10AA9400960207005084880090848000E80F5000DC
:10AAA40003003A00C804070001307F0060FE37004D
:10AAB400170507008E004000400020008008780041
:10AAC4009050E20002003A00500020008008780014
:10AAD4009070EF0056FE3700866A02000000000006
:10AAE400E20F5000700132000905070051002000F8
:10AAF40001307F0041040700363D020000000000E1
:10AB04006101B800B20407000A003A005C000200C8
:10AB14000100000086040700060034005204070008
:10AB2400F83A020000000000EF04070001307C0046
:10AB34003FFE370090848000E10F50000400320093
:10AB440069005000E20F5000050036002A0037006B
:10AB5400CA6A020000000000E0DF9F000400370022
:10AB64004A030700E0DF9F000004E0002B003200EE
:10AB74006FD89700E24F500008003A0072040700B3
:10AB8400363D0200000000000000E9000100200042
:10AB9400308488004184880043013700E14F50002D
:10ABA40015003A0015040700363D020000000000BD
:10ABB4000100200030848800418488005C00020089
:10ABC40001000000B5040700C90407008004070061
:10ABD40005003600240407001A3E020000000000AD
:10ABE4000000E00030013A006000200090848800FA
:10ABF4007C0407000EFE3700C50407006100200036
:10AC040001307F00E008210080C0EB0090CF1000ED
:10AC140006003A004000200090848800BC0407002D
:10AC24007200200002307F0001FE37007A30EF000E
:10AC34007C30EF008FD0BF00E14F400003003A00AA
:10AC44007EB0EF0080B0EF0003003700E107210081
:10AC540056B402000000000062040700E903070084
:10AC640023C0B3000001EB001100200060407C0011
:10AC7400604D02000000000090848000000040004D
:10AC8400C1912A00E0807800F7030700E23C02004B
:10AC94000000000090848000EC0F50000E003A0089
:10ACA40054040700E23C0200000000001A040700FC
:10ACB40021982A0060407C00E23C02000000000071
:10ACC4004C040700E23C0200000000004C040700B2
:10ACD400E23C02000000000090848000E10F50007C
:10ACE400020036001B040700EF003700A084800038
:10ACF400EB0F50000F0032000704070051992A009F
:10AD040060407F00E23C020000000000A08480005C
:10AD14000000400021302A00E08078000A04070087
:10AD2400E23C02000000000038040700E23C02009C
:10AD3400000000008ED0BF0044B6020000000000F6
:10AD44000008A30005003200F3030700419A2A001B
:10AD540060407F00E23C020000000000EE030700B8
:10AD6400D19B2A0060407F00E23C0200000000000A
:10AD740090848000E10F500005003200F0838000D1
:10AD840001848000E10F4000E08F4800060032009B
:10AD9400E1030700D19C2A0060407F00E23C0200EE
:10ADA400000000000A003700DB030700619D2A0051
:10ADB40060407F00E23C020000000000D603070070
:10ADC400F19D2A0060407F00E23C02000000000088
:10ADD400081121000A040700E23C02000000000000
:10ADE4009050E20004003200490407008100200072
:10ADF40001307C008EFD370004040700E23C0200B1
:10AE0400000000000404070089FD370060092100E8
:10AE1400608488009050E20069003200091121002A
:10AE2400BD030700319E2A0060C07C00E23C0200A2
:10AE3400000000002800370000C2B30080CF50009B
:10AE440005003A00F703070060C07C00D43B020011
:10AE54000000000020003700F0C2B30080CF500093
:10AE64000B00360060CCB30000C04000E64F500039
:10AE74000700360050CAB30000C04000E54F500040
:10AE840003003600A0C7B30080CF50000F00360087
:10AE9400E703070060C07C00D43B02000000000010
:10AEA4006FD89700D8C402000000000080407800EA
:10AEB400E2030700D43B0200000000006FD89700B3
:10AEC400ECC402000000000080407800DB030700AF
:10AED400D43B020000000000DB030700D6FF3A0069
:10AEE4008D030700D1C3B30060C07C00D43B0200D3
:10AEF40000000000081121002800370000C2B30040
:10AF040080CF500005003A00C603070060407C0073
:10AF1400D43B02000000000020003700F0C2B30060
:10AF240080CF50000B00360060CCB30000C040005E
:10AF3400E64F50000700360050CAB30000C040007E
:10AF4400E54F500003003600A0C7B30080CF500087
:10AF54000F003600B603070060407C00D43B0200BB
:10AF6400000000006FD89700D8C402000000000061
:10AF7400804078003C030700D43B0200000000003E
:10AF84006FD89700ECC402000000000080407800F5
:10AF940035030700D43B020000000000AA030700A9
:10AFA400D6FF3A00D503070060C07C00E23C0200F3
:10AFB400000000009050ED0090F0B70098FF3A00B8
:10AFC40092030700E23C0200000000009203070025
:10AFD4003B0007000000E00002003A000004780093
:10AFE400060037008ED0BF004AB302000000000004
:10AFF4008EF0EF00570307001800200052030700EB
:10B00400A83B0200000000000000E00024003A0019
:10B0140025003700081121004210DD000080E800FF
:10B0240060407C00A83B020000000000EF0F5000CD
:10B034001D0036001084800021848000B7FB0700C7
:10B044008703070018003A00AF03070001307C00B3
:10B05400F7FC37008ED0BF00E14F40000300320000
:10B064004AB30200000000008EF0EF008FD0BF0052
:10B07400E14F4000030032004AB302000000000028
:10B084008FF0EF0030030700F83A020000000000E0
:10B094009F0307000E0040000008EB000200370089
:10B0A4000800E000E2FC32004F0778004F06BE00C3
:10B0B4004F05BE004F04BE006F01B1000000060042
:10B0C4004200FA00889FBE008A9FBE006903070001
:10B0D400A83B020000000000D4838000E5838000C8
:10B0E400F2838000038480000401510085815900AB
:10B0F40001002000800F5100818F590001003600AB
:10B104000001BE008204780002004200E0804A0090
:10B11400D80207000200E000150032000A042000F3
:10B124000B112100090178008A8F540001003600B8
:10B134000A0178008ED0BF0073FB2F008380470084
:10B14400E0B30200000000000F03070036003200E5
:10B154001A03070073FB2F008380470060C07D0043
:10B164004A3C02000000000088845400EDFF3A00CD
:10B174005F030700F083800001848000800F51008A
:10B18400818F59002A003A00BD020700A100200067
:10B19400013079008630EF008830EF008ED0BF0098
:10B1A4008000EB005CB3020000000000E8C7B300BD
:10B1B4008ED0BF0061FB2F008F8040005CB3020083
:10B1C400000000000000E000040032008F020700CD
:10B1D400EF70970088CF5000F5FF3A008B0207000C
:10B1E4008FD0BF002108210056B4020000000000E7
:10B1F4008FD0BF00E107210056B402000000000018
:10B20400E10207000A003A007EB0EF0080B0EF00D0
:10B214008FD0BF004AB30200000000008FF0EF009F
:10B2240008007800030037001000200001003700F8
:10B234000000EB004F05BE004F04BE000080FA0082
:10B24400000006000004E00002003A004C00070081
:10B2540007003700E14F500002003A0005000700E4
:10B2640003003700E24F500001003A008400070059
:10B27400000006002800FA00889FBE008A1F78009C
:10B284009150E2003A0035005E020700620020009F
:10B294008000EB0060407C00AA3D0200000000003A
:10B2A4007A02070060407C00A63E02000000000015
:10B2B4006300400000047800C80FB2004002200080
:10B2C400800F540001003600000478000800E000FC
:10B2D40003003A0029FD2F008F8444001300370037
:10B2E40029FD2F008F8444000A1121008A020700DF
:10B2F400420020008900780060407D00AA3D0200E1
:10B304000000000033002000090178004100200003
:10B3140009007800A8C3020000000000640454007F
:10B32400E38444000800E000F0FF3A00804CEB00A6
:10B3340020FD2F000F004000A2C3B300E680570099
:10B34400904F1100030032000000E800808F50008D
:10B35400FBFF3A000058EB008000780020FD2F002E
:10B364000F004000626A02000000000091F0B70084
:10B374004F0578004F04BE000080FA00000006006C
:10B38400889FBE008A9FBE00091121003F0207006A
:10B3940060C07C00A63E02000000000000047800AB
:10B3A400C01021005184800001005000800F54001F
:10B3B4002E003900770207002E00370037020700FD
:10B3C400B1C3B3002011210065407800224002007F
:10B3D40000000000800478005A848000080178008E
:10B3E400800F540001003600000178000B11210089
:10B3F400490207008A00780060C07D00AA3D02006F
:10B40400000000000000450061C2B300015878004C
:10B4140050848800890F54000E003600640207002F
:10B42400543D0200000000000B04780003003700C4
:10B4340022020700543D020000000000A40207009D
:10B4440060407C0022400200000000000000E00098
:10B45400F7FF32001C020700A63E020000000000B5
:10B464004902070003003200D4FF37000800E0005F
:10B47400D2FF3A004F05BE004F04BE000000060094
:10B484000A00FA0010020700A63E020000000000B5
:10B4940080007800E90F50000500360020002000ED
:10B4A400908488007A30EF007C30EF000D00370084
:10B4B4009702070001017800EA8057007402070030
:10B4C400AA3D0200000000008040EB006A0050002A
:10B4D40001F07F006A8057001A0E0200000000008D
:10B4E400E40107000080FA00000006000200FA00F0
:10B4F400889FBE008A1F780000047800F00D0200C7
:10B5040000000000800178000000E0002800320004
:10B51400080578000801780002047800B840780033
:10B524008304E900D0C3B30080CF5000030032008D
:10B534007740500080CF500002003A00005DEB00DD
:10B5440017003700B0C2B30080CF500003003A00A8
:10B554006B405000005D78001100370050C2B3000A
:10B5640080CF50000D003A00E18F540011003600E6
:10B574001844780098FF9F002240900080FF9F00AD
:10B5840063044100E38451004FB8970090C4020063
:10B5940000000000005D780001003700015D7800C4
:10B5A4000900E000030032000801BE00DAFF3700A2
:10B5B400080578008040EB00015D78000A007800FF
:10B5C400014D78004F0578004F04BE000080FA005A
:10B5D40000000600889FBE008A1F780000047800DF
:10B5E400010578001004E00018003200880078009B
:10B5F4000A0078009E0C0200000000000000E00039
:10B6040006003A000A007800F00D02000000000075
:10B61400000044000000E8000D0037000800780036
:10B62400F00D020000000000000044000004E800E7
:10B6340008007800F00D0200000000000000440043
:10B644000004E8001804E000E8FF3A000000EB0002
:10B654004F0578004F04BE0000000600889FBE001E
:10B66400000478000101780080007800D0C3B300A2
:10B674002F000700800478000800E0000400320076
:10B684001804E000020032000800780097FF070069
:10B69400090078004F04BE0000000600889FBE0029
:10B6A4008A9FBE008C1F7800000578000106780090
:10B6B400010178008000780060C2B3001C0007001C
:10B6C40080057800E20F50000E003A00D883800015
:10B6D400E9838000E7010700363D02000000000016
:10B6E40001002000800F5400818F5C0005003A00A7
:10B6F4000C0178008A0078000040EB000C00070081
:10B70400800578000A00E000040032001A04E0001A
:10B71400020032000A00780074FF07000B00780072
:10B724004F0678004F05BE004F04BE00000006001F
:10B73400889FBE008A9FBE008C9FBE008E1F78002B
:10B744000047780081067800020678000004E000D3
:10B7540008003200510107008040780020112100C8
:10B764006540780022400200000000008005780057
:10B7740004003700BF010700363D0200000000004E
:10B78400800578002A002000E18F4500390032004E
:10B79400E10F560008003E000D00E00008003200F2
:10B7A4001F010700AA3D0200000000001F0107005E
:10B7B4001A002000260037000D00E00006003A00C1
:10B7C40017010700AA3D020000000000170107004E
:10B7D4000005EB001E0037000C81E900828F550044
:10B7E40012003600160107008D00780060407D00CD
:10B7F400AA3D0200000000000C0107000C81550066
:10B804000281E800B501070060407D00AA3D020006
:10B8140000000000050107008C8046000040EB009A
:10B82400E0F89F001A0020000900370032010700E9
:10B834008D00780096010700AA3D02000000000078
:10B84400FA0007000040EB0080F57E000005EB00E5
:10B854000E04E000070032008A0107008000EB00BC
:10B864002211210060407900543D020000000000D4
:10B87400EE0007000A0078004F0778004F06BE006C
:10B884004F05BE004F04BE00000006001000FA0081
:10B89400889FBE008A1F780090848000EA0F5000C1
:10B8A40058003200EB0F50003F003200E90F500007
:10B8B40084003A0008112100120107004200200010
:10B8C400019F2A0060407C00A63E020000000000A8
:10B8D40080007800E10F4000290032000E010700CB
:10B8E400010178008000EB0060407C00AA3D02006A
:10B8F40000000000D6000700DB000700363D020010
:10B9040000000000E90F50006E003600020107003D
:10B91400A2002000F680570060407C00AA3D02008F
:10B9240000000000CA000700A2002000519F2A0066
:10B93400768057006A0C0200000000000000E0005E
:10B944000B003A00A00020009084880026B5020075
:10B95400000000008EF0B70062002000F280570063
:10B9640066B50200000000002000200056003700E9
:10B97400B00020009084880020002000520037008E
:10B984009E000700363D02000000000064015000E4
:10B99400CA000700AA3D020000000000AC00070036
:10B9A4001000200048003700A500070060407D001B
:10B9B400363D0200000000009C000700D60007008E
:10B9C40060407D001C3D020000000000C0F92F0013
:10B9D400F1FF2F0046010700020040008380480069
:10B9E400C2F92F00F3FF2700820F5000838F580005
:10B9F40034003600F400070001307D000000EB0045
:10BA0400310037001B010700363D02000000000032
:10BA1400000478003601070001002000820F500066
:10BA2400838F580001003600020478000800E0000B
:10BA3400170032000A11210008017800F00F5400A9
:10BA44000100360002012000B3000700F680570011
:10BA540060407D00AA3D0200000000000001780063
:10BA6400D0838000E183800002005000E080580011
:10BA740080000700020454008ED0BF00F6805700F7
:10BA840066B50200000000000800E000EAFF3A008A
:10BA9400D0838000E1838000E00F5000E08F5800E5
:10BAA40008003A0010002000CAB50200000000009F
:10BAB4007300070071002000013079000000EB00E2
:10BAC40001003700100020004F0578004F04BE002D
:10BAD4000080FA00000006004000FA00889FBE00C3
:10BAE4008A9FBE008C1F780000017800DC000700EC
:10BAF40010003A000200780010B2020000000000BA
:10BB040000457800E14F4000370032000EB70200D4
:10BB14000000000030848800110037000A407800DB
:10BB24004AB30200000000008630EF008830EF00C6
:10BB34002D00370030848000F4B2020000000000C1
:10BB440000457800E14F4000270032004284800025
:10BB5400030020002100200068B40200000000005F
:10BB6400C4000700A83B0200000000008004780025
:10BB74000000E000150032000B0420000C1121002D
:10BB8400090178008B8F5400010036000B01780006
:10BB940061FB2F008F8040000A407800E0B3020070
:10BBA4000000000078000700DCFF3200830007007B
:10BBB40061FB2F008F80400060407E004A3C020001
:10BBC4000000000088845400EDFF3A000A40780029
:10BBD400F8B6020000000000408488000A407800A3
:10BBE4004AB30200000000004F0678004F05BE0073
:10BBF4004F04BE000080FA00000006000811210076
:10BC0400190037000811210043003700D083800059
:10BC1400E183800061004000E080480015003700A7
:10BC2400350007008000EB00990037000004540041
:10BC3400E0845C00D8838800E98388000000060063
:10BC4400D8838000E98380000A1121003200370084
:10BC5400A700070000015100E0815900D283880049
:10BC6400E3838800000006002B00070060407C008E
:10BC740000000600D0838800E183880000000600ED
:10BC8400A300070002112100000006001D000700A8
:10BC940022002000D1242A00000006008511210082
:10BCA400954278008582FB00C22ADD000002EB0089
:10BCB4008401780004017800000006008700070072
:10BCC40060407C00000006008611210016437800C5
:10BCD4000683FB004233DD008002EB00050278009E
:10BCE4008501780022002000D1242A00201121009F
:10BCF4006640780000000600620007000B0178002F
:10BD040000000600040007008002EB000502780032
:10BD140085017800000006007D0007000080E8002F
:10BD2400000006005000200090848800780037004E
:10BD34001284800023848000020050008380580015
:10BD44004240A90000000600F3FF070060407F00A6
:10BD5400000006006400070001307F0000000600B8
:10BD64005B00070060407F000000060055000700EC
:10BD740060407F00000006006500070021002000ED
:10BD840001307F0000000600000478000000E0009D
:10BD940000000600E3FF07007100200001B07C00F2
:10BDA40000000600DCFF070060C07E000000060003
:10BDB4004A00070060C07D0000000600D6FF0700AF
:10BDC400080178000000060051000700710005001A
:10BDD4003084800041848000800F5100818F59009D
:10BDE400000006004A0007007400200004307F00B1
:10BDF400000006003300070060407C0000000600DD
:10BE04003E00070060407C00000006003B00070085
:10BE140060407F00000006003B00070001307F0007
:10BE240000000600BCFF0700B1C2B300000006001A
:10BE3400B9FF070051C2B30000000600B6FF0700B7
:10BE440060C07C000000060060848000B040780080
:10BE5400A1DF9F00608488000104E0000000060068
:10BE64003084800041848000E00F5000E08F58004F
:10BE740000000600260007002111210060C07800A0
:10BE840000000600D8838000E9838000200037008A
:10BE94002311210060C0790000000600229D2400C7
:10BEA400B30620000001410081814900128488000A
:10BEB400238488000000060019000700A1C0B30015
:10BEC4000000060094FF070061092100000006003D
:10BED4001300070001C2B300000006008EFF070034
:10BEE4008000EB000000060009000700B100050017
:10BEF400D2838000E38380000000060086FF0700F1
:10BF0400D1242A000000060001000700910005006A
:10BF140018D1BF000080FB004200DD0000000600D5
:10BF24000300070084017800040178000000060083
:10BF340079FF07000002EB00000006000200FA008F
:10BF4400889FBE00CD22A800C922A9008000EB0072
:10BF540001128800F00020001012880021128800CD
:10BF64004302A80042A2A80041E2A800F10307008E
:10BF7400D1C1B3006680570002040700AFF89700F0
:10BF84000180FB000038A300F8FF3A000080EA00BB
:10BF9400E1046000F5FF3A001800200038BA880078
:10BFA40019BA88008940780080C0B30043040700B0
:10BFB4008940780090C0B3004004070011CAB30060
:10BFC400C0C0B3003D04070091C0B300D0C0B300AB
:10BFD4003A04070011CAB300A0C0B3003704070035
:10BFE40091C0B300B0C0B3003404070021CAB30049
:10BFF40040C0B3003104070091C0B30050C0B30087
:10C004002E04070021CAB30020C0B3002B0407008C
:10C0140091C0B30030C0B300280407000940780081
:10C02400700307000020200076040700D1C0B3008D
:10C03400094078002104070021C3B30020C0B300E5
:10C044001E04070021C1B30040C0B3001B04070055
:10C0540001C4B30030C0B30018040700F1C3B30037
:10C0640090C0B3001504070021C1B30060C0B30041
:10C0740012040700C1C0B30070C0B3000F0407006E
:10C08400E1CEB300A0C0B3000C04070051C0B3005C
:10C09400B0C0B30009040700403020005904070071
:10C0A400F18220009140780040C0B30003040700EF
:10C0B400018320009140780050C0B300FF030700C3
:10C0C400118320009140780020C0B300FB030700D7
:10C0D400218320009140780030C0B300F7030700AB
:10C0E400318320009140780009407800F303070071
:10C0F400418320009140780008407800EF03070056
:10C104008940780050C1B300EC03070021C1B3009B
:10C11400658057009B0307003FF8970048F7B70076
:10C124000110200000C1B3001A04070021472300B6
:10C1340040C1B30017040700890078000940780063
:10C1440014040700090078002E04070041C0B3005E
:10C15400F0C1B300FE0307004F04BE000080FA00E4
:10C16400000006000200FA0011C0B3000F80E900CD
:10C17400A60307007FB897004200DE00610060005C
:10C184000080FA00000006000200FA00F1C1B300CA
:10C194000F80E9007B030700EFF897000180FB00A4
:10C1A4004300DE000000A200610060000080FA008D
:10C1B40000000600881F78004617E20010003A00CD
:10C1C4001000200030BA880018BA80000804E90082
:10C1D40061040700010036000004780001C4B300C4
:10C1E400E0C1B300DA03070088407800C0C0B300A0
:10C1F400B2030700C840DE00D0C0B300AF0307009D
:10C204004F047800000006000600FA00889FBE0074
:10C214008A9FBE0090112000FA0307000AF02F0045
:10C22400FB0F200091C1B3006E8057005503070037
:10C234002FF49700E0002000F2030700E1C0B300F0
:10C244006D8057004F0307003FF097000080FB000C
:10C254008A84640080847400F1C0B3006C80570049
:10C26400480307004FF097004800DD008B8464000A
:10C274008084740090112000E203070091C1B30090
:10C284006B8057003F0307005FF09700804F540016
:10C29400E4FF3A00C0002000DA030700C1C0B30085
:10C2A4006A805700370307006FF097000080FB0097
:10C2B4000A04640000047400D1C0B300698057000C
:10C2C400300307007FF097004800DD000B04640092
:10C2D40000007400808F54000400360080805400F5
:10C2E400109A20000101500005003700129A200026
:10C2F400808F540002003200090050000001E90060
:10C30400020078004F05BE004F04BE000080FA0012
:10C31400000006001600FA00889FBE008A1F7800FD
:10C32400800478000105780090112000B50307000F
:10C3340091C1B30068805700120307000FFC9700F7
:10C344000000EB00AF0307000000EB000804E0006E
:10C354003A0032004617E20003003A0095FF070056
:10C364000000EB003500370010BA800020BA8800C6
:10C3740041742100914078000040EB004F03070016
:10C38400517421009140780010C0B3004B030700A2
:10C39400410120007C805700510207003FB89700FC
:10C3A4004EC5020000000000B0BF9F002FB19700EF
:10C3B400109A2000800F51000D003E00CFE097003E
:10C3C40061C060000A003A00CFB197000001280064
:10C3D4000080610006003A00BFB09700E05E2000D4
:10C3E400808F500002003E000378A30001003A0051
:10C3F4000000FE0012BA8800708057000500090092
:10C40400B05C78006900B1006000B10000CDEB00C1
:10C414007FF09700E84F500006003A006FF0970055
:10C424000004E00002003200E64F500001003A0030
:10C43400004D78004637EF00100020004F057800CB
:10C444004F04BE000080FA00000006000200FA005B
:10C45400889FBE000004780081447800D2BF9F000A
:10C4640031CAB30020C0B3001403070091C0B30065
:10C4740030C0B30011030700009B2000DFB8970011
:10C4840080804000D1BF9F00AFF8970060C0B30028
:10C494000A030700BFF8970070C0B3000703070042
:10C4A40061002000080078005D02070061002000A0
:10C4B400F08220005A02070080C0B300490207003E
:10C4C40060C0B3000904E00001003A0009407800AC
:10C4D400440207004F04BE000080FA00000006007A
:10C4E4001000FA00889FBE008A9FBE008C9FBE0089
:10C4F400AA03070016030700A803070003030700A5
:10C50400A1C0B300C0C1B30000030700A603070025
:10C514000F03070048D7BF0065405000E14F5000AB
:10C524006F003E000004EB00893E2000C1C1B3004F
:10C5340074805700930207004FE897006A00600078
:10C5440003003A000804E800890F5400F7FF3A009A
:10C55400C1C1B300738057008A0207005FE89700E7
:10C564000018A30003003A00703E2000800F54001E
:10C574005B0036008C030700E40207008040EB00F8
:10C58400728057007F0207006FE897000080FB006D
:10C5940009F02F00090565000005750011C0B300FE
:10C5A4007180570077020700FFEE97004868DD00AE
:10C5B400F80F2000080565000005750061C0B30090
:10C5C400708057006F0207000FF097000080FB0097
:10C5D400898464008084740071C0B3006F80570044
:10C5E400680207001FF097004800DD00888464009B
:10C5F400808474000904E800884578008840780045
:10C604000040EB00AD0207004844DE008844780097
:10C614008840780010C0B300A80207007C86570049
:10C62400810020000C007800AD0107000044EB00FD
:10C63400C1C1B3006E805700520207002FF097006B
:10C644000018A300200032003FB0970000D8A300D8
:10C654001D00320051030700BD0207004F0307000D
:10C66400AA020700A1C0B300C0C1B300A70207001B
:10C674004D030700B6020700C1C1B3006D80570027
:10C68400400207003FF097006A006000FAFF3200A2
:10C69400450307009D0207008B4078000040EB0033
:10C6A400860207008940780010C0B30083020700A7
:10C6B400810020000C007800890107000844E8008C
:10C6C400F04F5400DAFF3A008A4078000040EB0053
:10C6D4007A0207008D40780010C0B300770207008B
:10C6E4004F06BE004F05BE004F04BE000080FA0096
:10C6F40000000600881F78000903070002003600C6
:10C7040020672F0000844000884078000040EB0040
:10C714006A020700C840DE0010C0B30067020700C9
:10C724004F047800000006000400FA00881F780017
:10C73400668157000019780021C0B3000200780018
:10C7440010020700FA02070031C0B30063805700EB
:10C754000C0207001703070020C0B30057020700AC
:10C76400BFF8970030C0B3005402070008007800F7
:10C774004F0478000080FA00000006000400FA006C
:10C78400881F780066815700001978008040EB000C
:10C7940002007800FB010700E502070011C0B300A6
:10C7A40063805700F7010700020307000040EB0015
:10C7B40042020700BFF8970010C0B3003F02070011
:10C7C400080078004F0478000080FA00000006009A
:10C7D4000200FA00889FBE008A9FBE00810578008F
:10C7E400CF0207000200360020672F0000844000BB
:10C7F4008040EB006A805700E20107006A8057001E
:10C804003081FB0001F02F00010565000205750071
:10C8140011C0B300DB010700FFF497004848DD00B6
:10C824000A85FB0000057500884078000040EB0095
:10C8340022020700C840DE0010C0B3001F02070038
:10C844000B0078000C000700000478008A40780090
:10C854000040EB00190207008940780010C0B300C3
:10C8640016020700080078004F05BE004F04BE0002
:10C874000080FA0000000600FA874700889FBE0087
:10C884008A9FBE008C9FBE008E1F780080057800B2
:10C894006044B8008040EB0070805700B901070085
:10C8A4000FF09700D9020700010666000006760023
:10C8B40011C0B3006F805700B20107001FF7970043
:10C8C4004870DD000C86FB00000676000B00E000DB
:10C8D40020003200C0FD2F00808647008B007800C6
:10C8E400F48F55000100360041012000D1AF9F00B4
:10C8F4000D007800FA000700DFA897008185550035
:10C9040061806000050032000040EB0080F07E0092
:10C914005FA997000201E800D2AF9F00DFA897004B
:10C924000100E00009003200C0FD2F000081470033
:10C934003200780000044400E0844C000180E900E7
:10C9440080007800FAFF3A00D0AF9F000B00E000AF
:10C95400E2FF3A008C4078000040EB00D70107006A
:10C964008E40780010C0B300D40107006148B800BD
:10C9740008044000E0844800090044000080EA0004
:10C984004F0778004F06BE004F05BE004F04BE009F
:10C99400AF01B100000006001000FA00889FBE003D
:10C9A4008A9FBE008C9FBE00A0B79F00B1B79F00B6
:10C9B400C2B79F008005EB000B057800E10F400033
:10C9C400020032000B0678000C00370021C0B300CF
:10C9D400768057006B0107002FE897000080FB006A
:10C9E400A0B79F0031C0B3007580570065010700F0
:10C9F4003FE89700D0E79F001C0020008006EB0072
:10CA04003FB09700E10F40000C003A008040EB007B
:10CA1400748057005B0107004FE897000080FB001B
:10CA2400B0B79F0011C0B3007380570055010700D1
:10CA34005FE89700F0E79F001D002000CFB4970047
:10CA4400E18F540045003E000D00E0000E003A0066
:10CA54008D407800728057004A0107006FE8970004
:10CA64006A020700818565008085750011C0B300E6
:10CA740071805700430107007FE897004800DD00FC
:10CA84008B85FB00808575000C00E0000E003A00E9
:10CA940021C0B300708057003A0107000FF09700DF
:10CAA4005A020700010565000005750031C0B30096
:10CAB4006F805700330107001FF097004800DD0026
:10CAC4000A85FB0000057500EFE097000040EB00CD
:10CAD4007A010700FFE0970010C0B3007701070058
:10CAE400CFE0970020C0B30074010700DFE0970097
:10CAF40030C0B300710107000900E00006003200F5
:10CB04000004EB006B000700B60007000804E8000F
:10CB1400888F5400FBFF3A000D00E00006003A0045
:10CB24008B4078000D40780064010700C858DE008F
:10CB340010C0B300610107000C00E0004D003A0092
:10CB44008A40780020C0B3005C010700C850DE00B2
:10CB540030C0B30059010700460037000C00E00064
:10CB6400080032002FB09700008544008A40780006
:10CB740020C0B30051010700C850DE0030C0B3002C
:10CB84004E0107003FB49700088544008A04E90079
:10CB9400C9B79F00F1C1B3006E805700F9000700C8
:10CBA4002FF097000058A300FAFF3A00EFE0970037
:10CBB40000C1B30041010700FFE0970010C1B300BA
:10CBC4003E010700CFE0970040C1B3003B010700DE
:10CBD400DFE0970050C1B30038010700DE01070011
:10CBE40005003E00808F540003003600D0652F00FE
:10CBF40000004500C0B79F00788557009A40780030
:10CC040020C1B3002D010700F78457009940780034
:10CC140030C1B3002901070001C1B300F0C1B30062
:10CC24003A01070001C2B300F0C1B3004801070094
:10CC34000D00E0000F0032004FB197008200E800C1
:10CC4400C1B79F00C401070004003E00808F50005C
:10CC54000200360000005100C0B79F009A407800DF
:10CC64000040EB00150107009940780010C0B300A4
:10CC7400120107004F06BE004F05BE004F04BE0060
:10CC84000080FA00000006000200FA00F1C1B300BF
:10CC94000F80E900BB000700EFF897000180FB005C
:10CCA4004500DE000000A200610060000080FA0080
:10CCB40000000600AB01070000A02300401288001A
:10CCC400C2010700FEFF3A00C3010700FCFF320067
:10CCD400C4010700CD22A8000080FB00000006006C
:10CCE4000200FA0080017800CD22A900A0032000F0
:10CCF400401288000300E000010032008301E900D3
:10CD0400B2010700FEFF3A00B3010700FCFF320046
:10CD1400B70107000002EB00E18F5000130036005A
:10CD2400910107006022B800451288000482E800DF
:10CD3400A6010700FEFF3A00A7010700FCFF32002E
:10CD4400421280000300E000040032004810DE00BC
:10CD5400904198008381E800824978000480500063
:10CD6400E10F5000F0FF3E00A4010700848F500043
:10CD7400180036000001EB008002EB0084805000B4
:10CD8400451288000300E000080032008301E80037
:10CD94008E010700FEFF3A008F010700FCFF3200FE
:10CDA40040128000804978000600370087010700A0
:10CDB400FEFF3A0088010700FCFF32008C010700E7
:10CDC4008001EB000201E800828F5000ECFF3A0082
:10CDD40002024200CD22A800040078000080FA007C
:10CDE400000006000200FA005E0107000080FB005C
:10CDF40001A02700010070004012880073010700A1
:10CE0400FEFF3A0074010700FCFF320075010700C1
:10CE1400E0FF9F00CD22A8000080FA000000060079
:10CE24000200FA008001780001027800CD22A900F6
:10CE3400A00720004012880064010700FEFF3A00AA
:10CE440065010700FCFF320069010700E10F520091
:10CE5400280036001380FB004800DD000281FB003F
:10CE64000001710013409000680107000101610096
:10CE7400000171008381E8003B0107004212880031
:10CE84000482E900E10F520014003600F10F200083
:10CE940005F02F001380FB004800DD000101610054
:10CEA40000017100134090000080FB000501610047
:10CEB400000171008381E80044010700FEFF3A008D
:10CEC40045010700FCFF32004901070042128800B7
:10CED4000482E900E10F5200EEFF3E003B0107002F
:10CEE400FEFF3A003C010700FCFF3200400107004E
:10CEF400420107000400E0000B0032000301780047
:10CF0400848041003280FB00401288002F0107001A
:10CF1400FEFF3A0030010700FCFF32003401070035
:10CF2400810F5100F7FF3A00CD22A8000080FA00DB
:10CF3400000006000200FA0001C2B300E0C1B30021
:10CF44007200070010002000B0020200010000007F
:10CF5400CD22A900F00F2000401288001B01070019
:10CF6400FEFF3A001C010700FCFF3200020107002B
:10CF740010002000B0020200010000000080FA004E
:10CF8400000006000001070010010700FEFF3A0040
:10CF940011010700FCFF3200401280004822EF001C
:10CFA4000A010700FEFF3A000B010700FCFF3200F4
:10CFB40040128000CD22A8000049780002007800C9
:10CFC40000000600F000070000010700FEFF3A0021
:10CFD40001010700FCFF3200401280004822EF00EC
:10CFE400FA000700FEFF3A00FB000700FCFF3200D6
:10CFF400401280004822EF00F4000700FEFF3A00D0
:10D00400F5000700FCFF3200E9FF37000400FA00D6
:10D01400889FBE00800478000144780040212000ED
:10D02400780007008840780040C1B300230007005F
:10D0340011C0B30020C1B30020000700A0302000BD
:10D0440070000700A1C0B30068805700DDFF07002F
:10D054000FF8970061446000FAFF3A004021200075
:10D06400680007008840780020C1B300130007005F
:10D0740081C1B30067805700D2FF07001FF89700F3
:10D08400AC00070091C1B30066805700CDFF0700D4
:10D094002FF897004800DD000884FB0000047400AA
:10D0A4000000EB0057000700880C780009007800A6
:10D0B4004F04BE000080FA00000006000200FA00DF
:10D0C400CD22A9000064A0000080FB00401288006B
:10D0D400BE000700FEFF3A00BF000700FCFF32005D
:10D0E40098000700B9000700FEFF3A00BA000700E5
:10D0F400FCFF3200BE00070000000000000000003A
:10D10400CD22A8000080FA00000006000200FA0008
:10D11400CD22A9000080FB00000AB3004012880061
:10D12400AA000700FEFF3A00AB000700FCFF320034
:10D1340084000700A5000700FEFF3A00A6000700D0
:10D14400FCFF32008C0007000080FA00000006009B
:10D154000200FA00CD22A9000074A0000080FB00A8
:10D164004012880099000700FEFF3A009A00070069
:10D17400FCFF32007300070094000700FEFF3A0032
:10D1840095000700FCFF32007B0007000080FA00D6
:10D19400000006000400FA00881F780000447800AC
:10D1A400D1BF9F004021200016000700884078006E
:10D1B40040C1B300C1FF0700AFF8970060C1B300DE
:10D1C400BEFF0700BFF8970070C1B300BBFF0700A4
:10D1D400A03020000B000700A1C0B30064805700FA
:10D1E40078FF07004FF897000008A300FAFF3A0001
:10D1F4000000EB00030007004F0478000080FA00F1
:10D20400000006000200FA00F0BF9F0031C0B30026
:10D21400F0C1B300BDFF0700FFF89700F0C1B300F1
:10D22400CBFF07000080FA00000006000200FA00AD
:10D2340041C0B300F0C1B300B4FF0700D1C1B300D3
:10D244000F80E9004FFF0700EFF8970064C060000B
:10D25400FAFF3A00F1C1B3000F00E90049FF0700EB
:10D264007FF897000038A300FAFF3A0001C2B30028
:10D27400E0C1B300B6FF07000080FA00000006001A
:10D284000200FA0001C2B300E0C1B3009FFF07002F
:10D29400D1C1B3000F80E9003AFF0700EFF897000F
:10D2A40061C06000FAFF320041C0B300F0C1B300B6
:10D2B400A7FF07000080FA0000000600881F78001E
:10D2C4000044780050312000CEFF070088407800E9
:10D2D40050C1B30079FF07000000EB00C9FF07004D
:10D2E4004F047800000006000200FA00881F78004E
:10D2F40050312000C3FF070051C1B30064805700C0
:10D3040020FF07004FFC97000000EB00BDFF070063
:10D314000880FB004F0478000080FA00000006003B
:10D3240021BA800081004000748440000A00370064
:10D334000FF897003500070001046400000474002E
:10D344000000060040128000A0FF9F000180FB0047
:10D354004012880000000600109A2000800F54003C
:10D3640000000600CD22A90041E2A9004342A80022
:10D3740041E2A8000000060040128000A0FF9F00C8
:10D38400CD22A8000000060000017800CD22A900EB
:10D394008180FB00411288000000060001C8B30030
:10D3A400F0C1B3000000060081C0B300F0C1B300B7
:10D3B400000006001FF897004800DD000884FB0009
:10D3C40000047400EFF097000000060040C2BF00A4
:10D3D4000018A3000000060040C2BF000008A3001C
:10D3E400000006000500070040128000000006004F
:10D3F40040128000A0FF9F000000060041E2A90047
:10D404004342A90041E2A800000006000080FB009E
:10D4140001F02F0000000600A0838800810C20008A
:10D4240080804000B1838800C0838800000006002B
:10D4340022FE2000A1FD2000E0062100DEFE020005
:10D4440000000000A0FD200000000600000006000F
:10D454000000EB007257E200020032007277EF0026
:10D46400100020000000060020FE2000000006003E
:10D47400881F78000004780072002000C1252B006A
:10D484006A0C0200000000000000E0000800320006
:10D494004200200041262B00080078006A0C02009C
:10D4A40000000000010820000000E00001003A0034
:10D4B4008000EB00010078004F04780000000600B3
:10D4C400881F78000104780091262B009E0C02002E
:10D4D400000000000000E00007003A00F1262B00E5
:10D4E400080078009E0C02000000000001082000E3
:10D4F4000000E000010032008000EB000100780031
:10D504004F04780000000600889FBE0091272B007E
:10D5140060092100EC5A0200000000008004780039
:10D524000000E00017003200C0C3B300994F1000A0
:10D5340014003A000004EB00E8C07C00E00621007F
:10D54400EAFE0200000000000000E00006003200D5
:10D55400E20F5000060032000804E800FE0F5400F9
:10D5640008003200F4FF370072F7B70005003700F7
:10D5740010C0B30072F7B700E0062100E8FE020015
:10D58400000000000000EB004F04BE000000060095
:10D594001400FA008ED0BF0042012000F48057002E
:10D5A400C6B60200000000009200200011282B00E3
:10D5B400748057006A0C0200000000000000E000C4
:10D5C40003003A00400120000000E900FEFF3A0099
:10D5D40022012000E1282B00748057006A0C02000D
:10D5E400000000008000EB000000E00002003A00B0
:10D5F4000400070080007800010078000080FA0031
:10D60400000006005600FA00889FBE008A9FBE00F4
:10D614008C1F7800D8838000E98380000B112100DF
:10D624002D040700363D02000000000000057800CC
:10D63400290407001A3E0200000000000000450013
:10D6440001002000800F5400818F5C00FC003E002C
:10D6540021040700363D0200000000006101B8000B
:10D6640014002000D0838000E1838000800F5100EB
:10D67400818F5900FB0039003303200002FA2F0088
:10D684000F01410060002000010020008EEC020028
:10D69400000000006FA097000060A100E0A79F00B9
:10D6A4004CFD2F000C864700A700370061002000C6
:10D6B40060092100305B0200000000000000E0006F
:10D6C400DF003A0001072000C0092100505B02007E
:10D6D400000000000000E000D9003A0068092100C1
:10D6E400112C2B00080078009E0C020000000000A2
:10D6F4000000E0000C003A0001FA2F008F80400087
:10D70400C0092100F4C20200000000000000E00093
:10D71400CB0032000F9097009F909700A09F9F002E
:10D72400B19F9F0088003700412C2B00080078002F
:10D734009E0C0200000000000000E00002003A001D
:10D7440080FA2F0021003700712C2B00080078008C
:10D754009E0C0200000000000000E0000C003A00F3
:10D7640040FA2F0080804700C0092100F4C2020063
:10D77400000000000000E000B10032002F9097008C
:10D78400BF909700C09F9F00D19F9F006E003700FD
:10D79400B12C2B00080078009E0C02000000000051
:10D7A4000000E00002003A00C0FA2F000700370032
:10D7B400012D2B00080078009E0C020000000000E0
:10D7C4000000E00008003A0000FB2F0080804700C2
:10D7D400C0092100F4C20200000000000000E000C3
:10D7E40059003A0096003700512D2B0008007800AC
:10D7F4009E0C0200000000000000E00035003A002A
:10D80400C40921000041780005CDB300F6CBB30074
:10D81400F7C9B300A3072100010037000402E800A0
:10D82400944078000104E0000A00320005C0400082
:10D83400E94F50000F00360006C04000E54F50008D
:10D844000C00360007C04000E54F5000F3FF3E00D7
:10D85400080037000280FB007C00400001C3B300D5
:10D8640001F079000241E800EB4F510008003E004E
:10D87400F8FF37000280FB007C00400001F07900D3
:10D884000402E8000241E800EB4F5100E4FF3600D7
:10D8940068092100DBFC2F008B8547000C0578000C
:10D8A400290A210098407800D1D79F0018409000A1
:10D8B400004D78001A00780090C4020000000000B7
:10D8C400805D78000884E800888F54001E003200D0
:10D8D400F4FF3700912D2B00080078009E0C020005
:10D8E400000000000000E0000B003A00C009210025
:10D8F400DEC502000000000001FA2F008F80400006
:10D904007C804000C10921000F00090031587800D3
:10D914000001B1000C003700E12D2B000800780055
:10D924009E0C0200000000000000E00006003A0027
:10D9340010C3B3009C50E30003003A006FA09700AB
:10D944000060A000E0A79F00D0838000E1838000F6
:10D95400E00F5000E08F580054FF3A0000FA2F0007
:10D964000F0040003CE00200000000004FC8970098
:10D974000068A300090032005A03070001FA2F00CF
:10D984008F8040007C804000A10A21000F00090024
:10D99400B05878000001B1001D00370068FD2F0069
:10D9A40008844700102A2B001F000900305C78000F
:10D9B4000802B1007F7097000080FB00801F780090
:10D9C4004F7097000080FB00801F78001F70970045
:10D9D4000080FB00801F78006F6897000080FB00C8
:10D9E400801F7800812F2B00811F780008007800A9
:10D9F400840D0200000000003A030700A00A210081
:10DA04000F000900385878000801B100EA87570070
:10DA1400BA70EF00A00A210002C2B3008041EB00FB
:10DA2400A10B2100904F110001003A000348780037
:10DA34000000E800808F5000FAFF3A00060037002B
:10DA440010002000C07E88006109210040302B00B6
:10DA540013000900B0587800C000200090848800AA
:10DA64000002EB00040078004F0678004F05BE006A
:10DA74004F04BE000080FA0000000600881F7800F2
:10DA8400D5020700A83B020000000000F30F50007D
:10DA940006003600180307001A03070081312B0023
:10DAA40060407C00E23C0200000000004F0478006B
:10DAB4000000060016030700D1322B000303070001
:10DAC400E23C0200000000000000060031332B009D
:10DAD40060092100EC5A0200000000008000780078
:10DAE4000000E00004003200D9020700E23C02001A
:10DAF40000000000050037000503070081332B00F8
:10DB0400F2020700E23C02000000000000000600F0
:10DB1400881F7800B0020700A83B02000000000044
:10DB240091042000810F500006003600F502070022
:10DB340001342B0060407C00E23C02000000000045
:10DB4400ED0207004F047800000006000800FA0008
:10DB5400889FBE006C84570000ACBE0009112100F0
:10DB64000A0037006880570000405400E14F40002D
:10DB740005003200E3020700E1C2B30060C07C008C
:10DB8400D43B0200000000000804E8001880FB00F9
:10DB9400EC80570054C4020000000000D9020700C2
:10DBA400EC80570060C07C00E23C020000000000F2
:10DBB40065805700880F5000EAFF3A004F04BE000A
:10DBC4000080FA0000000600D1020700E181200075
:10DBD400BE020700E23C0200000000000000060054
:10DBE4002EC8AB0005003200C902070051352B00D6
:10DBF400B6020700E23C020000000000000006003C
:10DC04002380200094020700328020009502070040
:10DC140043802000900207005280200095020700F4
:10DC2400CAFF070000000600A38020008A02070044
:10DC3400B28020008B020700C38020008602070008
:10DC4400D28020008B020700C0FF070000000600FE
:10DC54006380200080020700728020008102070098
:10DC6400838020007C02070092802000810207004C
:10DC7400B6FF070000000600E380200076020700DC
:10DC8400F28020007702070003812000720207005F
:10DC94001281200077020700ACFF07000000060095
:10DCA400238120006C020700328120006D020700EE
:10DCB4004381200068020700528120006D020700A2
:10DCC400A2FF070000000600889FBE008A1F78009C
:10DCD4006C020700A83B020000000000F10F500096
:10DCE400030036008044EB00FA8220000A0037006B
:10DCF400680207001A0037000904E000050032003A
:10DD040083020700A1C3B30070020700D43B0200E2
:10DD1400000000000A05E8001A407800D8C4020098
:10DD240000000000804078002C020700D43B020071
:10DD3400000000001A407800ECC40200000000005B
:10DD44008040780026020700D43B02000000000057
:10DD54008944E800E6CF5400E7FF3A006602070072
:10DD64004F0578004F04BE000000060000000600C6
:10DD7400000006000000FE00000006006402070028
:10DD84006109210051020700E23C0200000000008A
:10DD94000000060000000600000006000000060067
:10DDA400000006005A020700D1352B004702070085
:10DDB400E23C0200000000000000060031020700FF
:10DDC400A83B020000000000A1042000810F5000C5
:10DDD40002003E002F020700060037004C02070035
:10DDE40021362B0039020700E23C0200000000004B
:10DDF4004102070000000600FC010700E23C0200AB
:10DE04000000000000000600FB010700E23C0200E5
:10DE14000000000000000600D60FE20004003200FB
:10DE2400F5010700E23C0200000000000300370097
:10DE3400EE010700E23C020000000000D62FEF00D4
:10DE440000000600D80FE20004003200EA010700D7
:10DE5400E23C02000000000003003700E301070079
:10DE6400E23C020000000000D82FEF000000060092
:10DE7400A1838000F2804000F5010700E23C02002B
:10DE840000000000000006000800FA006880570047
:10DE940041392B000302070010019000A0019000FB
:10DEA400829FBE00B3392B00831F78006E80570019
:10DEB400840D02000000000015020700EE805700E8
:10DEC40002020700E23C020000000000E68757005F
:10DED4000080FA00000006000C00FA006C80570075
:10DEE400F1392B0008000900315878009000B10086
:10DEF4000040EB00D0FF9F008F80E900804878004D
:10DF04008F00E90080487800A18380007148900068
:10DF14000058A3000400320011007800EC80570080
:10DF24001E7F020000000000F9010700EC8057008A
:10DF3400E6010700E23C0200000000000080FA0055
:10DF4400000006000800FA0068805700B13A2B0070
:10DF5400D401070000D09000213B2B00E14F50007A
:10DF640001003200713B2B0068805700AE0C0200A8
:10DF740000000000E6010700E8805700D301070015
:10DF8400E23C0200000000000080FA0000000600ED
:10DF94000800FA0068805700D13B2B009901070064
:10DFA4000008A30001003A00713B2B006880570071
:10DFB400AE0C020000000000D5010700E880570005
:10DFC400C2010700E23C0200000000000080FA00E9
:10DFD400000006000800FA0068805700413C2B004E
:10DFE400880107000028A30001003A00713B2B00C0
:10DFF40068805700AE0C020000000000C401070056
:10E00400E8805700B1010700E23C02000000000074
:10E014000080FA00000006000800FA00688057003B
:10E02400B13C2B007B0107000008A30001003A006B
:10E03400713B2B0068805700AE0C0200000000000A
:10E04400B3010700E8805700A0010700E23C02008A
:10E05400000000000080FA00000006000800FA003A
:10E0640068805700213D2B00660107000018A300BB
:10E0740001003A00713B2B0068805700AE0C02008F
:10E0840000000000A2010700E88057008F0107008C
:10E09400E23C0200000000000080FA0000000600DC
:10E0A4000800FA0068805700913D2B0059010700D1
:10E0B4000028A30001003A00713B2B006880570040
:10E0C400AE0C02000000000091010700E880570038
:10E0D4007E010700E23C0200000000000080FA001C
:10E0E400000006000600FA0066805700013E2B007F
:10E0F40005000900315878006000B100A083800059
:10E1040020109000E680570054C402000000000074
:10E114007F010700E68057006C010700E23C020023
:10E12400000000000080FA00000006000600FA006B
:10E1340066805700613E2B000500090031587800C5
:10E144006000B100B083800010109000E68057009A
:10E1540054C40200000000006D010700E68057006F
:10E164005A010700E23C0200000000000080FA00AF
:10E17400000006000800FA0068805700C13E2B002A
:10E184004801070040319000D0319000829FBE00CA
:10E19400B3392B00831F78006E805700840D020072
:10E1A400000000005A010700EE80570047010700F5
:10E1B400E23C020000000000E68757000080FA00FD
:10E1C400000006000800FA00B08380001001BE00C1
:10E1D40076F602000000000068815700333F2B00F0
:10E1E40006000900335978007200B100809FBE0018
:10E1F400B0392B00801F78006E805700840D020018
:10E204000000000042010700EE8057002F010700C4
:10E21400E23C020000000000E68757000080FA009C
:10E22400000006000800FA0068805700A13F2B0098
:10E234001C01070040309000E880570054C40200DD
:10E24400000000003201070011402B001F010700ED
:10E25400E23C0200000000000080FA00000006001A
:10E26400B1838000EE804000F9000700E23C020028
:10E274000000000000000600B08380001001BE0012
:10E2840076F60200000000000001BE00B0838000AA
:10E29400601090000038A3000400320000E427005E
:10E2A4005100200002015000838158000200BE008A
:10E2B400000006000800FA006880570081402B0027
:10E2C400D40007000038A30001003A00713B2B0082
:10E2D40068805700AE0C0200000000000C0107002B
:10E2E400E8805700F9000700E23C0200000000004B
:10E2F4000080FA00000006000800FA006880570059
:10E30400F1402B00C70007000018A30001003A00E9
:10E31400713B2B0068805700AE0C02000000000027
:10E32400FB000700E8805700E8000700E23C020019
:10E33400000000000080FA00000006000800FA0057
:10E344006880570061412B00B60007000028A30035
:10E3540001003A00713B2B0068805700AE0C0200AC
:10E3640000000000EA000700E8805700D70007001B
:10E37400E23C0200000000000080FA0000000600F9
:10E384000800FA0068805700D1412B00A90007005B
:10E394000018A30001003A00713B2B00688057006D
:10E3A400AE0C020000000000D9000700E88057000E
:10E3B400C6000700E23C0200000000000080FA00F2
:10E3C400000006000800FA006880570041422B0054
:10E3D400980007000028A30001003A00713B2B00BD
:10E3E40068805700AE0C020000000000C80007005F
:10E3F400E8805700B5000700E23C0200000000007E
:10E404000080FA00000006002000FA0000FE2F0041
:10E414000F004000B1422B001F0009003158780062
:10E424000002B10010002000801F7800801FEB0064
:10E4340021002000811F7800B2442B00821F780045
:10E4440080FD2F000F004000840D0200000000003A
:10E454007C0007008F8040009C000700E23C020023
:10E4640000000000E88757000080FA000000060062
:10E474002000FA0000FE2F000F00400041452B0051
:10E484001F000900315878000002B1000000EB00C1
:10E49400801F7800801F780020002000801F7800F3
:10E4A400B1442B00811F780080FD2F000F00400035
:10E4B400840D020000000000620007008F8040000D
:10E4C40082000700E23C020000000000E8875700D9
:10E4D4000080FA00000006000A00FA00C0838000F1
:10E4E40090B8920000B89200E10F4000E08F58000D
:10E4F400010036006000B8006A81570043472B00D2
:10E504000900090033597800A200B100809FBE00C1
:10E51400B0392B00801F780070805700840D0200F2
:10E52400000000007A000700F08057006700070031
:10E53400E23C020000000000E68757000080FA0079
:10E5440000000600A28380008250900080C4B300C3
:10E5540080CF500010003A00925090006B40400071
:10E5640080CF500006003A0069000700E1472B0005
:10E5740056000700E23C02000000000015003700CE
:10E5840063000700A1482B0050000700E23C020092
:10E59400000000000F0037009250900090C4B300B8
:10E5A40080CF500006003A005900070031492B0083
:10E5B40046000700E23C02000000000005003700AE
:10E5C40053000700D1492B0040000700E23C020041
:10E5D40000000000000006002E00070008112100C2
:10E5E4004800070060407C00000006004800070067
:10E5F40091382B003500370045000700E1382B0027
:10E60400320037002700070070109000213B2B00D8
:10E61400000006002800070060109000213B2B003A
:10E62400000006002400070050489000213B2B0006
:10E63400000006001B00070070489000213B2B00DF
:10E64400000006003200070081FD2F0000000600D4
:10E654002F0007001D003700934178008381FB00E1
:10E6640000000600124178004811DD00030071002B
:10E6740000000600124178004811DD00830071009B
:10E6840000000600220007002111210060C078006C
:10E694000000060010002000308488008830EF005D
:10E6A4000000060006000900315878007000B1002F
:10E6B400A08380000000060006000900315878009D
:10E6C4007000B100B0838000000006002211210018
:10E6D40060407900000006000A00070060C07D0069
:10E6E4000000060060092100312E2B0014000900EF
:10E6F40031587800000006008630EF008830EF00C3
:10E7040000000600020007000080E8000000060088
:10E7140018D1BF000080FB004200DD0000000600AD
:10E72400000178000100E0000D003A0080A52900F6
:10E73400801F780060012000801F780050A6290007
:10E74400801F780030A72900801F7800C086210030
:10E754000C0D020000000000580D02000000000033
:10E764001100980000C3B300404198005041980044
:10E77400604198000100780064FB02000000000082
:10E7840000000600B1C4B300014878000000060090
:10E79400881F7800000478001001900082489000DF
:10E7A4008180FB00124890004800DD0001027000E7
:10E7B400A24890008180FB00324890004800DD00B0
:10E7C4008102700040B9800051B98000800F52006E
:10E7D400818F5A000F00320044B9880055B988006F
:10E7E40018029000844990008381FB001449900032
:10E7F4004811DD0003007100A44990008381FB00EF
:10E80400344990004811DD0083007100EAFB0200E6
:10E814000000000060B9800071B98000E00F500072
:10E82400E08F58001A00320018029000C440900093
:10E834008180FB00544090004800DD00010170001D
:10E84400E44090008180FB00744090004800DD00AB
:10E854008101700062B9880073B9880018029000C1
:10E86400C44190008381FB00544190004811DD00B5
:10E8740003007100E44190008381FB007441900027
:10E884004811DD0083007100D4FB02000000000089
:10E8940018009000406890004600DE0061016000AE
:10E8A4008280FB0080B98000808F50000A00320013
:10E8B40081B988000204E000040032000040EB004B
:10E8C40052E3020000000000030037000040EB00A8
:10E8D40044E30200000000004F047800000006003A
:10E8E400C800FA00889FBE008A9FBE008C1F780073
:10E8F4008005780010A929000D0407001C002000E1
:10E904008C1F78000005EB008A1F7800200020008F
:10E91400801F780090B52900801F78000E007800D1
:10E92400840D0200000000001B0190008C40780060
:10E934000E007800020001000EF894000080FB0035
:10E94400801F7800D0B62900801F78000E00780060
:10E95400840D0200000000001B0190008C40780030
:10E964000E007800020001005C00020001000000BB
:10E974000004BE00B4FD0200000000000A0178009B
:10E984000004540081845C00D070220071002000D7
:10E99400800F5400818F5C0001003E000C01780060
:10E9A400821F7800B0B72900801F78000E0078001D
:10E9B400840D020000000000E103070002000100D2
:10E9C40066045700E0E72F000005440088809600A5
:10E9D400314090000080FB00801F780021409000AF
:10E9E4000080FB00801F7800114090000080FB0035
:10E9F400801F78001180FB00801F780090B82900E8
:10EA0400801F78000E007800840D020000000000D2
:10EA1400CB030700020001004AD892000080FB00EB
:10EA2400801F780000BA2900801F78000E0078004B
:10EA3400840D020000000000C10307000200010071
:10EA44007AE890000080FB00801F7800E0BA29007B
:10EA5400801F78000E007800840D02000000000082
:10EA6400E0FD2F0080874700B50307000200010086
:10EA74005AD892000080FB00801F7800C0BB290098
:10EA8400801F78000E007800840D02000000000052
:10EA9400AB0307000200010048409500384195008F
:10EAA400A84195000080FB0001FD2F00811F40005C
:10EAB4000281FB00811F41008381FB00819F410093
:10EAC400A0BC2900801F78000E007800840D02008D
:10EAD400000000009A03070002000100EB1F45003C
:10EAE400E0BD2900801F78000E007800840D02002C
:10EAF400000000009203070002000100084895008E
:10EB0400F840950068419500D84195000080FB00CD
:10EB1400801F78008180FB00811F78000281FB0048
:10EB2400821F78008381FB00831F7800C0BE290008
:10EB3400801F78000E007800840D020000000000A1
:10EB44007F030700020001004A689000FA8757001B
:10EB54000004E000100032004A68900021C4B300B1
:10EB6400E84F50000D0032004E60950031C4B300F0
:10EB7400E74F5000090032004E60950041C4B300D5
:10EB8400E14F5000050032004E60950051C4B300BF
:10EB9400E24F50000100320011C4B3000100FB0039
:10EBA400801F780030C02900801F78000E00780094
:10EBB400840D020000000000610307000200010050
:10EBC40050EA2F00801F470010C12900801F7800E1
:10EBD4000E007800840D02000000000058030700B6
:10EBE40002000100E88757004F0678004F05BE0079
:10EBF4004F04BE000080FA0000000600C800FA00BE
:10EC0400889FBE0080047800F0C1290048030700F3
:10EC14000E0178003035240011E424000099BE0070
:10EC240000922400E16424000099BE00F004200056
:10EC340000097800460307000200010080E72F0066
:10EC440000044700084092000080FB00801F780009
:10EC540070CE2900801F78000E007800840D020019
:10EC6400000000003A03070002000100284092005F
:10EC74000080FB00801F780050CF2900801F78009F
:10EC84000E007800840D020000000000300307002D
:10EC940002000100184092000080FB00801F7800F1
:10ECA40030D02900801F78000E007800840D020007
:10ECB40000000000260307000200010030102000BD
:10ECC400801F440010D12900801F78000E007800B6
:10ECD400840D0200000000001D0307000200010073
:10ECE400386092000080FB00801F7800F0D129007A
:10ECF400801F78000E007800840D020000000000E0
:10ED04001303070002000100486092000080FB002A
:10ED1400801F7800D0D22900801F78000E00780070
:10ED2400840D020000000000090307000200010036
:10ED3400586092000080FB00801F7800B0D3290047
:10ED4400801F78000E007800840D0200000000008F
:10ED5400FF0207000200010028D892000080FB0097
:10ED6400801F780090D42900801F78000E0078005E
:10ED7400840D02000000000000FE2F008087470081
:10ED8400F3020700020001004F04BE000080FA00F5
:10ED940000000600DC00FA00889FBE008A1F78008D
:10EDA400000578005E3C9600B0D62900E00207001A
:10EDB400384090000080FB00801F780028409000BD
:10EDC4000080FB00801F7800184090000080FB004A
:10EDD400801F78001880FB00801F780030E3290032
:10EDE400801F78000E007800840D020000000000EF
:10EDF400DB02070002000100784090000080FB0065
:10EE0400801F7800684090000080FB00801F78001D
:10EE1400584090000080FB00801F7800484090001C
:10EE24000080FB00801F780040E42900801F7800E8
:10EE34000E007800840D020000000000C8020700E4
:10EE440002000100384890000080FB00801F780019
:10EE5400284890000080FB00801F7800184890002C
:10EE64000080FB00801F7800084890000080FB00B1
:10EE7400801F780070E52900801F78000E0078005C
:10EE8400840D020000000000B5020700020001002A
:10EE9400784890000080FB00801F7800684890004C
:10EEA4000080FB00801F7800584890000080FB0021
:10EEB400801F7800484890000080FB00801F780085
:10EEC400D0E62900801F78000E007800840D02002F
:10EED4000000000080FD2F0080874700A00207008B
:10EEE40002000100385090000080FB00801F780071
:10EEF400285090000080FB00801F7800185090007C
:10EF04000080FB00801F7800085090000080FB0008
:10EF1400801F7800F0E72900801F78000E00780039
:10EF2400840D0200000000008D02070002000100B1
:10EF3400785090000080FB00801F7800685090009B
:10EF44000080FB00801F7800585090000080FB0078
:10EF5400801F7800485090000080FB00801F7800DC
:10EF640010E92900801F78000E007800840D02004B
:10EF7400000000007A0207000200010038589000E7
:10EF84000080FB00801F7800285890000080FB0060
:10EF9400801F7800185890000080FB00801F7800C4
:10EFA400085890000080FB00801F780070EA290058
:10EFB400801F78000E007800840D0200000000001D
:10EFC4006702070002000100486890004600DE0066
:10EFD400E11F6000F0EB2900801F78000E0078002C
:10EFE400840D020000000000E0FD2F008087470030
:10EFF4005B02070002000100FC1F440090EC2900A2
:10F00400801F78000E007800840D020000000000CC
:10F014005302070002000100890C20008E84440082
:10F0240070D5290013000900B05C78004901B100D3
:10F03400D0022000080040001080FB00E868900027
:10F04400C808DD0080807000786890000080FB00B4
:10F05400087190004811DD000001710018709000E3
:10F064000080FB00A8719000C819DD008081710048
:10F07400090078000A020700891F780060ED290062
:10F08400801F78000E007800840D0200000000004C
:10F094003302070002000100E88757004F0578009B
:10F0A4004F04BE000080FA0000000600DC00FA00F5
:10F0B400889FBE008A1F78000005780030EF290081
:10F0C4001B02070080E72F00000447001868920025
:10F0D4008868920078619200E86192000080FB00E9
:10F0E400801F78008180FB00811F78000281FB0073
:10F0F400821F78008381FB00831F780030E329009E
:10F10400801F78000E007800840D020000000000CB
:10F11400130207000200010058689200C8689200B8
:10F1240038699200A86992000080FB00801F780073
:10F134008180FB00811F78000281FB00821F780020
:10F144008381FB00831F780040E42900801F78003E
:10F154000E007800840D0200000000000002070089
:10F164000200010018709200887092007869920081
:10F17400E86992000080FB00801F78008180FB001A
:10F18400811F78000281FB00821F78008381FB00CD
:10F19400831F780070E52900801F78000E00780036
:10F1A400840D020000000000ED01070002000100D0
:10F1B40058709200C870920038719200A871920041
:10F1C4000080FB00801F78008180FB00811F780095
:10F1D4000281FB00821F78008381FB00831F78007B
:10F1E400D0E62900801F78000E007800840D02000C
:10F1F4000000000080FD2F0080874700D801070031
:10F2040002000100187892008878920078719200C8
:10F21400E87192000080FB00801F78008180FB0071
:10F22400811F78000281FB00821F78008381FB002C
:10F23400831F7800F0E72900801F78000E00780013
:10F24400840D020000000000C50107000200010057
:10F2540058789200C878920038799200A879920080
:10F264000080FB00801F78008180FB00811F7800F4
:10F274000281FB00821F78008381FB00831F7800DA
:10F2840010E92900801F78000E007800840D020028
:10F2940000000000B20107000200010018C0920043
:10F2A40088C0920078799200E87992000080FB008F
:10F2B400801F78008180FB00811F78000281FB00A1
:10F2C400821F78008381FB00831F780070EA290085
:10F2D400801F78000E007800840D020000000000FA
:10F2E4009F0107000200010028D092004600DE00C2
:10F2F400E11F6000F0EB2900801F78000E00780009
:10F30400840D020000000000E0FD2F00808747000C
:10F31400930107000200010028D092004700DE009C
:10F32400E11F6000B0FB2900801F78000E00780008
:10F33400840D0200000000008901070002000100A2
:10F3440020142000801F440090EC2900801F7800C6
:10F354000E007800840D0200000000008001070008
:10F3640002000100890C20008E844400F0ED290085
:10F3740013000900B05C78004901B1003015200089
:10F38400080040001080FB00C8D09200C808DD00CF
:10F394008080700058D092000080FB0068D19200F9
:10F3A4004811DD000001710078D092000080FB005C
:10F3B40088D99200C819DD008081710009007800A5
:10F3C40037010700891F780060ED2900801F78004D
:10F3D4000E007800840D02000000000060010700A8
:10F3E40002000100EC8757004F0578004F04BE006F
:10F3F4000080FA0000000600E400FA00889FBE00C6
:10F404008A9FBE008C1F78008005780080E72F005B
:10F414008004470049FE920070FC29004401070063
:10F424008A0C20000E054500680D20000E044400DF
:10F43400080078005AFB02000000000006000900E2
:10F44400381D7800EA00B100E800B1003EC8910020
:10F454000080FB00801F78002EC891000080FB0014
:10F46400801F78001EC891000080FB00801F780078
:10F474001A80FB00801F7800F0082A00801F7800A3
:10F484000E007800840D0200000000002C0107002B
:10F49400020001007EC891000080FB00801F7800FC
:10F4A4006EC891000080FB00801F78005EC8910048
:10F4B4000080FB00801F78004EC891000080FB0094
:10F4C400801F7800800A2A00801F78000E007800D0
:10F4D400840D020000000000190107000200010071
:10F4E4003ED091000080FB00801F78002ED0910058
:10F4F4000080FB00801F78001ED091000080FB007C
:10F50400801F78000ED091000080FB00801F7800DF
:10F51400300C2A00801F78000E007800840D020051
:10F524000000000006010700020001004ED0910017
:10F534000080FB00801F7800C00D2A00801F780027
:10F544000E007800840D020000000000E8FD2F008A
:10F5540088874700FA0007000200010039F0920092
:10F56400A9F0920019F1920089F192000080FB0049
:10F57400801F78008180FB00811F78000281FB00DE
:10F58400821F78008381FB00831F7800E00E2A002D
:10F59400801F78000E007800840D02000000000037
:10F5A400E70007000200010079F09200E9F0920000
:10F5B40059F19200C9F192000080FB00801F78008D
:10F5C4008180FB00811F78000281FB00821F78008C
:10F5D4008381FB00831F780080102A00801F78003D
:10F5E4000E007800840D020000000000D400070023
:10F5F4000200010039F89200A9F8920019F992006A
:10F6040089F992000080FB00801F78008180FB0054
:10F61400811F78000281FB00821F78008381FB0038
:10F62400831F780040122A00801F78000E007800A3
:10F63400840D020000000000C10007000200010068
:10F644000C86FB008C1F7800E0132A00801F7800D2
:10F654000E007800840D0200000000008887470037
:10F66400B7000700020001004F0678004F05BE00F6
:10F674004F04BE000080FA00000006000000FA00FB
:10F68400889FBE0081447800014878002F18B0009C
:10F69400E1E72F0001844700C0000900301C780016
:10F6A4002818B1002018B1001C88020000000000D6
:10F6B40088077800268802000000000009407800CE
:10F6C400A2030200010000004F04BE000080FA0003
:10F6D400000006000600FA00889FBE008A1F78001A
:10F6E400010578000204780000CDB3001240400008
:10F6F400A1C2B300814F500006003E008204E8001E
:10F7040000CDB30019404000A1C2B300814F5000A6
:10F7140005003600110020000A0078008CF1020078
:10F72400000000001B003700630020006C815700BC
:10F7340000042000010020008EEC02000000000004
:10F7440018447800C8F79F0099447800D9F79F00BF
:10F754000004200001002000F2EC02000000000080
:10F76400610020006C80570018ED020000000000CA
:10F7740036ED0200000000001A01900011C0B30031
:10F7840010152A0002000100208A02000000000077
:10F794000000FE004F0578004F04BE000080FA0010
:10F7A400000006000600FA00889FBE008A1F780049
:10F7B400000578000204BE00630020006C8157003D
:10F7C40000042000010020008EEC02000000000074
:10F7D400B8BF9F00C9BF9F000004200001002000A3
:10F7E400F2EC020000000000610020006C80570071
:10F7F40018ED02000000000036ED020000000000D9
:10F80400783D9900098599004F0578004F04BE00A2
:10F814000080FA0000000600C800FA00881F780083
:10F824000104780061F32F008F80400052152A00F4
:10F83400C7000900B2587800810CB10080809100A3
:10F8440070389100E10F4000E08F5800010036004D
:10F854006000B800809FBE00D0212A00801F78007D
:10F8640000F32F000F004000840D02000000000090
:10F874001801900011C0B30000F32F000F004000E6
:10F8840002000100E68757004F0478000080FA0068
:10F8940000000600208A02000000000000000600AC
:10F8A4000600FA00889FBE008A9FBE008C9FBE009F
:10F8B40000057800F1B79F0082BF9F0093BF9F00AF
:10F8C4008004EB008905780072865700ADC3B3004D
:10F8D400040037000B00E000020032008D747D004C
:10F8E4008904E8003C44780008407800D8C4020049
:10F8F4000000000000F57C0008407800ECC4020021
:10F904000000000089004500904098008984E800C8
:10F914008B05E800E68F5500EEFF3A004F06BE0067
:10F924004F05BE004F04BE000080FA000000060030
:10F93400C7000900305F78008E0CB100000006009B
:10F944001B01900011C0B3000E00780000000600F7
:10F954001901900011C0B3000E00780000000600E9
:10F964001A01900011C0B3000E00780000000600D8
:10F974008040EB0021E0980021F898008000EB0023
:10F98400413898006011B8001200980023009800D4
:10F994003200980043009800F04890000104A10050
:10F9A40071489800F04890000114A1007148980033
:10F9B400F04890000124A10071489800F04890009C
:10F9C4000154A1007148980011C0B30041C89800C7
:10F9D400F01090000130A10071109800E007B00011
:10F9E4001AE40200000000000000060061C4B30035
:10F9F40021509800F1C6B30031509800ECC050007B
:10FA040041509800F2C040005150980081C0E90074
:10FA140061509800EEC0500071509800EDC0400055
:10FA2400015898008040EB00115898002158980024
:10FA340031589800415898005158980061589800DE
:10FA4400715898007011900001C0980041C098004E
:10FA540001D0980061052000011898001118980041
:10FA6400211898003118980041189800F5C05000EA
:10FA7400217898008102200021109800C1FF2F00F6
:10FA8400010161000220A00072109800000006002D
:10FA9400881F78008A9FBE0000047800E007B00049
:10FAA400FEE4020000000000B1BB80000100E80099
:10FAB400B0BB8800E18F500007003200030039001A
:10FAC400E28F5000070032007637EF00080078001C
:10FAD400340007000600370008007800940007008F
:10FAE40003003700080078006AF7020000000000F5
:10FAF400781090000038A300240032005C0002005B
:10FB04000100000038159000C81590000A0150004B
:10FB14008B815800030033000200BE00520307002B
:10FB24000900370061006100010020008301D10059
:10FB34000281D30002007000838070004A03070032
:10FB44000001BE004A030700027A2300038A24004E
:10FB54003E070200000000000000E00005003C0039
:10FB64005C00020001000000800F5500818F5D00E1
:10FB740006003600781090000030A1007014980040
:10FB8400080078008EA4020000000000080078003D
:10FB9400ECA00200000000004F05BE004F047800F6
:10FBA40000000600889FBE008A9FBE008C9FBE0096
:10FBB4008004780070389000E20F50000C0032008E
:10FBC40079489000F1CDB30001406000F04C9800FA
:10FBD4000040EB0080D49800794890000140600018
:10FBE400250307000000EB00F09498004C00370058
:10FBF40009809000E10F500044003A00799690008B
:10FC0400EE0F560018003C0009A5900099A590003D
:10FC140069999000F99990000A00BE004207020019
:10FC2400000000000000E0003D003200EA9C980063
:10FC3400FB9C98000C0446000809B0000200240054
:10FC4400C36124000A00BE00460702000000000051
:10FC5400AE0702000000000000B47C000C00E800C5
:10FC6400F09498002E0037000A0920000905450089
:10FC74006066B8008005EB001A0478006140B900A2
:10FC8400F90207000800E00003003D000200200024
:10FC940003782400F60207000001BE000C00BE0039
:10FCA400F30207000006BE008B05E8000A85E800A1
:10FCB400EF8F5500F0FF3A000000EB00F09498003D
:10FCC40002002000031724000C00BE00FE05020001
:10FCD40000000000E4070200000000004200DD0014
:10FCE400A2002000110009000280D800E292200046
:10FCF40000015100929C9800820C78007948900091
:10FD04000054A000DC020700050037007948900089
:10FD14000054A100F04C98000040EB0080D49800FF
:10FD24004F06BE004F05BE004F04BE000000060093
:10FD3400881F78000004780000809000E20F5000D3
:10FD440006003200784890000034A100704C9800FE
:10FD54000000EB00209C98003500370078489000A4
:10FD64000034A000704C9800784890000018A3005C
:10FD74002F003A0028989000E10F50001E00320036
:10FD8400E20F500021003200A8A09000E0232000E0
:10FD9400808F50000A003E00784890000018A300AD
:10FDA40023003A0010002000209C98006011B80045
:10FDB4000800780074A40200000000001C00370052
:10FDC400502D2000808F5000190036007848900094
:10FDD4000018A30016003A0020002000209C980080
:10FDE40048319000D83190000800780074A40200D3
:10FDF400000000000E003700A8A09000E0232000BF
:10FE0400808F50000A00360004003700A8A090003C
:10FE1400502D2000808F500005003E00080078001F
:10FE24006CA40200000000000000EB00209C98007D
:10FE34004F047800000006000002BE000000E0004D
:10FE440004003D00D0C2B300804878000402EA00F8
:10FE540002003700B0C2B300804878004206200098
:10FE6400110009000202D80001C3B300814140001F
:10FE7400934298000280B90000005200A2002000C2
:10FE8400801F7800110009000200D80000017800EA
:10FE94004F00780001C3B30001424100A44298001E
:10FEA400E4C2B300B44298006A11B90002005000E1
:10FEB40001404000C04298000040EB00D04298004E
:10FEC40000000600D000FA00889FBE00800478007D
:10FED40000D32A00C7000900305F78008E0CB100FF
:10FEE4006600570081F32F008100400070C0960027
:10FEF4000058A3000B003200880C20000E044400BC
:10FF040080D22A0007000900305C78008800B10024
:10FF14001100780088007800C7FF0700881F780068
:10FF24000200370060E02A00801F780081DF2A0089
:10FF3400811F78000E007800840D0200000000008C
:10FF4400E487570051020700020001001EC096001A
:10FF54000018A300020032006000B800020037005D
:10FF64002E189700BE189700809FBE00F1E02A006B
:10FF7400811F78000E007800840D0200000000004C
:10FF8400E68757004102070002000100660457009B
:10FF94007818970088209700809FBE00E1E12A002E
:10FFA400811F78000E007800840D0200000000001C
:10FFB400360207000200010078C09600E11F6000CD
:10FFC400D0E22A00801F78000E007800840D020021
:10FFD400000000002D0207000200010078C0960016
:10FFE4000000D100E11F6000B1E32A00811F780006
:10FFF4000E007800840D02000000000023020700B8
:020000040001F9
:100004000200010078C096004200DE00E11F60009B
:1000140090E42A00801F78000E007800840D02000E
:1000240000000000190207000200010078C09600D9
:100034004500DE00E11F600071E52A00811F7800A1
:100044000E007800840D0200000000000F0207007B
:100054000200010078C096004300DE00E11F60004A
:1000640050E62A00801F78000E007800840D0200FC
:1000740000000000050207000200010078C096009D
:100084004400DE00E11F600031E72A00811F780090
:100094000E007800840D020000000000FB01070040
:1000A40002000100C2C2BF000000FB000080EA00A1
:1000B4004F00DE00801F780010E82A00801F7800BF
:1000C4000E007800840D020000000000E0FD2F0007
:1000D40080874700ED010700020001004F04BE00C5
:1000E4000080FA0000000600C800FA00889FBE00E5
:1000F4008A9FBE000005780000F32F000F00400027
:10010400F1E82A00C700090031587800800CB100DA
:10011400E604500088F32F0008844400F21F4400D2
:1001240070F52A00801F7800C0F22F000F004000F5
:10013400840D020000000000D80107000F004000F9
:100144000200010048309000D8309000809FBE002B
:1001540051F62A00811F780060F22F000F00400042
:10016400840D020000000000DE01070060F22F0091
:100174000F0040000200010089C89600EA8757007A
:1001840070C4B30080CF50000E003A0099C89600A6
:1001940000C0E80080CF500005003A00920420001F
:1001A400821F780040F72A00801F78001A00370069
:1001B40071042000811F780042F72A00821F780012
:1001C4001500370080C4B30080CF50000E003A0001
:1001D400BFF094006B40400080CF500005003A000F
:1001E40030052000801F780041F72A00811F780025
:1001F4000900370082042000821F780040F72A009B
:10020400801F78000400370011042000811F78004B
:1002140042F72A00821F7800C0F22F000F0040002E
:10022400840D0200000000009C0107000F00400044
:1002340002000100E487570020F32F0001F32F0090
:100244008F8040000084400008D090000000FB0034
:10025400801F780022F82A00821F7800C0F22F0045
:100264000F004000840D0200000000008B01070015
:100274000F004000020001000903200088844400AC
:1002840018042000E48757006B042000B91F78008D
:10029400881F780010F92A00801F7800A0F22F0030
:1002A4000F004000840D0200000000008D010700D3
:1002B400A0F22F000F004000020001000804E80033
:1002C400E68757008B0F5400F0FF3A0020F32F000D
:1002D40001F32F008F8040000084400028789000B4
:1002E4000000FB00801F780002FA2A00821F7800B9
:1002F400C0F22F000F004000840D02000000000037
:10030400660107000F004000020001007810900011
:100314000000D100E11F6000E0FA2A00801F78008D
:1003240080F22F000F004000840D02000000000046
:100334006C01070080F22F000F0040000200010052
:10034400A8109000811F7800C2FB2A00821F780049
:1003540040F22F000F004000840D02000000000056
:100364006001070040F22F000F004000020001006E
:1003740078109000E11F6000A0FC2A00801F780024
:1003840000F22F000F004000840D02000000000066
:100394005401070000F22F000F004000020001008A
:1003A400781090004200DE00E11F600081FD2A0009
:1003B400811F7800C0F12F000F004000840D02005F
:1003C4000000000047010700C0F12F000F004000AB
:1003D40002000100F48757004F05BE004F04BE0021
:1003E4000080FA00000006000000FA00889FBE00AA
:1003F4008A1F7800000578008104780002047800E0
:1004040001012000020078004E03020001000000F8
:100414000004E00005003A002100200009007800F3
:100424008CF102000000000010003700720045004B
:1004340088007800AE0C0200000000008F0CB000B1
:1004440080F32F0000844700630009003A1C780001
:10045400880CB1008A0CB1004A8702000000000039
:100464008807780026880200000000004F05780005
:100474004F04BE000080FA00000006000000FA00ED
:10048400881F7800000278008101780006010700C7
:100494000500360021002000030078008CF10200E2
:1004A400000000000A003700217A98008F0CB00089
:1004B40080F32F0000844700000107004A870200F0
:1004C4000000000088077800268802000000000071
:1004D4004F0478000080FA00000006000000FA00D3
:1004E400881F7800800378008101780082027800F8
:1004F400ED0007000B003E000100FB00F1FB2F00A4
:100504000103400092409000B0C2B30080CF50007D
:10051400090032000084EB0000C0E80080CF5000E6
:100524000600320021002000030078008CF1020054
:10053400000000002500370018002000354190001D
:100544000201FB00400620000091B9002540900004
:100554000000FB0004FD2F0004004000843E200046
:100564000480B90000014100454090000000FB00F8
:100574006A00B90000014100554090000000FB00F2
:100584000001410000B32E000001410006024300B7
:100594000403B00002C0B90000B27B008F0CB000AD
:1005A40080F32F000084470063000900371C7800A3
:1005B400880CB100870CB1004A87020000000000DB
:1005C4008807780026880200000000004F047800A5
:1005D4000080FA00000006000000FA00881F78007E
:1005E400000278008101780010C4B300924F10001B
:1005F4000500320011002000030078008CF1020095
:10060400000000000B00370010C4B3000052980033
:100614008F0CB00080F32F0000844700A700070070
:100624004A8702000000000088077800268802003C
:10063400000000004F0478000080FA00000006006B
:100644000101780070489000110020000018A300F8
:100654000500320051002000020078008CF10200F5
:10066400000000008000EB0001007800000006009C
:100674000001BE00704890000018A300060032007C
:1006840051002000030078008CF1020000000000FB
:100694008000EB0009003700724890001100200030
:1006A4000028A30005003A00C100200003007800E0
:1006B4008CF10200000000008000EB00EAFF37002C
:1006C4000000FA00881F78008180FB008100EA00A6
:1006D400CF08DE0081804000701190000210A1005C
:1006E40001017100721098008F0CB00081F32F008B
:1006F40001844700760007004A87020000000000DA
:100704008807780026880200000000004F04780063
:100714000080FA00000006000000FA00881F78003C
:10072400221098008F0CB00081F32F000184470041
:10073400670007004A87020000000000880778006D
:1007440026880200000000004F0478000080FA00B0
:10075400000006000000FA00881F78008180FB007A
:100764008100EA00CF08DE00C208DD0070119000AD
:100774000220A10001017100721098008F0CB000DA
:1007840081F32F0001844700510007004A870200CB
:10079400000000008807780026880200000000009E
:1007A4004F0478000080FA00000006000000FA0000
:1007B400881F78008001780001027800704890005A
:1007C4000058A30005003A007100200004007800DE
:1007D4008CF10200000000000D00370082D1980067
:1007E4008F0CB00080F32F000084470063000900E1
:1007F400331C7800880CB100830CB1004A870200D6
:10080400000000008807780026880200000000002D
:100814004F0478000080FA00000006000000FA008F
:10082400881F7800E1806000701190000200A10030
:1008340001017100721098008F0CB00081F32F0039
:1008440001844700220007004A87020000000000DC
:100854008807780026880200000000004F04780012
:100864000080FA0000000600A80504000000000053
:100874008406040000000000F04C980079489000C1
:100884000034A100F04C980000000600190190000B
:1008940011C0B3000E00780000000600110007002C
:1008A400C0F22F000000060092407800F0CBB300A5
:1008B40000C04000E44F500000000600630009003F
:1008C400341C7800880CB100840CB10000000600D0
:1008D40063000900301C7800880CB100800CB10062
:1008E400000006001A01900011C0B30000000600C9
:1008F400505021000100200044372100B53A210066
:100904004509DD00CB01DE00830171004501DD00F6
:100914000001410081814900344078000080FB00DF
:10092400010020000200400083804800850F52002F
:10093400F3FF3A0000000600889FBE008A9FBE00B5
:100944008C1F78000005BE0002067800C202070072
:1009540010C0B300DF000700F13A2100950307003F
:10096400B0D3BF004800DD0001047000113B21003A
:1009740090030700B2D3BF004800DD00810470007B
:10098400DBFF0700800F5400818F5C00CC003A002D
:1009940035030700EB0F5000C9003A007200450010
:1009A400A137210010000900315878001001B1006E
:1009B400000320000A004000729C8000839C800099
:1009C4000298BE00929C8000A39C80000298BE0006
:1009D400B39C8000030878008DD3BF00207D98006D
:1009E400FDD3BF006140600000D5980010C0B30083
:1009F40040CD98009137210091407800015598002E
:100A0400E13F21009140780080C06000C208DD0011
:100A14007A489000B8CFB3000840600001407000ED
:100A2400704D9800B1382100620307008CD3BF00D9
:100A340010030700201598001103070062006000EE
:100A4400FA1290000510A1008082720075159800BA
:100A5400313D210091407800614D98000B0307005F
:100A64000106B000463721000B0307005205980029
:100A7400630598005A019000EA019000120598005D
:100A8400230598001A009000AA00900030059800F1
:100A940041059800C8D3BF0040C598000080FB0002
:100AA400000040004005B00006004000FE020700C0
:100AB40010259800313B21009140780001C5980031
:100AC400F20207000104B000F3020700621D98005F
:100AD400731D9800EA02070061006000E7FF2F0021
:100AE400878262008082720075159800FDD3BF0072
:100AF4004400DE0064006000B2FF2F0082826200C6
:100B040080827200751598006E804500E1392100DD
:100B140010000900315878001001B1008339210018
:100B240093417800F35D9800FDD3BF000080FB0083
:100B34004700DE004200DD00DB48900088C0600012
:100B440080C07000D14D980099D3BF000080FB0095
:100B540090159800CA02070064006000EB12900030
:100B64008282620080827200E5159800813E210035
:100B740091407800C14D9800C40207004107B000BD
:100B840086804000CC020700C2059800D305980077
:100B94004B009000DB009000808DBE001B01BE0066
:100BA400A2059800B3059800B5020700680060002C
:100BB4000530A10080827200E5159800FDD3BF00C6
:100BC4004500DE006100600087826200808272005E
:100BD400E5159800A1392100F60207009BD3BF0058
:100BE4004800DD0001017000C1392100F102070055
:100BF4009DD3BF004800DD0081017000A21598005C
:100C0400B3159800633721009341780083D5980089
:100C140078D3BF00004E7800E13F21009140780076
:100C24008100D000F08060006B1090000040A100B3
:100C340001007000E0159800F13F2100DD0207007B
:100C440000D4BF008B02070031C72200810F50007F
:100C540009003200A3020700FE93A9000040EB0044
:100C640001F4B70002F4B70003F4B70004F4B700CA
:100C74000000EB0013003700FED3BF004400DE0089
:100C84006100600080E5980011402100C90207005E
:100C940002D4BF004800DD00010170003140210092
:100CA400C402070004D4BF004800DD0081017000C5
:100CB40082259800932598000000EB00010037007E
:100CC400100020004F0678004F05BE004F04BE0000
:100CD4000000060012C9B30041372100F3010700E8
:100CE400000006000000FA0000C0EB00E9F3B700C2
:100CF400EAF3B700EBF3B700ECF3B700EDF3B7009A
:100D0400EEF3B700EFF3B700F0F3B700F1F3B70079
:100D1400F2F3B700F3F3B700F4F3B700F5F3B70059
:100D2400F6F3B700F7F3B700F8F3B700F9F3B70039
:100D3400FAF3B700FBF3B700FCF3B7006683570080
:100D440064F52F0004024300A6E296001401BE00DD
:100D54000580FB004200DD00813E210001004000CF
:100D640012409800C810DE002140980033409800DB
:100D7400C818DE004140980005007800E8F3B70089
:100D84006E004200E139210010000900B0587800DB
:100D94001001B10056F0960098F3B700246090005B
:100DA40099F3B700641090004200DE0061406000D7
:100DB4004300DD0072CFB300D13F21004E02070093
:100DC400FDF3B700641090004300DE006140600052
:100DD4004400DD00F3CEB30083C060007802070056
:100DE400446090009AF3B700546090009BF3B700FE
:100DF400646090009CF3B700746090009DF3B700AA
:100E040064109000614060004500DD000154A100C1
:100E14006B02070036E096004200DE0061006000CD
:100E24004700DD000174A100650207006410900012
:100E34004400DE00614060004300DD00E13F21002A
:100E44002D020700FEF3B7002602070004E090001D
:100E5400614060004400DD0083C0600080C0700019
:100E640001007800FEF3B70004C0900001F4B7005D
:100E740014C0900002F4B70024C0900003F4B7003B
:100E840034C0900004F4B7000080FA0000000600AB
:100E94000000FA00889FBE0000C0EB00D4F3B70046
:100EA400D5F3B700D6F3B700D7F3B700D8F3B7003C
:100EB400D9F3B700DAF3B700DBF3B700DCF3B7001C
:100EC400DDF3B700DEF3B700DFF3B700E0F3B700FC
:100ED400E1F3B700E2F3B700E3F3B700E4F3B700DC
:100EE400E5F3B700E6F3B700E7F3B700EA8357008A
:100EF40084F32F000482430067C3960057199700B8
:100F0400E71997000680FB004200DD00413D210007
:100F140001004000F50F200005486100C810DE0004
:100F2400114098008580610021409800C818DE00B7
:100F34003140980006007800D3F3B70004C0900055
:100F4400B3F3B70044C09000C8F3B70084D0900056
:100F5400E1C06000E2CFB300FDD3BF0002406000F7
:100F640001407000FDF3B70072004200A137210078
:100F740010000900B05878001001B10000032000EF
:100F8400040040003004BE00789C8800899C8800DE
:100F94003004BE00989C8800A99C8800100078004A
:100FA400B09C8800247890008DF3B70007C89600A1
:100FB40079F3B70024109000050060008BF3B700AC
:100FC400546090008CF3B700741090000000D100BE
:100FD400614060004200DD00D13F21009140780073
:100FE4000124A100C90107006140600000404000E5
:100FF4000114A100C50107004200DE006140600049
:101004004600DD000164A100ED010700F7C0960071
:10101400C208DE00E1806000FED3BF000240600031
:1010240001407000FEF3B7004F04BE000080FA00D8
:10103400000006000000FA000FF8940078F3B700EF
:101044000080FA0000000600B0C0B30074F3B700DB
:101054007573EF0026FE0700AFF3B7004801DE000A
:1010640002007800B0F3B70001007800B1F3B700D4
:101074004808DE00B2F3B7000100070000000600D4
:1010840012C9B3004137210010C0B3004201070068
:1010940000000600889FBE008A9FBE008C9FBE0091
:1010A4008E1F78006055B800000778008EC090004D
:1010B40076010700403B2100970107000104B000BE
:1010C400828040006E18900000C1EB0082486000EE
:1010D4005E789000904098007E189000F20F2000F7
:1010E40002006000A04098007E789000B040980014
:1010F4004137210081044600180020008C46780006
:101104000C404400B9407800120107000804E800CC
:10111400E50F5400FAFF3A000D40E800FD00070017
:101124000080FB0002F02F00020565000005750039
:101134000DC0E800F70007004800DD00F10F2000B3
:10114400010565000005750063C04600F100070055
:101154000080FB0002F02F00828565008085750009
:1011640064C04600EB0007006F0107008EC29000C8
:101174008580FB00C208DD000104B0006F01070098
:10118400030032000540E80000C79800C7FF37009D
:101194004EC090000080FB0000004000913C210004
:1011A4008100400042372100828450004005B00095
:1011B40082007800020040002EC190001240980086
:1011C4003EC1900022409800018544001800200090
:1011D4000946780008C04400BA407800DD000700E2
:1011E4000804E800E30F5400FAFF3A000C40E8005A
:1011F400C80007000080FB0001F02F008185650016
:10120400808575000CC0E800C20007004800DD00BE
:101214008B85FB00808575004EC190000280FB0029
:1012240000004000813C2100010040001E01070035
:10123400808F5500030032000240E80040C7980048
:10124400D3FF37004F0778004F06BE004F05BE009E
:101254004F04BE0000000600889FBE008A9FBE00A7
:101264008C9FBE008E1F78006055B8000007780080
:10127400EE48900005010700403D210026010700CB
:101284001E019000AE0190000106B0004437210019
:101294008480400000C0EB00804861004810DE00FC
:1012A40090409800F40F200004806100A040980052
:1012B4004818DE00B0409800270107000C404400A5
:1012C400B9407800A30007000804E800E50F5400C3
:1012D400FAFF3A001E009000AE00900050079800FC
:1012E400610798000D40E8008A0007001F0107000D
:1012F4008800070023010700860007002701070074
:101304008400070008010700EE4A90008580FB0076
:10131400C208DD000106B000080107000300320026
:101324000540E800604F9800D1FF37004F07780070
:101334004F06BE004F05BE004F04BE00000006006D
:10134400889FBE008A9FBE008C9FBE008E1F7800BF
:101354006055B80000077800CE489000CB00070025
:10136400903E2100EC0007001E01BE004107B000C2
:101374004437210084804000F40F20000400610001
:10138400904098004810DE00A0409800048061005E
:10139400B04098004818DE00C0409800EE000700F6
:1013A4000C404400B94078006A0007000804E800D3
:1013B400E50F5400FAFF3A001E00BE0040079800F3
:1013C400510798000D40E80052000700E7000700AD
:1013D40050000700EB0007004E000700EF00070075
:1013E4004C000700D0000700CE4A90008580FB0027
:1013F400C208DD004107B00042372100828040006E
:10140400AD000700820F5500838F5D00030032009A
:101414000540E800404F9800CFFF37004F077800A1
:101424004F06BE004F05BE004F04BE00000006007C
:1014340076F3B70004FF0700000006008A000700E7
:101444000000E80074F3B7004800DE0075F3B7004D
:101454000BFF070000000600C482A8002012200031
:101464001013880000002800001388000000060004
:101474000080FB004013880060C2BF000008A30086
:10148400FDFF3200401380000080FB0000000600D6
:10149400C482A90050C0B300F5FF07000040EB0070
:1014A400F3FF0700C482A800F7FF3700889FBE003F
:1014B4008A9FBE0080447800810578000245780048
:1014C400F3FF070063046000FDFF3A00C482A90033
:1014D40030C0B300E6FF070009407800E4FF0700CE
:1014E4000A04E000070032008B0478000040EB009F
:1014F400DFFF0700805C78000844E800884F55004F
:10150400FAFF3A00C482A8004F05BE004F04BE0093
:1015140000000600889FBE0080447800DCFF0700BE
:1015240063046000FDFF3A00C482A90030C0B30028
:10153400CFFF070009407800CDFF0700084078007E
:10154400CBFF0700C482A8000080FB004F04BE004C
:1015540000000600889FBE000044780081447800A3
:10156400CBFF070063006000FDFF3A003300070073
:10157400C482A90020C0B300BDFF07000840780062
:10158400BBFF070009407800B9FF0700C482A80028
:101594004F04BE0000000600889FBE008A9FBE0064
:1015A400804478000105780082457800B8FF070080
:1015B40063046000FDFF3A0020000700C482A90014
:1015C40020C0B300AAFF070009407800A8FF070065
:1015D4000B04E000120032003A407800A4FF070038
:1015E4008944E8006F8064000A003A00C482A800BD
:1015F400A7FF07000008A300FDFF3A000F00070043
:10160400C482A90020C0B30099FF070009407800F4
:1016140097FF07000844E80088CF5500EEFF3A0022
:10162400C482A8009AFF07000008A300FDFF3A0047
:101634004F05BE004F04BE0000000600C482A9008E
:1016440060C0B3008AFF0700C482A800000006003F
:10165400D10220008080400062C0B300A0CFB3005C
:1016640092FF0700000006004137210051000700E7
:1016740075D3BF004800DD000100700000000600C3
:10168400FDD3BF000000D100000006008180FB00F4
:10169400C208DD0000000600868040004C00070000
:1016A4008401700000000600904090008180FB00DF
:1016B40020409000EFFF3700114290000482FB00AD
:1016C400214090004800DD00040170003142900088
:1016D4000482FB00414090004800DD00840170005A
:1016E4000000060030C7B300FFF3B700C0C2B30068
:1016F40000F4B700000006009140780082C060004A
:1017040080C0700001007800000006002C00070073
:101714007410900000000600008040004237210051
:1017240002065000000006004800DD00F10F200012
:101734008185650080857500000006004237210020
:10174400828040002200070084017000820F55004F
:10175400838F5D00000006004037210080044600AE
:10176400180020008C467800000006000080FB0072
:1017740001F02F0001056500000575000DC0E800AB
:10178400000006004800DD00F20F2000020565009D
:101794000005750063C04600000006000080FB00E1
:1017A40004F02F00848565008085750064C04600C0
:1017B40000000600914078008180FB0000000600D4
:1017C40080C0700001007800FDF3B700000006003F
:1017D4001182FB00114090004800DD0004017000FC
:1017E400214290000482FB00314090004800DD005B
:1017F400000006007C17E20003003A0010002000FD
:10180400E0BB88005CF6EF005CD6BF00E14F40000F
:1018140003003200F6CC0200000000005CF6EF008A
:101824002F0307006076EF006096A8006036A800DA
:10183400000006005CD6BF00E14F40000300320008
:10184400F6CC0200000000005CF6EF005E36EF000C
:10185400000006005E16E20002003A0020030700C2
:101864006016A90000000600F0B280000000E0004D
:1018740001003200100020000000060000B38000C8
:10188400610060000000060000B380006200600098
:10189400020032006036A90010002000000006009B
:1018A40000B380004300DE00F5FF37001203070099
:1018B40000000600889FBE008A9FBE008C9FBE0069
:1018C400F2B280000080EB008080EB000200400058
:1018D400E0804800EB0F5000E08F58000E013E00FE
:1018E400006001000B003700120037003900370098
:1018F4004400370059003700AE003700D5003700E8
:10190400E6003700D3003700E4003700D100370089
:10191400E2003700030307005CCB02000000000074
:101924005CF6B700E14F4000FB00320020002000CD
:10193400F0B28800C003200050B388006C36EF007A
:101944008676EF006016A9006056A900B460020014
:10195400000000000000E000EF0032005CD6BF0091
:1019640034CD020000000000B1122000810F5000AD
:10197400E900360001B380004408DE000080EA007C
:10198400610060004400DD000140A100808070001F
:1019940001B38800E8020700F10F2000FE0C0200EA
:1019A400000000008000EB0010C0B300E20107005B
:1019B4005C00020001000000E50207000EC2020004
:1019C40000000000EE02070030002000F0B28800A2
:1019D400D10037005CD6BF001ECE0200000000001C
:1019E400910F2000810F5000220036006076A8007D
:1019F400CD000700E24F5000C7003A00400020002D
:101A0400F0B288005CD6BF0034CD020000000000B4
:101A140011102000810F5000BF003600C6020700DD
:101A24008180E900FE0C0200000000008000EB0051
:101A340030C0B300C00107005C00020001000000D8
:101A4400C30207000EC2020000000000CC0207001F
:101A540050002000F0B28800AF0037005CD6BF0011
:101A64001ECE020000000000910F2000810F5000E4
:101A74000F003E005C00020001000000CF020700DE
:101A8400A500340030B3800041B38000F20320008D
:101A9400820F5000E08F58009D003E00000040007F
:101AA4008180480030B3880041B388009800370033
:101AB4009D000700E54F50008A003A005CD6BF0045
:101AC400F6CC0200000000005CF6EF005C000200AF
:101AD40001000000BF0207006016A80033B48000B4
:101AE4000308A30001003200830207000328A300B7
:101AF4000A003200D0B38000E1B3800006E8B700EA
:101B04004801DE000200780007E8B7000100780011
:101B140008E8B7004808DE0009E8B7000318A30086
:101B24000A003200B0B38000C1B380000AE8B700F5
:101B34004801DE00020078000BE8B70001007800DD
:101B44000CE8B7004808DE000DE8B7000338A3002E
:101B540008003200F0B380000EE8B7004800DE0051
:101B64000FE8B70000B4800010E8B7004800DE00BA
:101B740011E8B7000040EB0012E8B70013E8B70023
:101B840014E8B70015E8B7000348A3006200320068
:101B940010B4800012E8B7004800DE0013E8B70074
:101BA40020B4800014E8B7004800DE0015E8B70050
